:100000000C94661A0C946CEE0C9441EE0C9416EE63
:100010000C94EBED0C94C0ED0C9495ED0C946AED02
:100020000C943FED0C94971A0C94971A0C94971A11
:100030000C94971A0C94971A0C94971A0D94C6085E
:100040000C94971A0C94971A0C94971A0C94971A6C
:100050000C94971A0C94971A0C94971A0D946F306D
:100060000C94971A0C94D2F10C94A8F10C94971A52
:100070000C94971A0C94971A0C94971A0C94971A3C
:100080000C94971A0C94971A0C94971A0C94971A2C
:100090000C9442F70C94B8F60C94FAF60D945E0AA0
:1000A0000C94971A0C94971A0C94971A0C94971A0C
:1000B0000C94971A0C94971A0C94971A0C94971AFC
:1000C0000C94971A0C94971A0C94971A0C947EF12E
:1000D0000C9454F10C94971A0C942AF10C9400F19E
:1000E0000C94971A07634236B79BD8A71A396856FB
:1000F00018AEBAAB558C1D3CB7CC5763BD6DEDFD4A
:10010000753EF6177231BF000000803F0800000006
:10011000BE922449123EABAAAA2ABECDCCCC4C3EFC
:1001200000000080BEABAAAAAA3E00000000BF00EB
:100130000000803F0000000000084178D3BB4387E7
:10014000D1133D190E3CC3BD4282AD2B3E68EC82FB
:1001500076BED98FE1A93E4C80EFFFBE01C4FF7F80
:100160003F00000000000C9476A70D9451240C94DD
:100170002A1C0C9445E80C9471E90C94D1340C942D
:10018000EDFF0C9451260D94B5190D940F240C9489
:100190004FD90C94F7B30C946D6E0C9413BB0C9464
:1001A000EFE90C94AC6D0C941A430C94E42A0C9473
:1001B0005BD90D94961A0C9404780C949C7A0C9448
:1001C0007F5E0D941B230D94C4310C94B2B20C9439
:1001D0009CAB0C94B0A70C94861C0C9447B70C9461
:1001E0005AC80C9460560C9445680D9460240C9485
:1001F000BF770D94BF2A0C94C4DD0D9447240C9452
:100200001DFD0D94A71A0C9475AF0C94B3B70C9404
:10021000F5300C9483A70C943B350C940AA30C94F2
:1002200056AB0C9472270C94CD780C94CDE90C94B9
:10023000321C0C946A5E0C94E7410C94EB370C94DE
:10024000551B0C9469D90C940C300C94BBE60C949F
:10025000A8C80D9419240C94A6550C94CB550C9455
:10026000E9A60C9462680C940CAC0C946DEA0C94A6
:1002700080850C94AFD80D9473190D9413230C94AE
:1002800025480C9434230C94D0340C94EDE90D944F
:1002900077000C94B9A60C94355F0D945F040C9410
:1002A00011240C9438C70C9420310C9457F00C9402
:1002B00039DC0C94DD9F0C94AB410D944D230D94CF
:1002C000E41F0D943A230D9414080C94031C0C9411
:1002D000D2A70C949E9A0D9474240C9440A20D9471
:1002E000BF190C94944C0C949EE70C94BF6E0C9424
:1002F00063B50C9428B80C94BDB70C94097B0D948D
:10030000BE2A0C9406DC0C9459DC0C947EAA0C9446
:10031000AAB70D94811B0C94F8670C9452AB0D9402
:100320007E240C94D44C0C94BDAB0C94D0DC0C9477
:10033000E7300C946E6F0C94742F0C9442EA0C947A
:1003400013560D94D6130C94B6780C9454680C94F0
:10035000A2A70C948A1C0C941C410C9404BB0C9412
:100360000CB60C9485FF0D9405240C9404B10C94E8
:1003700083B10C9423200C9454440D941F230C94AB
:1003800071A10C94C8A30C94E2200C94FAB30D94C0
:100390001D140D9436230D9434140D94D02A0C940E
:1003A000F3780C940A300C943D350D94C9190C94D3
:1003B0002C1C0C949C1A0D9455190C94EC1F0C9445
:1003C0005ED90C940BA70C9469B50C94E5AB0C9416
:1003D000623F0C949E1B0C9484550C949E340D9497
:1003E00064070C945EAB0C94357A0C941FC30D9487
:1003F000EF130C9494560C94262A0C94B32F0C945F
:10040000AD780C944EAB0C9418740D946A240D9432
:10041000A0070C949F7B0C9448560C94E9EA0C942A
:1004200025A30C9474A30C94F0550C947AC20D94EB
:10043000CD2A0C94B7A60D9448230D94361B0C942A
:1004400004300C94B9E90C9478A60C94F1E80C945F
:10045000FE9A0C94A31A0C948AE70C9437790C94A6
:10046000BADB0C9466B50C9463790C94DA400C9466
:10047000DD300D949D190D94C71A0C947A1B0C94C1
:100480004B680C94796C0D9437010C9453EA0C94DE
:10049000143B0C9464FC0D94F91F0C944FA30C9422
:1004A00091A70D942B240C94D72A0C9432E70C942A
:1004B0007E260C94DE4F0D9432230C94B66F0C9470
:1004C000CCAA0C9427A80C948EA60C943DC80C942E
:1004D000A5260D94DD1F0C9466FD0C948E1C0C94C7
:1004E00018360C94A4E80D9440230C944AD80C942C
:1004F0008BC80D9428230C944CD90C94F81B0C94A5
:10050000E5EB0D94FE130C945DA30C949CDD0C9410
:10051000D2AB0C948C1C0C94E5240C942AB80C944B
:10052000477A0C94586F0C9472DC0C94EEA50C94E2
:10053000687B0C94B8C80C9473B40D9400200C9490
:10054000F42F0D94DD130C9444EA0C94CCE90C9434
:100550005CDB0C9427440C944CFC0C947E440C946F
:100560000DA60C9477FA0C9493350D944E230C94AD
:10057000C3D80C94841C0C94F9410C9439780C94D5
:10058000311B0C94E43A0C94B3E80C94DC4B0C94BF
:10059000A5370C944B410C94A7FC0C9437560C9443
:1005A00062AB0C9433A40C946CB40D9405010C94C0
:1005B00007A80C9400790C9436780C9415730C945D
:1005C0009DA70C94AC6E0C94281C0D9452230C9493
:1005D00059B80C94C42F0C94093B0C94301C0C9407
:1005E000D6D80C947D1B0C9438A30C9463A10C9466
:1005F000D1A50D94D3190C94EC740C9439AC0C94D3
:10060000FA780C94B3A30C948A430C94991A0C9422
:1006100094950C94892A0C9466AB0C94ADAE0C9412
:1006200069C80D94F8230C9498CA0D94D61F0C94A5
:10063000837B0D943D240C9452C30C9418550C9458
:1006400037AC0C943CFD0D942C230C94881C0C941A
:10065000C5780C9401EB0C94D0A70C9442E90C944F
:1006600027850C9452A70C94339C0C945DB50C9484
:1006700041D90D9465190D940D230C9442790C9475
:10068000A2430D9433240D94CF1F0C94996D0C94B8
:10069000C82C0C9448200C943F680D9423240C948F
:1006A000AAA60C94C4E90C94E3E90C9426300C94AB
:1006B000EBB70C946CD90C9493770C942B460C9458
:1006C000182F0C94562F0C9451B10D94481B0C9478
:1006D00067AB0C94FFE80C94ABC80C94386A0D948B
:1006E00022230C9429E90C9496DD0C943C350D944E
:1006F00017230C94D8B70D9488240D94AB190C943F
:1007000008300C948AD80C94D41C0C9490DB0C9474
:1007100060B50C94C6770C9435E70C944D2B0C9473
:10072000B2E90D9444230C94C9EA0C94C98C0C943E
:100730007CAB0D9492240C9466EA0C94EA1B0D9405
:10074000AC000C9409790C945C790C946ACA0C94F2
:100750004D790C94FFB70D94EC030C9403A60C9404
:1007600001620C94245F0C9418790C9443EA0C9465
:10077000B6A50C94362F0C94C6B70C94D02E0C94BE
:100780006AAB0C94D4780D945E000C949EE90C94A2
:10079000EBA50C94E9DC0C94CA6B0D9481190C94B4
:1007A000764C0C94B29A0C94F9790C9479990C9437
:1007B0007BE70C94D2340C94BA1F0C9468220C94EE
:1007C00073430C94C24C0C94F6A20C94802A0C94A3
:1007D000F2AD0D94F21F0C949FAA0C940DBB0D94D6
:1007E00000240C94A6AB0C9441C20C943BE90C94ED
:1007F0001D7A0C9488E90C941DB80C94D0E80C94E4
:10080000B0DC0C947ED90C94E9C20C9413B80C940F
:10081000A2DD0C946DEF0C94ACE70C94CF340C94E7
:10082000CADD0C94ED1B0C9475C70C9411AE0C949E
:10083000295F0C945CA70C946EB50C942DA20C94BB
:1008400033A70D940F390C94B9C70C94197B0C94F1
:10085000AE4C0C942E1C0C94E72D0D94CF000C94F0
:1008600033E70C9400B40C94BFAB0C94A2E90C9445
:10087000D9A60C9481FF0C94B9AA0C94FBC70C94D4
:10088000BE1B0C94FBAB0C945AAB0C94401B0C9409
:100890001EA70C9468CA0C9434E70D94B01A0C94FB
:1008A00089680C94F8E70C948B5B0C949AEA0C948E
:1008B00049250D9493190C94A2B10C94FFAB0C94A0
:1008C000EAAD0C94631B0C94B9AB0C94EDA24E41B1
:1008D0004E494E495459494E46CDCCCC3D0AD723BA
:1008E0003C17B7D13877CC2B329595E6241FB14F02
:1008F0000A000020410000C84200401C4620BCBE47
:100900004CCA1B0E5AAEC59D746364696E6F7073DA
:100910007578585B00203C3C200041433A0041433D
:100920003A2053657269616C207573656420627941
:10093000204143202D2064697361626C696E6720D9
:1009400073657269616C206C6F6767696E6720619F
:100950006E6420636D640041433A204F7574206FCC
:1009600066206D656D6F72790041433A20496E696A
:10097000743A200041433A2044652D496E69743A27
:1009800020004552520041433A20426164204352C4
:10099000430041433A204F4B00203E3E200041435C
:1009A0003A0041433A20506F6C6C696E67004143D6
:1009B0003A20556E6D75746500000000000000005F
:1009C0000000004F4E00000000000000004F4646AF
:1009D00000000000000000524553540000000000D9
:1009E00000544F47474C450000000048414C54001C
:1009F0000000000000584F4E0000000000000058AA
:100A00004F4646000000000000494E435245415306
:100A100045000044454352454153450000454E4181
:100A2000424C450000000044495341424C450000FF
:100A300000554E465245455A450000465245455AD6
:100A400045000000004155544F00000000000046E2
:100A5000414E5F4F4E4C5900004849474800000046
:100A60000000004D454449554D000000004C4F57D3
:100A700000000000000000484541545F434F4F4CC8
:100A80000048454154000000000000434F4F4C0017
:100A90000000000000445259000000000000005215
:100AA00047420000000000000048535600000000CC
:100AB0000000007261770071756569740073776971
:100AC0006E67006C6F636B00556E6B6E6F776E2098
:100AD0007375666669782000556E6B6E6F776E2051
:100AE000636D642000436F756E7465723A20004434
:100AF0004D582D4F757420496E69743A2000444D4D
:100B0000582D4F75742073746F703A2000417373C1
:100B100069676E65643A00444D58206374726C3A9C
:100B20002000693136000169333200027531360028
:100B3000037533320004693868000569386C0006B3
:100B4000753868000775386C000878313000093155
:100B50003030000A44656661756C74207365726993
:100B6000616C206D6F6465204E383120757365644B
:100B700000384531002600384E3100060038453235
:100B8000002E00384E32000E00384F31003600384B
:100B90004F32003E00374531002400374532002CEB
:100BA00000374F31003400374F32003C00374E31B0
:100BB000000400374E32000C00206164646564203C
:100BC0006279206E756D20004D4255533A200041E8
:100BD0006464696E67207265677320776974682042
:100BE000616374696F6E733A00416464696E672073
:100BF000726566657272656420726567733A00415A
:100C00006464696E672070726566657463682072DB
:100C10006567733A004D4255533A204D6F646275D3
:100C2000732074656D706C617465206E6F742066DE
:100C30006F756E643A20004D4255533A20496E76E6
:100C4000616C69642074656D706C6174652E002C34
:100C5000002C002C002C004D4255533A20636F6E3F
:100C6000666967206661696C65643A004D42555358
:100C70003A20636F6E666967206572726F72004D0D
:100C80004255533A20636F6E666967206C6F6164EA
:100C9000656420004D4255533A204F7574206F66AD
:100CA000206D656D6F7279004D4255533A20506F3B
:100CB0006C6C696E67206572726F7220004D4255D0
:100CC000533A204E6F7420737570706F7274656440
:100CD0002072656720747970650A004D425553444F
:100CE0003A2049676E6F726564202D2065717561C9
:100CF0006C2077697468207365747465642076610C
:100D00006C004D425553443A204D61707065643A11
:100D1000004D425553443A204E65737465644D61ED
:100D2000707065643A004C6173744B6E6F776E201F
:100D300076616C75653A2000536561726368696E0F
:100D400067207265673A2000206F7574206F6620F7
:100D500072616E6765206275666665722C206665D5
:100D6000746368696E670064656620726567232036
:100D7000004D425553443A20536561726368696E71
:100D8000672072656723003A002066726F6D2074D9
:100D900079706520004D425553443A2020676F74A6
:100DA00020002076616C3A0020004D42555320729D
:100DB00065733A20002076616C206E6F7420636842
:100DC000616E6765642E20436F6E74696E75650091
:100DD0004D4255533A003A20657175616C2074613B
:100DE00072676572742E003D004D4255533A0020E3
:100DF00076616C206368616E6765642E004D4255B4
:100E0000533A00204E6F773A00204C6173743A00D9
:100E1000202300207072656665746368200020528C
:100E200065672F636F696C206D7573742062652030
:100E3000696E740020696E7465726E616C207365F2
:100E40006E64206572726F72202D206E6F20726545
:100E5000672F636F696C0020696E7465726E616CD8
:100E60002073656E64206572726F72202D206E6F24
:100E70002074656D706C6174650020696E746572B4
:100E80006E616C2073656E64206572726F72202DC6
:100E9000206E6F2073746F7265004D425553443A53
:100EA00020656E64506F6C6C20004D425553443A7F
:100EB00020506F6C6C2000206E6F7420666F756E12
:100EC00064004D4255533A2020706172616D2000DC
:100ED0002073656E64696E672063616E63656C6C18
:100EE0006564004D4255533A2020706172616D2057
:100EF000004D4255533A2020002073656E642065F2
:100F000072726F722E20004D4255533A20200041DC
:100F100064642040563A20002056616C3A20004D0F
:100F2000425553443A207375666669783A00206FDB
:100F3000722073756666697820004D4255533A20D9
:100F40004E6F2074656D706C61746520666F7220E1
:100F5000004D6F746F723A2074696D656F7574001F
:100F6000556E6B6E6F776E20636D64004D6F746F9E
:100F7000723A20466F7263656420657865637574A4
:100F8000696F6E0056454E543A20636F6E6669670E
:100F9000206661696C65640056454E543A20696E5E
:100FA00069740056454E543A2050494420503D0043
:100FB00056454E543A2044652D496E697400564595
:100FC0004E543A204368616E2062616C616E6365C5
:100FD0003D00207365742052455645525345206D9F
:100FE0006F64650056454E543A205049443A2000FB
:100FF0002073657420444952454354206D6F6465E5
:101000000056454E543A205049443A20002073651A
:10101000742052455645525345206D6F6465005605
:10102000454E543A2050415353205049443A2000F1
:101030002073657420444952454354206D6F6465A4
:101040000056454E543A2050415353205049443A9B
:101050002000206F75743A00207365743A0020698F
:101060006E3A0056454E543A2000204F75743A00AF
:10107000205265713A0056454E543A2000206D3397
:10108000002066726F6D2000204D617820726571BE
:101090003A002066616E253A0020616374697665C6
:1010A00020563A0056454E543A20546F74616C20D5
:1010B000563A0056454E543A2076616C75652000CC
:1010C00041432061697220726F6F6D74656D703A73
:1010D000200056454E543A004143206D6F64653AF6
:1010E000200056454E543A004143206169722074F5
:1010F000656D703A200056454E543A005049443AC6
:1011000020616C726561647920696E697469616CD3
:10111000697A6564005049443A20496E76616C6989
:101120006420706172616D2061727261792E002C91
:10113000002C002C002C005049443A20636F6E664E
:101140006967206661696C65643A005049443A20D9
:10115000636F6E666967206572726F7200504944F2
:101160003A20636F6E666967206C6F616465642006
:10117000005049443A204F7574206F66206D656DAC
:101180006F7279005049443A2044652D496E697464
:101190002000203C414C4D3E0020443A0020493A7A
:1011A0000020503A0020696E3A00207365743A00BE
:1011B0005049443A20005049443A20496E76616CC7
:1011C000696420706172616D2061727261792E00B4
:1011D000536574206F757420746F2000205049444B
:1011E00020616C61726D2E20002050494420616C9A
:1011F00061726D3A20636C6F736564005049443AC4
:1012000020556E6B6E6F776E2073756666697820F9
:10121000005049443A20556E6B6E6F776E20636DB7
:1012200064200020536574706F696E743A005049F1
:10123000443A200020496E7075742076616C7565A3
:101240003A005049443A200020696E697400200039
:1012500050574D2D4F75742023002073746F70000C
:10126000200050574D2D4F75742023003D005069CC
:101270006E3A0020696E69740070696E23007265B1
:101280006C61794374723A20002073746F7000525D
:10129000656C61792D4F757420230072656C6179DE
:1012A0004374723A200069646C65006F666600687A
:1012B000656174696E670066616E00647279696E5B
:1012C0006700636F6F6C696E6700616374696F6E4E
:1012D0000020697320004F7574200072656C61797D
:1012E0004374723A2000556E6B6E6F776E20737583
:1012F00066666978200072656C61794374723A2081
:1013000000556E6B6E6F776E20636D6420007265A2
:101310006C61794374723A2000616374696F6E0086
:1013200072656C61794374723A200053686F77007C
:1013300020636D643D002D000000000000636D64BB
:101340000000736574000076616C000064656C00D9
:10135000004853560000524742000066616E00008C
:101360006D6F6465006374726C006875650000736E
:101370006174000074656D70007261770000200078
:101380002E00696E00735F6F7574006D79686F6D04
:1013900065004354524C2F657865633A204F75744D
:1013A0004F664D656D6F72793A2000202D3E20000A
:1013B0004D5154543A2000202D3E2000456D697453
:1013C0003A203C00202D3E20004974656D436D6439
:1013D0003A2000202D3E20004974656D3A200020FF
:1013E0006661696C65643A004D6F64627573206F65
:1013F0007020004D423A206F6B003D004D423A2074
:101400005643230020636D643D003D004D423A2069
:1014100056435F6865617423004D423A204E6F74F5
:1014200020737570706F72746564207265672074C4
:101430007970650A002056616C3A30780020543A81
:1014400000205265673A3078004D423A204164648A
:10145000723A00444D58000000000000444D5852BC
:101460004742570000444D58524742000000505731
:101470004D0000000000004D42555344494D00000E
:10148000544845524D4F00000052454C4159000010
:10149000000047524F555000000000564354454D40
:1014A000500000004D425553564300000041434850
:1014B0004149455200005350494C45440000004DFD
:1014C0004F544F52000000005049440000000000FB
:1014D000004D425553000000000055415254425205
:1014E00044470052454C415950574D00444D5852C5
:1014F000474257570056454E545300000000454C94
:10150000455641544F5200434F554E5445520000EA
:1015100048554D0000000000004D455243555259BA
:10152000000020002D3E00436F6E76657274696E78
:101530006720002D3E0057726F6E672041737369FC
:10154000676E6D656E742000524742783A20002025
:10155000764C6576656C3A0020436F6E76563A009D
:1015600020436F6E76533A0020486F743A00436F01
:101570006C643A0020436F6E766572746564205621
:101580003A00436F6E76657274656420533A002D9D
:101590003E0057726F6E672041737369676E6D65A9
:1015A0006E7420002D3E0057726F6E67204173737A
:1015B00069676E6D656E7420004D41503A2076610A
:1015C0006C206D617070656420746F2020004D4147
:1015D000503A2076616C75652061626F7665207285
:1015E0006967687420626F756E64200020697320DB
:1015F00062656C6F77206C65667420626F756E64CF
:1016000020004D41503A2076616C756520004D41B7
:10161000503A20636D64206D617070656420746F52
:101620002000000000000000000000004F4E0000FD
:101630000000000000004F464600000000000000CF
:1016400052455354000000000000544F47474C459A
:101650000000000048414C54000000000000584FBA
:101660004E00000000000000584F464600000000F9
:101670000000494E43524541534500004445435202
:10168000454153450000454E41424C450000000095
:1016900044495341424C45000000554E4652454591
:1016A0005A450000465245455A4500000000415544
:1016B000544F00000000000046414E5F4F4E4C5911
:1016C0000000484947480000000000004D454449DB
:1016D000554D000000004C4F570000000000000076
:1016E000484541545F434F4F4C004845415400002A
:1016F00000000000434F4F4C000000000000445227
:1017000059000000000000005247420000000000A5
:10171000000048535600000000000000205375668A
:10172000663A002041543A0053746F7070696E67D6
:1017300020496E7075747300206973200044656CD5
:101740006574696E6720636F6E662E2052414D206E
:101750007761733A0053746F70706564006E6F74D4
:1017600068696E6720746F2073746F700053746FB4
:101770007070696E67206368616E6E656C73202E91
:101780002E2E0043616E206E6F7420636C65616E57
:10179000202D206C6F636B6564004D5154543A20CA
:1017A000436F6D706C6574652E2052656D6F766544
:1017B00020746F706963200024636F6D6D616E64C7
:1017C000004D5154543A20436C65616E557020723F
:1017D000657461696E656420746F706963200022AE
:1017E0000022004F75744F664D656D6F7279210050
:1017F0005D20003A5B004D5154543A005D00456D48
:101800007074793A205B000A003A004D41433A0077
:10181000476F7420495020616464726573733A00A5
:10182000276970205B69705B2C646E735B2C677733
:101830005B2C7375626E65745D5D5D5D27202D2088
:10184000736574207374617469632049500A00469B
:1018500061696C656420746F20636F6E666967757B
:1018600072652045746865726E6574207573696E63
:101870006720444843502E20596F752063616E20C5
:10188000736574206970206D616E75616C6C79216F
:1018900000204D41534B3A002047573A0020444E18
:1018A000533A004C6F616465642066726F6D206608
:1018B0006C6173682049503A000A7573657320445F
:1018C0004843500A005374617274696E67206C61FA
:1018D0006E004D5154543A2074727969796E6720C4
:1018E0006E656E78742062726F6B6572004D515434
:1018F000543A20546F6F206D616E7920636F6E6E65
:10190000656374696F6E206572726F72732E2052F8
:10191000657374617274204C414E0020747279209A
:10192000616761696E20696E2035207365636F6E33
:101930006473004D5154543A206661696C65642C9F
:101940002072633D004D5154543A204177616974CF
:10195000696E6720666F722072657461696E656476
:1019600020746F7069637300636F6E6E6563746576
:10197000642061732000202E2E2E00207573657266
:101980003A003A000A4D5154543A20417474656D3E
:101990007074696E6720636F6E6E656374696F6ED5
:1019A00020746F2000646973636F6E6E6563746585
:1019B00064005573696E67204D51545420706173F3
:1019C00073776F72642066726F6D20636F6E6669E5
:1019D0006700446576696365204E616D653A004D28
:1019E0005154543A204174206C65617374206465CD
:1019F00076696365206E616D6520616E6420627238
:101A00006F6B6572204950206D757374206265207C
:101A1000636F6E6669677572656400246E6F6465D6
:101A200073004F4E2C4F46462C48414C542C524587
:101A300053542C584F4E2C584F46462C544F474722
:101A40004C450024666F726D617400656E756D00A3
:101A50002464617461747970650068737600636FE3
:101A60006C6F7200302D32353500696E74656765B4
:101A70007200666C6F617400332E302E3100246862
:101A80006F6D696500757074696D652C667265654A
:101A90006865617000303864656436325F323032B8
:101AA000362D30312D3039004C69676874487562C5
:101AB0002000246E616D6500526562696E6420735A
:101AC0007563636573732E20495020616464726589
:101AD00073733A004572726F723A20726562696E72
:101AE00064206661696C0052656E65776564207379
:101AF0007563636573732E20495020616464726559
:101B000073733A004572726F723A2072656E657730
:101B10006564206661696C000A4E6F206C696E6BAB
:101B200000436F6E74696E75652077697468207004
:101B3000726576696F75736C79206C6F616465642A
:101B400020636F6E666967003330732045455052DD
:101B50004F4D206973206E6F742072656C6F6164E5
:101B600065642E205265626F6F74004D5154543A73
:101B700020416363657074696E6720636F6D6D618A
:101B80006E64732E2E2E0A004E6F204D5154542039
:101B9000636F6E66696775726564004C6F61646936
:101BA0006E6720636F6E6669672066726F6D207066
:101BB0006F7274616C2064697361626C65642E205D
:101BC00075736520676574204F4E20746F20656EB5
:101BD00061626C6500436F6E666967206973207689
:101BE000616C696400436F6E74696E756520776916
:101BF00074682070726576696F75736C79206C6F8C
:101C00006164656420636F6E66696700536574750F
:101C100070204F5441004D5154543A207365742044
:101C200066697273742062726F6B657200437572BD
:101C300072656E74204C414E20636F6E6669672832
:101C400069702C646E732C67772C7375626E657483
:101C5000293A000A55736520746865736520636FBF
:101C60006D6D616E64733A202768656C7027202D56
:101C7000207468697320746578740A276D61632025
:101C800064653A61643A62653A65663A66653A3017
:101C900030272073657420616E642073746F7265E1
:101CA000204D41432D6164647265737320696E2019
:101CB000454550524F4D0A276970205B69705B2C77
:101CC000646E735B2C67775B2C7375626E65745DF5
:101CD0005D5D5D27202D20736574207374617469C8
:101CE000632049500A277361766527202D20736190
:101CF00076652063757272656E7420636F6E6669B7
:101D00006720696E204E5652414D3B204F4E7C4F0E
:101D10004646202D20656E61626C652F6469736193
:101D2000626C65206175746F736176650A276765FB
:101D30007427205B636F6E66696720616464725DFF
:101D400027202D2067657420636F6E6669672066A3
:101D5000726F6D207072652D636F6E666967757244
:101D600065642055524C20616E642073746F7265F7
:101D700020616464722C204F4E7C4F4646202D20FB
:101D8000656E61626C652F64697361626C65206465
:101D90006F776E6C6F6164206F6E20737461727404
:101DA00075700A276C6F616427202D206C6F616449
:101DB00020636F6E6669672066726F6D204E5652A3
:101DC000414D0A2770776427202D20646566696E6F
:101DD0006520616E642073746F7265204D51545498
:101DE0002070617373776F72640A276F7461707704
:101DF0006427202D20646566696E6520616E64200D
:101E000073746F72652048545450204150492070BB
:101E1000617373776F72640A276C6F67205B7365F9
:101E20007269616C5F6C6F676C6576656C5D205B79
:101E30007564705F6C6F676C6576656C5D27202DCF
:101E400020646566696E65206C6F67206C657665D9
:101E50006C2028302E2E37290A276B696C6C2720BE
:101E60002D2074657374207761746368646F670AEA
:101E700027636C65617227202D20636C6561722079
:101E8000454550524F4D0A2773656172636827209C
:101E90002D2073656172636820312D77697265202A
:101EA0006465760A277265626F6F7427202D207231
:101EB00065626F6F7420636F6E74726F6C6C6572A5
:101EC00000536F6674207265626F6F74696E672E5F
:101ED0002E2E00206E657700206973200031575444
:101EE0003A003157543A20536561726368696E67EE
:101EF000206465760052414D3D000A312D776972AC
:101F00006520000A6D71747420000A6D6F6462753B
:101F100073207632000A6D6F64627573207631200B
:101F2000282B29000A696E7075747320000A697481
:101F3000656D7320000A436F6E666967757265642C
:101F40003A002F00496E3A2000496E697469616C4D
:101F5000697A696E6720496E7075747300315754E1
:101F60003A207365747570207265736F6C7574694F
:101F70006F6E20003157543A204453323438322D9A
:101F8000313030206E6F742070726573656E74002E
:101F90003157543A204453323438322D31303020C6
:101FA00049324320726573746F726564003157540F
:101FB0003A20427573207265736574206572726F82
:101FC00072003157543A204275732052657365741C
:101FD00020646F6E65003157543A204453323438D0
:101FE000322D3130302070726573656E742C207222
:101FF00065736574004572726F7220312D772069A8
:102000006E6974003157543A204453323438325F89
:102010003130305F4932435F544F5F31575F425236
:102020004944474520696E697400444D584F7574A2
:102030002E20467265653A00444D58696E204275FF
:102040006666657220616C6C6F6320657272004910
:102050006E697420696E2063683A003B003D005051
:10206000696E3A003B003D4C4F5700546865726DF5
:102070006F3A004F6E652077697265205265616422
:10208000790A00467265653A00444D58206F7574B0
:1020900020737461727465642E204368616E6E658E
:1020A0006C733A2000444D5820696E20737461723D
:1020B0007465642E204368616E6E656C733A0042ED
:1020C000726F6B65727320636F6E66696775726598
:1020D000643A004170706C79696E6720636F6E6658
:1020E0006967004C6F6164656420455441473A005C
:1020F0004E6F2073746F72656420636F6E666967DC
:10210000004C6F616465642066726F6D20454550B8
:10211000524F4D006C6F6164206661696C656400AC
:102120004A534F4E206465746563746564004C6F58
:102130006164696E6720436F6E6669672066726FBF
:102140006D20454550524F4D00436F6E66696720C4
:102150006175746F736176653A000A5379736C6FB9
:1021600067206465627567206C6576656C3A00531C
:10217000657269616C206465627567206C6576655F
:102180006C3A0053617665640A0053657420647983
:102190006E616D69632049500A004F5441205061BF
:1021A0007373776F726420757064617465640A007C
:1021B0004E6F204950206164726573730020536133
:1021C000766564004C6F6164696E672048545450B2
:1021D00020636F6E666967206F6E2073746172741E
:1021E00075703A00000000000000000000004F4E33
:1021F00000000000000000004F4646000000000004
:10220000000052455354000000000000544F47475F
:102210004C450000000048414C5400000000000004
:10222000584F4E00000000000000584F4646000086
:1022300000000000494E43524541534500004445CB
:102240004352454153450000454E41424C45000034
:10225000000044495341424C45000000554E46524F
:1022600045455A450000465245455A450000000084
:102270004155544F00000000000046414E5F4F4E54
:102280004C590000484947480000000000004D45F7
:102290004449554D000000004C4F5700000000001D
:1022A0000000484541545F434F4F4C00484541545E
:1022B000000000000000434F4F4C000000000000F1
:1022C0004452590000000000000052474200000044
:1022D0000000000048535600000000000000636F3B
:1022E000756C64206E6F742070617273653A2000A3
:1022F000557064617465640A00454550524F4D2025
:10230000636C65617265640A004D515454205061DC
:102310007373776F726420757064617465640A000A
:102320002B002D00455461673A2000476574204515
:102330005441473A2000485454502F312E31002543
:10234000733A2025730D0A0020485454502F312E23
:10235000310D0A486F73743A2025730D0A41636387
:102360006570743A202A2F2A0D0A436F6E6E6563DA
:1023700074696F6E3A20636C6F73650D0A00257384
:102380000020000D0A00474554006661696C6564D1
:1023900020746F20636F6E6E6563740A004552523D
:1023A0004F523A2053657276657220726574757269
:1023B0006E65642000436F6E666967206E6F7420DF
:1023C0006368616E6765640A00446F6E652E0A007B
:1023D000436F6E6669672070617273696E6720660D
:1023E00061696C65640A004765742061626F72748C
:1023F000656400676F7420436F6E6669670A0068E2
:1024000074747020726574636F6465200066726511
:10241000652000436F6E666967205552493A20680F
:102420007474703A2F2F002044656661756C7420B7
:10243000636F6E6669672073657276657220757367
:1024400065643A20006C617A79686F6D652E7275EB
:10245000000A282D294352595054000A282D29508A
:10246000554C5345206F6E2050494E3132000A289A
:102470002D2943414E000A282D294D4552435552DE
:1024800059000A282B294D554C544956454E5400A5
:102490000A282B2950574D5F52454C4159000A28B4
:1024A0002D294D444E53000A282D2955415254429E
:1024B0005249444745000A282D295359534C4F4748
:1024C000000A282B29504944000A282D294D435041
:1024D0003233303137000A282D294152544E4554A9
:1024E000000A282D294F5441000A282B295350490E
:1024F000204C4544000A282B294D4F544F5220436D
:102500005452000A282B2941432048414945522072
:102510006F6E2053657269616C32000A282B294363
:10252000435338313120262048444331303830007D
:102530000A282B29524553544152545F4C414E5F57
:102540004F4E5F4D5154545F4552524F5253000A03
:10255000282D294841524452455345542C20757327
:10256000696E6720736F6674000A282B29434F55E4
:102570004E544552000A282B29444854000A282B5F
:10258000294453323438322D313030000A282B2977
:102590004F57495245000A282D2949504D4F444272
:1025A0005553000A282B294D4F444255532030786B
:1025B00030362061742053657269616C332073700A
:1025C0006565643A39363030000A282B2941444188
:1025D0004652554954204C4544000A282B29444D65
:1025E00058000A282B2957697A6E657435313030C6
:1025F000000A282B294672656552616D2070726948
:102600006E74696E67000A282B2957415443484469
:102610004F47000A282B29434F4E54524F4C4C49E8
:102620004E4F000A4669726D77617265204D4143D5
:1026300020416464726573732064653A61643A6230
:10264000653A65663A66653A3037006C617A796852
:102650006F6D652E7275000A436F6E666967207331
:1026600065727665723A003230313130334C002079
:10267000432B2B2076657273696F6E3A0030386495
:10268000656436325F323032362D30312D303900CC
:102690000A4C617A79686F6D652E7275204C696796
:1026A000687448756220636F6E74726F6C6C6572CB
:1026B0002000204F464600204F4E002042595041F6
:1026C000535300536176656420746F204545505222
:1026D0004F4D00536176696E6720636F6E66696760
:1026E00020746F20454550524F4D2E2E00434353CA
:1026F0003831313A20416C726561647920696E69C4
:102700007469616C697A6564004343533831313AC6
:1027100020496E6974206572726F722000434353C2
:102720003831313A20496E697400484443313038B9
:10273000303A20416C726561647920696E69746910
:10274000616C697A656400446576696365205365E8
:102750007269616C204E756D6265723D0020446542
:10276000766963652049443D3078004D616E756639
:10277000616374757265722049443D307800484445
:1027800043313038303A20496E69742E2000432C92
:102790002052483D00484443313038303A20537489
:1027A000617475733D00484443313038303A204EEF
:1027B0006F7420696E697469616C697A6564004D33
:1027C0007367496E76616C69640052656164526535
:1027D00067496E76616C6964004D6561734D6F6425
:1027E00065496E76616C6964004D61785265736904
:1027F0007374616E636500486561746572466175E6
:102800006C7400486561746572537570706C790002
:102810004343533831313A204572726F722000437E
:1028200043533831313A204661696C656420746FD6
:1028300020676574204552524F525F4944207265AB
:102840006769737465722E005D20626173656C69DF
:102850006E655B005D2074564F435B0020434F3232
:102860005B006363733831313A2064617461206EB8
:102870006F7420617661696C61626C65006363737B
:10288000383131206E6F7420696E697469616C69CA
:102890007A656400556E6B6E6F776E207375666631
:1028A00069782000556E6B6E6F776E20636D6420C3
:1028B00000636C724374723A2000444D58494E3A9A
:1028C00000454F46003D00494E3A002500C2B04346
:1028D00020483D0020444854323220747970652EDF
:1028E00020543D00494E3A00204E6F20656D6974BA
:1028F0002064617461210020436F756E74657220DD
:10290000747970652E2076616C3D00494E3A002046
:10291000436F756E74657220747970652E20494E10
:10292000434F525245435420496E7465727275701C
:1029300074206E756D626572212121004952513AF1
:1029400000416374697661746520696E200041639B
:1029500074697661746520696E20002D3E00200048
:1029600023002D3E00200050656E6465643A2023EC
:10297000002D3E00456D69743A002D3E00456D699D
:10298000743A002D3E00456D69743A002D3E0045B5
:102990006D69743A003D004C454741435920494E0A
:1029A0003A0020666F7220286D73293A0043545212
:1029B0004C3A205363686564756C6520636D6420D0
:1029C00000206D730020666F7220004354524C3A11
:1029D0002041726D656420002044697361726D65E9
:1029E00064004354524C3A20002074696D653A00EB
:1029F0004354524C3A205265733A004354524C3A75
:102A0000206D6F6D656E74617279206576656E7488
:102A1000002054533A0020543A00544845524D3A4D
:102A200000436C65616E696E6720616C61726D2038
:102A3000003D0050696E3A004354524C3A20436FB7
:102A40006D6D616E6420626C6F636B65642062798A
:102A500020647269766572004354524C3A204F4E9E
:102A60003A416C7265616479204163746976650AE4
:102A7000004354524C3A2048414C543A416C7265E0
:102A800061647920496E6163746976650A00435414
:102A9000524C3A20584F4E3A2044697361626C653B
:102AA000640A004354524C3A20584F4E3A416C72DB
:102AB00065616479204163746976650A0043545204
:102AC0004C3A20584F464620736B69707065642EEF
:102AD000205072657620636D643A004354524C3A3C
:102AE000205475726E6564206F66662066726F6D25
:102AF0003A004354524C3A20526573746F726564C5
:102B00002066726F6D3A004354524C3A2049676E0A
:102B10006F7265642C206368616E6E656C20636DF6
:102B2000643D0020457865633A004354524C3A2096
:102B30004163746976653A004354524C3A204841E7
:102B40004C543A416C726561647920496E616374DA
:102B50006976650A004354524C3A20584F4E3A2049
:102B600044697361626C65640A004354524C3A20B4
:102B7000584F4E3A416C72656164792041637469C3
:102B800076650A004354524C3A20584F464620730B
:102B90006B69707065642E205072657620636D6479
:102BA0003A004354524C3A205475726E6564206F5B
:102BB00066662066726F6D3A004354524C3A20525A
:102BC0006573746F7265642066726F6D3A00446954
:102BD0007361726D696E67206E6F742061757468C1
:102BE0006F72697A6564004354524C3A20636F6D8A
:102BF0006D616E64206A75737420666F7220004385
:102C000054524C3A204E6F7420656E6F7567682081
:102C10006D656D6F727920666F722067726F757067
:102C2000206F7065726174696F6E00496E76616CB9
:102C300069642061726700496E76616C6964206125
:102C4000726700496E76616C696420617267004347
:102C500054524C3A20556E6B6E6F776E20737566CA
:102C600066697800536B697070696E67207363687A
:102C70006564756C65642067726F75702065786532
:102C800063004354524C3A206368616E6E656C2059
:102C900066726F7A656E004354524C3A20636861E5
:102CA0006E6E656C2066726F7A656E00536B69702C
:102CB00070656420686F6D69652073747566660061
:102CC0002000205375623D00204974656D3D00432E
:102CD00054524C3A2052414D3D004354524C3A20FC
:102CE0004F75744F664D656D6F72793A2000282DCF
:102CF000292000282B2920002076616C7565206929
:102D000073200020756E6B6E6F776E0A005D3D005C
:102D10005B0020696E76616C696400200041435459
:102D20004956453A00206F6B003A00206661696C95
:102D30006564003A005265747279696E6720564383
:102D400054454D5020434D440A00526574727969D0
:102D50006E6720564320434D440A005265747279D1
:102D6000696E67206D6F6462757320434D440A007D
:102D70005265747279696E6720434D440A0020657C
:102D800072726F723D004D423A20706F6C6C696ECA
:102D90006720002056616C3A20004D423A20004DD9
:102DA000423A204E6F7420737570706F7274656450
:102DB0002072656720747970650A004D423A207070
:102DC0006F6C6C696E672064696D6D657220004D73
:102DD000423A20496C6C6567616C20617267756D61
:102DE000656E74730A00206572726F723D004D4209
:102DF0003A20706F6C6C696E6720504920002D007E
:102E00004D423A2050492056616C203A004D423ADA
:102E100020706F6C6C696E6720504920004D423AFB
:102E200020706F6C6C696E6720464D206661756C12
:102E3000742000206572726F723D004D423A20701E
:102E40006F6C6C696E6720002D004D423A20464D34
:102E50002056616C203A004D423A20706F6C6C69CC
:102E60006E6720464D20004354524C2F706F6C6C9F
:102E70003A204F75744F664D656D6F72793A200038
:102E8000207365632072656D61696E696E670053BA
:102E900074617475732064656666657265640A00A2
:102EA0002D3E005075623A20002D3E005075623A6A
:102EB00020002D3E005075623A2000000000000006
:102EC000636D640000736574000076616C000064DB
:102ED000656C00004853560000524742000066618E
:102EE0006E00006D6F6465006374726C00687565D8
:102EF0000000736174000074656D7000726177008A
:102F0000002D3E005075623A20002D3E0050756243
:102F10003A200053454E445354415455533A20559A
:102F20006E6B6E6F776E20636D64200A0000000088
:102F3000000000000000004F4E00000000000000F4
:102F4000004F464600000000000000524553540068
:102F50000000000000544F47474C45000000004867
:102F6000414C54000000000000584F4E000000008B
:102F7000000000584F4646000000000000494E4344
:102F80005245415345000044454352454153450095
:102F900000454E41424C4500000000444953414227
:102FA0004C45000000554E465245455A45000046E6
:102FB0005245455A45000000004155544F0000005D
:102FC00000000046414E5F4F4E4C590000484947B3
:102FD000480000000000004D454449554D000000E8
:102FE000004C4F5700000000000000484541545F6E
:102FF000434F4F4C0048454154000000000000433F
:103000004F4F4C00000000000044525900000000E7
:1030100000000052474200000000000000485356E4
:10302000000000000000003157543A204275732020
:103030007265736574206572726F72003157543A0D
:103040002042757320526573657420646F6E65004D
:103050003157543A204453323438322070726573F9
:10306000656E742C2072657365740049324320527A
:103070006573657400005EBCE2613FDD83C29C7EC7
:1030800020A3FD1F419DC3217FFCA2401E5F01E3E1
:10309000BD3E6082DC237D9FC1421CFEA0E1BF5D7E
:1030A0000380DE3C62BEE0025CDF81633D7C22C0C7
:1030B0009E1D43A1FF4618FAA427799BC584DA38E0
:1030C00066E5BB5907DB856739BAE406581947A599
:1030D000FB7826C49A653BD987045AB8E6A7F91B42
:1030E00045C6987A24F8A6441A99C7257B3A64867F
:1030F000D85B05E7B98CD2306EEDB3510F4E10F2AC
:10310000AC2F7193CD114FADF3702ECC92D38D6F48
:1031100031B2EC0E50AFF1134DCE90722C6D33D115
:103120008F0C52B0EE326C8ED0530DEFB1F0AE4C2E
:103130001291CF2D73CA947628ABF517490856B46F
:10314000EA6937D58B5709EBB536688AD495CB2910
:1031500077F4AA4816E9B7550B88D6346A2B7597C9
:10316000C94A14F6A8742AC896154BA9F7B6E80AF6
:1031700054D7896B35436F6E6E65637465642E003A
:10318000436F6E6E2E2061626F72746564003E3E06
:103190002000496E76616C696420636F6D6D616EAD
:1031A0006400000020002300260029002C002F00CE
:1031B0003200000100000301060109013E3E3E000D
:1031C0004E6F204D414320636F6E6669677572656F
:1031D000643A20736574206669726D776172652741
:1031E00073204D41430A00454550524F4D207369AD
:1031F000676E6174757265206F6B00496E697469E2
:10320000616C697A696E6720454550524F4D2E00BA
:103210002072656164206572726F7220666F722021
:10322000003E2000203C003157543A003157543AB8
:10323000206E6F7420696E6974003157543A2042D1
:103240005553592074696D656F7574003157543A40
:10325000204453323438325F4552524F525F434F0D
:103260004E464947003157543A20312D77697265EF
:103270002073686F727465640072656164790024FC
:10328000737461746500757074696D65006672654C
:1032900065686561700024737461747300204578FB
:1032A00070697265640A00202D746172676574200C
:1032B0007A6F6E652D0020416C61726D20457870CB
:1032C000697265640A0020636D643A002043757278
:1032D0003A00205365743A002054696D65723A00D3
:1032E000204C6F636B733A0052414D3D0000002249
:1032F00000250028002B002E0031003400020100C0
:1033000000050108010B0100000A0B02090C0D0E5B
:103310000807030401000000000000000000000096
:10332000000000000000000000000000000000009D
:10333000000000121110000000000000000000005A
:10334000000000000000000000000000004D425599
:10335000533A204164642040533A20000000210089
:10336000240027002A002D00300033000101000056
:10337000040107010A010102102020080810204062
:103380001020408002010201080402010102040829
:1033900010204080804020100804020180040201B7
:1033A0008040201008040201080402010102040800
:1033B000102040800102040810204080050505050A
:1033C000070508080808020202020A0A080804049D
:1033D00004040101010101010101030303030303CB
:1033E0000303040707070C0C0C0C0C0C0C0C02025A
:1033F000020206060606060606060B0B0B0B0B0B57
:103400000B0B556E73706563696669656420657240
:10341000726F722E0047454E455249435F455252E6
:103420004F5200494E5445524E414C5F4552524F07
:1034300052004932435F4552524F520049445F4562
:1034400052524F5200535543434553530043435345
:103450003831313A200057726F6E67207061796C95
:103460006164004D5154543A204354524C2F7478A7
:10347000743A204F75744F664D656D6F72793A20BE
:1034800000202D3E2041543A004368616E2074793B
:1034900070653A004E6F2073746F726564207661B8
:1034A0006C756573202D2064656661756C743A20B7
:1034B00000536176656420455441473A0053657472
:1034C00020455441473A20002104E30011241FBE47
:1034D000CFEFD1E2DEBFCDBF00E00CBF19E0A0E02E
:1034E000B2E0E4E3FFE902E00BBF02C007900D92F7
:1034F000A63CB107D9F720E1A6ECB9E001C01D92C6
:10350000AE3FB207E1F71AE1C5E6DAE100E006C036
:1035100021970109802FFE010F945E47C436D10721
:1035200080E00807A9F70F94CE310D94884F0C94D2
:10353000000090E080E00895DC01ED91FC910284B0
:10354000F385E02D1994DF92EF92FF920F931F9372
:10355000CF93DF93EC010C891D890115110559F0FA
:103560001D8A1C8AC801DF91CF911F910F91FF9096
:10357000EF90DF900895EC85FD858E859F85DF01B6
:10358000A80FB91F2C91243209F055C011962C9127
:103590002B3709F050C00296E80FF91FF12CE12CEF
:1035A000DF01D190DD2009F446C08DE7D816E9F09F
:1035B0008FEFE81AF80AF4CF198A188A2C853D850E
:1035C0002115310579F08E859F85280F391FF90166
:1035D0002081222321F001969F878E873EC01D8681
:1035E0001C86C0CF0FEF1FEFBDCFE114F10419F11E
:1035F0001C928E859F8502966C857D85680F791F4C
:10360000E881F9810684F785E02DCE011995998B23
:10361000888B1B8A1A8AEC85FD858E859F85E80F2D
:10362000F91FEE0DFF1DD2828E859F850396E80E51
:10363000F91EFF86EE86288939892115310509F49E
:10364000BDCF8A899B89280F391FF9012081222348
:1036500009F4B2CF01969B8B8A8B022F220F110B9C
:1036600081CFDC011C96ED91FC911D971E968D91EA
:103670009C91E80FF91F8081082E000C990B08958A
:10368000FC01A581B681109769F094818091310287
:10369000891740F0ED91FC9111970190F081E02D98
:1036A000CD01199581E090E00895DC0115968D918A
:1036B0009C91009739F0DC01ED91FC910680F78137
:1036C000E02D19940895FC01838594859C0144E0C4
:1036D000359527954A95E1F756E0959587955A9542
:1036E000E1F72817390719F081E090E0089582E0AA
:1036F00090E0089583E090E00895DC011296ED914A
:10370000FC9113973097B9F016968D919C91843067
:10371000910541F08530910541F0039749F482E02D
:1037200090E0089581E090E0089581E190E00895AF
:10373000828590E0089590E080E0089585E090E033
:1037400008951F93CF93DF930097A1F0FC0110859C
:10375000212F2F70223071F4EC01618572858385F1
:1037600094850F94A44569877A878B879C87107FFF
:1037700013601887DF91CF911F9108958EE090E03C
:103780000895CF93DF93FC01C681D78180858F7028
:10379000853079F08630E1F42097D1F0E881F98125
:1037A000309719F080818F7B79F40A80DB81C02DFE
:1037B000F3CF209769F0CE010E94C11B811105C093
:1037C0000A80DB81C02DF5CF81E0DF91CF91089594
:1037D00080E0FBCF84E190E00895DC01ED91FC9165
:1037E0000484F585E02D60E0199581E090E008956E
:1037F000DC011496ED91FC9180E0309711F085A1E9
:10380000817090E00895CF93DF93EC016EEF7AE042
:1038100082ED9FE00E94AFF0EA81FB810280F3819C
:10382000E02D6081718182ED9FE00E9499F082ED30
:103830009FE00E9443EFE881F9810484F585E02D43
:1038400060E0CE01199581E090E0DF91CF9108957D
:103850000D942D3D0D942D3D0D942D3D0D942D3D3C
:103860000D942D3DEF92FF920F931F93CF93DF9313
:103870008C0160EB7FE082ED9FE00E94AFF082ED73
:103880009FE00E9443EFD8011496ED91FC91309790
:1038900049F1C681D781209729F1E881F9813097D4
:1038A000E9F080818823D1F06BE175E0CE010F94BF
:1038B000F7127C01009791F0FC0181859285A38528
:1038C000B4850097A105B10549F00F942D3DD701AE
:1038D00019961D921D921D921C921C970A80DB81E5
:1038E000C02DD9CFD801ED91FC910484F585E02D50
:1038F00060E0C801199581E090E0DF91CF911F91C0
:103900000F91FF90EF9008950D942D3D0D942D3D56
:103910000D942D3D0D942D3D0D942D3DEF92FF9274
:103920000F931F93CF93DF93EC018B018091CD090F
:103930009091CE090097A9F0FC0120852F702630C8
:1039400081F40F94F712FC0190859F70943049F434
:1039500081859285DF91CF911F910F91FF90EF901C
:103960000895EE88FF88C70101970D97D0F46FE1A5
:1039700075E0C8010F94CB4B892B99F48FE2888FA7
:1039800085E08E9DB0018F9D700D1124685C7C4E8A
:1039900046E050E0CE0149960F940440CE0148968F
:1039A000D9CF90E080E0D6CF2F923F924F925F9296
:1039B0006F927F928F929F92AF92BF92CF92DF923F
:1039C000EF92FF920F931F93CF93DF93CDB7DEB7A4
:1039D000AA970FB6F894DEBF0FBECDBF5C010E8F65
:1039E0001F8F28A339A34AA35BA36CA37DA31C8AC2
:1039F0001B8ADC0118968D919C9101979E8B8D8B73
:103A0000E114F104D1F0CE0145969F938F93029774
:103A10009F938F9383E295E09F938F93FF92EF9212
:103A20000F94804C0FB6F894DEBF0FBECDBF019748
:103A300021F48B899C899E8B8D8B6B897C894AE0D4
:103A400050E082ED9FE00E9450F066E373E182ED6A
:103A50009FE00E94AFF06D897E894AE050E082EDE0
:103A60009FE00E9450F060E373E182ED9FE00E94CE
:103A7000AFF0FE8DFAA74AE050E06F2F82ED9FE095
:103A80000E9466EF82ED9FE00E9443EF19861A863E
:103A90001B861C861D861E861F86188A8A85807F47
:103AA00084608A87D50118968D919C912D893E89D5
:103AB000281739071CF001979E8B8D8B8B899C8969
:103AC00097FF02C01C8A1B8A8B889C885401312C6A
:103AD000212C8D899E898A159B050CF46AC1BAA593
:103AE000B13091F1B23009F453C1EE24EA94FE2CC6
:103AF0000E8D1F8D28A139A14AA15BA16CA17DA1CA
:103B0000CE0109960E945DA529833A834B835C838D
:103B10006D837E838F8398878091D3099091D40998
:103B2000FC0122813381A216B30608F088C06F859C
:103B30002E8530E050E040E0542F432F322F2227D3
:103B4000462B6D85262B33C1E090D309F090D40924
:103B5000F70182819381A816B90608F070C0968596
:103B60005385018512854084A92FB0E06484712CAF
:103B7000658570E09401220D331D951372C0A90173
:103B8000440F551F240F351F200F311FA20FB31FE5
:103B90009C91F301E20FF31F1081260F371FD9010B
:103BA0000C91442009F452C0512C712C612C692FC6
:103BB00070E0762F6627072E000C880B990BA30167
:103BC00092010F94E746C901772766276EA37FA36A
:103BD00088A799A7612F70E0762F6627072E000C23
:103BE000880B990BA30192010F94E746542F432FA2
:103BF000322F22278EA19FA1A8A5B9A5822B932B96
:103C0000A42BB52B8EA39FA3A8A7B9A7602F70E004
:103C1000762F6627072E000C880B990BA3019201C3
:103C20000F94E7466EA17FA188A599A5262B372B77
:103C3000482B592B232B242B252B09F4A0C0FFEF55
:103C4000AF1ABF0A2FEF221A320A43CF212F30E0DA
:103C500050E040E0542F432F322F2227492B202BB6
:103C6000E9CFC901880F991F880F991F800F911FF5
:103C7000A80FB91F3C91DC01A50FB11D0C91F301F8
:103C8000E80FF91FD080860F971FDC011C9144209C
:103C900009F463C0512C712C612C632F70E0762FD6
:103CA0006627072E000C880B990BA30192010F9435
:103CB000E746922F8827772766276EA37FA388A7DA
:103CC00099A7602F70E0762F6627072E000C880BCF
:103CD000990BA30192010F94E746A90133272227EC
:103CE0008EA19FA1A8A5B9A5822B932BA42BB52BA0
:103CF0008EA39FA3A8A7B9A7612F70E0762F662790
:103D0000072E000C880B990BA30192010F94E74634
:103D10006EA17FA188A599A5622B732B842B952B6F
:103D20006EA37FA388A799A76D2D70E0762F6627D5
:103D3000072E000C880B990BA30192010F94E74604
:103D4000542F432F322F22278EA19FA1A8A5B9A5BA
:103D5000282B392B4A2B5B2B6DCF802F90E0B0E0C6
:103D6000A0E0DC0199278827B32BAC01412B8A0105
:103D70009D011D29012B022B032B09F060CF2FEF92
:103D80003FEF4FEF50E0B501C7010E94A2F557CFBA
:103D90008091D3099091D409DC0112962D913C9128
:103DA000A216B30608F04BCF20E030E0A901B50120
:103DB000ECCFCC2009F488C00091D3091091D4092C
:103DC000D80119968D919C91892B09F473C00F9499
:103DD000B424F801C784D088E188F2886C157D0589
:103DE0008E059F0520F46787708B818B928BF8017D
:103DF000C784D088E188F2886C197D098E099F09F3
:103E00006C3271408105910510F3F894D801149635
:103E10008D919C9115979A8B898B1996ED91FC91B8
:103E20007F01BFEFEB1AFB0A80818D8FF801908133
:103E30000388F489E02DD80155968C91992309F4D3
:103E40005EC09081982B9C8F9081809589238B8F69
:103E50008B8D888F88E08F8B5C8D6B8D4D8D3F892E
:103E6000288D89899A89D701508347FD252F3A9556
:103E70002083262F39F0441F00C00000608300001B
:103E800000C0F2CF38E04D9160830000019761F7E8
:103E9000D8015496FC93EE9353974D8F3F8B288F08
:103EA0009A8B898B78940F94B424F8016787708B70
:103EB000818B928B6BE273E182ED9FE00E94AFF009
:103EC00082ED9FE00E9443EF81E090E0AA960FB65A
:103ED000F894DEBF0FBECDBFDF91CF911F910F9140
:103EE000FF90EF90DF90CF90BF90AF909F908F901A
:103EF0007F906F905F904F903F902F9008959081AA
:103F0000982B9C8F9081809589238B8F8B8D8A8FA6
:103F100088E0898F5C8D6B8D4D8D398D2A8D8989D7
:103F20009A89D701508347FD252F00C000C0208308
:103F300000C000C000C000C000C060830000262F89
:103F40003A9541F0441F000000C000C000C000C00E
:103F500000C0E8CF38E04D9100C0608300C00197F9
:103F600009F7D8015496FC93EE9353974D8F398FF0
:103F70002A8F96CFCF93DF93EC016BE972E182ED4C
:103F80009FE00E94AFF06FE872E182ED9FE00E9437
:103F9000AFF06C817D814AE050E082ED9FE00E94AD
:103FA00050F069E872E182ED9FE00E94AFF082ED8F
:103FB0009FE00E9443EF60E08C810F948423E881AE
:103FC000F9810484F585E02D60E0CE01199581E04A
:103FD00090E0DF91CF9108950F931F93CF93DF93DC
:103FE0008C0169E275E082ED9FE00E9447EFC0918D
:103FF000D309D091D4094C815D8170E060E089855E
:104000009A850F94F844209771F089859A850F94CA
:104010002D3D8E819F8197FD03C060E00F94842326
:10402000CE010F942D3DD801ED91FC910484F585CE
:10403000E02D60E0C801199581E090E0DF91CF911B
:104040001F910F910895CF93DF93EC0169E375E021
:1040500082ED9FE00E9447EF40E050E0BA018A8184
:104060009B810E940CB0E881F9810484F585E02DE4
:1040700060E0CE0119956D858C810F9456236D8576
:104080008D810F94562381E090E0DF91CF910895C8
:10409000CF92EF92FF920F931F93CF93DF9300D0B5
:1040A00000D01F921F92CDB7DEB77C0109831A831F
:1040B0002B833C834D835E836F83788765EE7AE044
:1040C00082ED9FE00E94AFF0CE0101960E94A87B96
:1040D000898181112DC00B81013091F130F010E008
:1040E000023009F040C0CC2001F160E0CE01019621
:1040F0000E947377F70102811381892B81F0C80137
:104100000E944DB0672B682B692B79F44FEF5FEF5E
:10411000BA0180E00F94C30FAB01BC0103C040E0C3
:1041200050E0BA01C8010E940CB081E090E02EC0BE
:104130008031D0F58E30D8F58130C9F18230D9F197
:1041400068ED7AE082ED9FE00E94AFF04AE050E037
:10415000698182ED9FE00E9466EF82ED9FE00E9400
:1041600043EF01E010E068EC7AE082ED9FE00E940E
:10417000AFF04AE050E0B80182ED9FE00E9450F0BD
:1041800082ED9FE00E9443EF90E080E028960FB61A
:10419000F894DEBF0FBECDBFDF91CF911F910F917D
:1041A000FF90EF90CF9008958351843048F6F70147
:1041B00002811381A4CF40E050E0BA01F70182816F
:1041C0009381B1CFFC01828193810E944CB821E0A0
:1041D00030E0823011F430E020E0C90108950F93FF
:1041E0001F93CF93DF938C01D0E0C0E00115110540
:1041F000B1F0BE016E5D744FC8010F94CD3F892BA5
:1042000051F4FE01EA5DF44F849190E0DF91CF918B
:104210001F910F9108952596C233D10539F781E09A
:1042200090E0F4CFCF92DF92EF92FF920F931F9323
:10423000CF93DF93EC01EC81FD81309709F4A4C0AA
:104240008A819B81892B09F49FC08081882309F48E
:104250009BC07A016B01E881F9810284F385E02D2E
:10426000CE0119950397D9F4EC81FD8180A591A524
:10427000A2A5B3A5892B8A2B8B2B89F00F94C92774
:10428000EC81FD8100A511A522A533A5601B710B52
:10429000820B930B663971058105910528F38F8197
:1042A000988521E0E21AF108DC01ED91FC91028091
:1042B000F381E02DA701B60119958F819885DC0166
:1042C000ED91FC910190F081E02DD601129660E015
:1042D0009D012C193D092E153F0518F42D91620FF3
:1042E000F7CF19950C811D814FEF5FEFBA0180E088
:1042F0000F94C30FF80160A771A782A793A76AE183
:1043000079E082ED9FE00E94AFF04AE050E06E81DC
:1043100082ED9FE00E9466EF65E179E082ED9FE02B
:104320000E94AFF08601C8018C199D098E159F056A
:10433000B8F4D8016C9140E150E06A3050F468E480
:1043400075E082ED9FE00E9499F040E150E0F801B5
:10435000608182ED9FE00E9466EF0F5F1F4FE3CF09
:1043600082ED9FE00E9443EFE881F9810484F585A6
:10437000E02D63E0CE01DF91CF911F910F91FF906F
:10438000EF90DF90CF901994DF91CF911F910F9113
:10439000FF90EF90DF90CF900895FF920F931F93BF
:1043A000CF93DF93CDB7DEB764970FB6F894DEBF37
:1043B0000FBECDBF8C01F62EDC0116966C91FF204E
:1043C00011F081E06827F80184810F945623F801E9
:1043D00087819085A185B285883E9340A105B1056E
:1043E00008F463C06BED72E182ED9FE00E94AFF0D4
:1043F00066ED72E182ED9FE00E94AFF0D801149665
:104400006D917C914AE050E082ED9FE00E9450F077
:1044100061ED72E182ED9FE00E94AFF06F2D70E0E0
:104420004AE050E082ED9FE00E9450F082ED9FE074
:104430000E9443EF8FE290E09C878B87FE013D96C0
:1044400088E0DF011D928A95E9F76AEC72E1CE01FE
:104450000B960F94C23FF801828193810E944CB861
:10446000FF2079F162EC72E1853151F06BEB72E182
:10447000863131F06FEA72E18F3011F467EB72E14F
:10448000CE0101960F94D63FD8011296ED91FC9182
:104490000280F381E02DAE01455F5F4FBE016F5F8B
:1044A0007F4F808191810F94842864960FB6F89491
:1044B000DEBF0FBECDBFDF91CF911F910F91FF9057
:1044C00008956BEA72E18230D9F266EA72E1D8CFE0
:1044D000AF92BF92CF92EF92FF920F931F93CF9321
:1044E000DF9300D000D01F921F92CDB7DEB75C01E2
:1044F00009831A832B833C834D835E836F83788784
:1045000060E273E182ED9FE00E94AFF0CE01019680
:104510000E94A87BE114F10439F069E173E1C7015D
:104520000F94CD3F009759F1F501028113810115D8
:10453000110519F18981811165C08B81813009F4E0
:1045400069C078F1823059F1082F10E066EF72E10E
:1045500082ED9FE00E94AFF066EE72E182ED9FE097
:104560000E94AFF04AE050E0B80182ED9FE00E9467
:1045700050F082ED9FE00E9443EF90E080E02896AB
:104580000FB6F894DEBF0FBECDBFDF91CF911F9164
:104590000F91FF90EF90CF90BF90AF900895CC20F7
:1045A000D9F060E0CE0101960E947377892B09F45F
:1045B00050C0C8010E944DB0672B682B692BF9F4DD
:1045C0004FEF5FEFBA0180E00F94C30FAB01BC0166
:1045D000C8010E940CB013C0C8010E944CB88E30B4
:1045E00019F050F4813059F460E0CE0101960E9438
:1045F0007377892B21F0DDCF83518430A8F381E0DC
:1046000090E0BDCF803100F58E3098F6813089F290
:104610008230F9F06EE073E182ED9FE00E94AFF02E
:1046200061E073E182ED9FE00E94AFF04AE050E06C
:10463000698182ED9FE00E9466EF82ED9FE00E941B
:1046400043EF01E010E082CF8351843008F4B1CF12
:10465000E1CF40E050E0BA01C8010E940CB060E038
:10466000C5010E94CD21CBCF4F925F926F927F9276
:104670008F929F92AF92BF92CF92DF92FF920F9351
:104680001F93CF93DF9300D000D01F921F92CDB71E
:10469000DEB76130710509F482C0FC01628173816B
:1046A0006115710509F47BC08C0119821A821B8285
:1046B0001C821D821E821F8218868A81807F8A83C7
:1046C00040E050E2CE0101960E94B07660E0CE015B
:1046D00001960E9473776C01F801828193810E9498
:1046E0004DB02B013C01F801278130854185528571
:1046F000D6010F9433472FEF30E040E050E00F94A5
:10470000E74649015A010F94C927FF24F394811405
:104710009104A104B10461F064197509860997092F
:10472000FF24F394681579058A059B0508F4F12C9C
:10473000411451046104710491F1F801878090845F
:10474000A184B2840F94C927F80181149104A104B3
:10475000B10451F06419750986099709681579053E
:104760008A059B0508F449C0A280B3804FEF5FEF34
:10477000BA0180E00F94C30FAB01BC01C5010E94D8
:104780000CB0CD2861F0F80184810F94AC0FF801D2
:104790009681891304C061E0C8010E94CD2190E098
:1047A00080E028960FB6F894DEBF0FBECDBFDF9134
:1047B000CF911F910F91FF90DF90CF90BF90AF905E
:1047C0009F908F907F906F905F904F900895FF2003
:1047D000D9F060E0C8010E94CD21F8018281938167
:1047E0000E9471BA892BD9F640E050E0BA01F80175
:1047F000828193810E940CB0D2CF84810F94AC0F40
:10480000F80196818913E3CFCD2849F2F80184811C
:104810000F94AC0FF80196818913C1CFF110BFCF6F
:10482000BACFAF92BF92CF92DF92EF92FF920F93E7
:104830001F93CF93DF93CDB7DEB768970FB6F89489
:10484000DEBF0FBECDBFFC01098B1A8B2B8B3C8BBF
:104850004D8B5E8B6F8B788F82819381009709F4EB
:10486000A1C024813581232B09F49CC0CC2009F4FC
:1048700099C06F0170E060E00E94D9B0192FD60195
:10488000ED91FC91008CF18DE02DC60119955C0134
:104890008230910509F47AC0039709F445C095E088
:1048A000F1E0AF16B10409F091E019861A861B8673
:1048B0001C861D861E861F86188A8A85807F892B06
:1048C0008A87EE24EA94FE2C09891A892B893C896F
:1048D0004D895E896F89788DCE0109960E945DA50C
:1048E000F1E0AF16B10409F453C082E0A816B10498
:1048F00009F049C06F8570E0D60114968C910F9431
:10490000C02361E070E0C6010E9426E66E8570E07B
:104910000F94C02362E070E0C6010E9426E66D8518
:1049200070E00F94C0232FC0612F661F6627661F9B
:10493000CE0141960E9473775C01BC01D6011496AA
:104940008C910F94C0236EE672E182ED9FE00E948D
:10495000AFF0F601648175814AE050E082ED9FE09E
:104960000E9450F06CE672E182ED9FE00E94AFF091
:104970004AE050E0B50182ED9FE00E9450F082EDE8
:104980009FE00E9443EF81E090E00EC094E08DCF65
:1049900063E070E0C6010E9426E6688970E00F942B
:1049A000C023A8CF90E080E068960FB6F894DEBFF1
:1049B0000FBECDBFDF91CF911F910F91FF90EF9070
:1049C000DF90CF90BF90AF900895CF93DF93EC012D
:1049D00062E672E182ED9FE00E94AFF06C817D8122
:1049E0004AE050E082ED9FE00E9450F060E672E104
:1049F00082ED9FE00E94AFF0EA81FB810280F381AB
:104A0000E02D6081718182ED9FE00E9499F06AE55E
:104A100072E182ED9FE00E94AFF082ED9FE00E9484
:104A200043EFE881F981008CF18DE02DCE011995DD
:104A30008130910529F0029759F060E08C811AC00D
:104A400063E070E0CE010E9426E660E00F948423CC
:104A500060E08C810F94842361E070E0CE010E94BD
:104A600026E660E00F94842362E070E0CE010E94AD
:104A700026E660E00F948423E881F9810484F585BB
:104A8000E02D60E0CE01199581E090E0DF91CF91BB
:104A90000895CF92DF92FF920F931F93CF93DF93EE
:104AA00000D000D01F921F92CDB7DEB76C01F02E60
:104AB0001A83022F10E0FF2029F00115110511F4CF
:104AC00001E010E040E050E061E070E0F60182813A
:104AD00093810E94E1B101301105A9F10230110565
:104AE00041F0012BB1F56CE67FE082ED9FE00E9482
:104AF000AFF08A818F70B9F1F60102811381C8018C
:104B00000E944DB0672B682B692B89F401E010E0FF
:104B1000C80128960FB6F894DEBF0FBECDBFDF9157
:104B2000CF911F910F91FF90DF90CF9008954FEF9D
:104B30005FEFBA0180E00F94C30FAB01BC01C80165
:104B40000E940CB0E3CFF1E0FF1681F082E0F8168E
:104B500069F060E67FE082ED9FE00E94AFF082EDB9
:104B60009FE00E9443EF10E000E0D2CFF601C28048
:104B7000D380C6010E944DB0672B682B692B31F2A0
:104B80004FEF5FEFBA0180E00F94C30FAB01BC01A0
:104B9000C6010E940CB0BCCFCF92DF92EF92FF9281
:104BA0000F931F93CF93DC011296ED91FC9160E07F
:104BB000848195810F94A9138C01009729F0FC0141
:104BC00080858F708530D1F066EB71E18DE29FE0DA
:104BD0000E94AFF08DE29FE00E9443EFC12CD12CE8
:104BE00090E8E92E9FEBF92EC701B601CF911F91F6
:104BF0000F91FF90EF90DF90CF900895C8010F9430
:104C00003A14813040F18630A8F1893020F565E012
:104C1000C8010F94A913FC0190859F709330F9F49B
:104C2000C184D284E384F484C1E060E0C8010F94BD
:104C3000A913FC0190859F70933009F561857285F9
:104C40008385948520E030E0A9010F949D4587FF7E
:104C50001FC0C111C9CFC12CD12C7601C5CF923054
:104C600049F461857285838594850F94A4456B0111
:104C70007C01DACFC0E0C12CD12C7601D6CF9230A6
:104C800039F461857285838594850F94A445DACFC4
:104C9000C111AACFC12CD12C8FE7E82E83E4F82EC6
:104CA000A3CFCF93DF93EC0164E871E182ED9FE045
:104CB0000E94AFF0EA81FB810280F381E02D6081E8
:104CC000718182ED9FE00E9447EFEC81FD8130977A
:104CD00021F0808191810F942D3D8C819D810F94D5
:104CE0002D3D70E060E08A819B810E94C9AF1D82EA
:104CF0001C8281E090E0DF91CF910895CF93DF9304
:104D0000EC016AE475E082ED9FE00E9499F0EA818F
:104D1000FB810280F381E02D6081718182ED9FE053
:104D20000E9447EF8C819D81009711F00F942D3DDB
:104D300070E060E08A819B810E94C9AF1D821C8265
:104D400081E090E0DF91CF910895CF93DF93FC0154
:104D500022813381232B59F1EC0164E779E082ED64
:104D60009FE00E94AFF04AE050E06E8182ED9FE04C
:104D70000E9466EF82ED9FE00E9443EF8C819D814F
:104D80000F942D3D70E060E08A819B810E94C9AF45
:104D90001D821C82E881F9810484F585E02D60E0A4
:104DA000CE01199581E090E0DF91CF91089590E0D8
:104DB00080E0FACFCF92DF92EF92FF92CF93DF9312
:104DC00069017A010F94AB0EEC01892BC9F088853B
:104DD000982F9F70923039F0933071F0911110C07C
:104DE000807F82608887C701B6010F946F4869870A
:104DF0007A878B879C8704C0C986DA86EB86FC8617
:104E0000CE01DF91CF91FF90EF90DF90CF9008958A
:104E1000CF92DF92EF92FF920F931F93CF93DF9386
:104E2000009701F1DC011896EC91EF70E630D1F4B7
:104E300069017A018B01EC010F94F7120097A1F43C
:104E4000A7019601B801CE010F94EC20B801CE0164
:104E5000DF91CF911F910F91FF90EF90DF90CF9056
:104E60000D94F71290E080E0DF91CF911F910F91A8
:104E7000FF90EF90DF90CF900895CF92DF92EF9266
:104E8000FF920F931F93CF93DF93009701F1DC0103
:104E90001896EC91EF70E630D1F469017A018B013C
:104EA000EC010F94F7120097A1F4A7019601B80145
:104EB000CE010F94C820B801CE01DF91CF911F9190
:104EC0000F91FF90EF90DF90CF900D94F71290E04C
:104ED00080E0DF91CF911F910F91FF90EF90DF90D5
:104EE000CF9008952F923F924F925F926F927F9250
:104EF0008F929F92AF92BF92EF92FF920F931F9368
:104F0000CF93DF93CDB7DEB72C970FB6F894DEBF03
:104F10000FBECDBF6130710509F463C18C01FC0186
:104F2000E280F38040E050E061E070E0C7010E9461
:104F30000AB2672B682B692B09F453C140E050E09B
:104F400062E070E0C7010E940AB2672B682B692BF0
:104F500089F480912702882309F443C140E050E09E
:104F600062E070E0C7010E94E1B1809127028150A8
:104F700080932702F801E280F380C7010E944DB0C0
:104F80004B015C0119821A821B821C821D821E82C7
:104F90001F8218868A81807F8A8340E050E2B701B1
:104FA000CE0101960E94B07660E0CE0101960E948B
:104FB00073777C01F801828193810E944CB8823022
:104FC00011F0853011F4F12CE12CF80186819AEC76
:104FD000980F903108F0B7C121853285A90170E0A2
:104FE00060E049875A876B877C8743845484712C9F
:104FF000612C0F9497249C01990F440B550B241995
:10500000350946095709AFEFB0E00F9428472985C5
:105010003A854B855C8524193509460957090F9453
:105020000947390137FDB9C15FEF6516710411F009
:105030000CF0B6C181149104A104B10409F08BC134
:10504000E618F70856EFE5165FEFF5060CF0F6C028
:10505000F801658585810F945623F801A280B380FD
:10506000C5010E944DB0672B682B692B59F44FEF97
:105070005FEFBA0180E00F94C30FAB01BC01C50123
:105080000E940CB0F801B48065858EEF8B0D8C30DA
:1050900028F084ED8B0D833008F070C0AA27BB2761
:1050A000AE19BF09662309F45CC09D01A1E0BFEF02
:1050B0000F946D4729E130E040E050E00F9409473C
:1050C000BA01A90141505F4F6F4F7F4F942F852F39
:1050D000692F782F6F3F710519F014F06FEF70E0B2
:1050E0006634710514F466E470E08B2D78C061E5D8
:1050F0007FE082ED9FE00E94AFF082ED9FE00E9492
:1051000043EF69E575E082ED9FE00E9447EFF8010B
:10511000658584810F945623F801658585810F94F8
:10512000562340E050E0BA01F801828193810E9449
:105130000CB040E050E061E070E0F80182819381C2
:105140000E94B8B140E050E062E070E0F801828176
:1051500093810E94B8B1809127028F5F80932702CC
:1051600040C02FEF30E00F94754729E130E040E078
:1051700050E00F940947922F832FAACF858191E0A9
:1051800069279EEF980F9C3020F08C52833008F0F6
:10519000D6C08B2D0F945623AA27BB27AE19BF0963
:1051A000F80185858823B1F12FEF30E00F94754722
:1051B00029E130E040E050E00F940947922F832F1F
:1051C000692F782F6F3F710519F014F06FEF70E0C1
:1051D0006634710514F466E470E0F80185810F947B
:1051E000C02390E080E02C960FB6F894DEBF0FBE8F
:1051F000CDBFDF91CF911F910F91FF90EF90BF90A6
:10520000AF909F908F907F906F905F904F903F9066
:105210002F9008959D01A1E0BFEF0F946D4729E104
:1052200030E040E050E00F940947BA01A901415035
:105230005F4F6F4F7F4F942F852FC2CFFBE0EF164C
:10524000F1040CF45ECFF801658584810F94562338
:10525000F801A280B380C5010E944DB0672B682B76
:10526000692B59F44FEF5FEFBA0180E00F94C30F41
:10527000AB01BC01C5010E940CB0F801B580658589
:105280008EEF8B0D8C3020F084ED8B0D8330B0F4DD
:10529000662351F09701A1E0BFEF0F946D4723E320
:1052A00030E040E050E00ACF2FEF30E0D7010F941C
:1052B000754723E330E040E050E05BCF848191E02C
:1052C00069279EEF980F9C3018F08C528330B8F508
:1052D0008B2D0F945623F80185858823E1F02FEF5D
:1052E00030E0D7010F94754729E130E040E050E00D
:1052F0000F940947922F832F692F782F77FF02C0D1
:1053000070E060E06F3F710519F014F06FEF70E02E
:10531000F801848164CF9701A1E0BFEF0F946D473E
:1053200029E130E040E050E00F940947BA01A901BB
:1053300041505F4F6F4F7F4F942F852FDDCF8B2DC7
:105340000F9456234ECF66246A94762C81149104D0
:10535000A104B104F1F0F80127803084032C000C83
:10536000440855080F94C9272114310441045104FD
:1053700009F4BDCE681979098A099B09621573057C
:105380008405950508F0B3CEFFEF6F167F0609F090
:1053900057CE4FE7E41AF10855CE712C612C4ACE56
:1053A00066246A94712C46CE8F929F92AF92BF92E0
:1053B000CF92DF92EF92FF920F931F93CF93DF93E1
:1053C000CDB7DEB760970FB6F894DEBF0FBECDBF86
:1053D000E986FA860B871C872D873E874F87588B77
:1053E0006115710511F0011103C090E080E0CCC09F
:1053F0007B015C01DB018D909C9019821A821B82DB
:105400001C821D821E821F8218868A81807F8A8369
:1054100067E675E0C7010F94F7126C016CE675E062
:10542000C7010F94F7127C01C114D10451F1F601A8
:1054300080858F70843029F5818592850E94EF20C8
:10544000182F8930B1F134F48130E4F4C12CD12C1F
:10545000760168C08A30D1F7B701CE0109960E9463
:10546000347F29833A834B835C836D837E838F8370
:1054700098873F7009F4B9CFCE0101960E941C793C
:1054800015C011E0B701CE0109960E94347F29832F
:105490003A834B835C836D837E838F8398873F70D1
:1054A00009F4A3CFCE0101960E94D8786B017C014C
:1054B00039C0B701CE0109960E94347F29833A830F
:1054C0004B835C836D837E838F8398873F7009F461
:1054D0008CCF31503B3008F0B9CFE32FF0E0882774
:1054E000EB58F54D8F4F0D945E47892A892A262A5D
:1054F000802A802AE42AD72AD72AD72A802A802AF3
:105500002D813E814F815885AAE0B0E00F94284755
:10551000CDCFCD80FAE0CF9E600111240D2C000C80
:10552000EE08FF0880913102893020F4809130022A
:105530008930E8F06FE17FE082ED9FE00E94AFF0FC
:10554000B40182ED9FE00E9499F068E17FE082ED76
:105550009FE00E94AFF02AE030E0B701A60182EDA3
:105560009FE00E9408F082ED9FE00E9443EFD5018A
:105570001296ED91FC9162E0848195810F94A913BC
:10558000009779F581E090E060960FB6F894DEBF61
:105590000FBECDBFDF91CF911F910F91FF90EF9084
:1055A000DF90CF90BF90AF909F908F90089520E0B4
:1055B00030E040E251E46D817E818F8198850F94C7
:1055C00003460F946F4872CF6D817E818F819885DD
:1055D0002AE030E040E050E00F94094769017A0189
:1055E000A1CFFC0120852F70263061F6B4010F9405
:1055F000F7125C01009731F2DC0118968C91189734
:105600008F709BEF980F923008F0BCCF450185302A
:1056100029F416968C90169717969C90F501808524
:105620008068808760E775E0C4010F94F712FC0181
:10563000892B61F0C186D286E386F486812F82951C
:10564000807F10851F70182B10879CCF6FE07FE044
:1056500082ED9FE00E94AFF0D5016D917C9182EDCB
:105660009FE00E9499F082ED9FE00E9443EFA70126
:10567000960160E775E0C4010F94C82060E775E00B
:10568000C4010F94F712FC01892B09F47BCF12950A
:10569000107F90859F70192BD7CF2F923F924F92FA
:1056A0005F927F928F929F92AF92BF92CF92DF9242
:1056B000EF92FF920F931F93CF93DF9300D000D010
:1056C0001F921F92CDB7DEB709831A832B833C83C9
:1056D0004D835E836F837887DC011496ED91FC9196
:1056E0000FEF1FEF3097F9F057014C01C288D388B4
:1056F000E114F10489F1F7018081882369F1C11473
:10570000D10489F1B701C6010F94F712E980FA803C
:105710000B811C812D813E814F815885BC01C401C4
:105720000E94D4298C01C80128960FB6F894DEBFD8
:105730000FBECDBFDF91CF911F910F91FF90EF90E2
:10574000DF90CF90BF90AF909F908F907F905F90B1
:105750004F903F902F900895C114D10421F0D601AD
:105760001696CD90DC907B80F12C0FEF1FEF272C4D
:10577000312C512C412CC114D10449F16CE175E05C
:10578000C6010F94F7120097E9F0FC0120852F70F5
:105790002230C1F481859285A385B4858215930555
:1057A000A405B50579F4E980FA800B811C812D816F
:1057B0003E814F815885B601C4010E94D4298C01D5
:1057C000FF24F394D6011296CD90DC90D4CFF11043
:1057D000AACF6AE37FE08DE29FE00E94AFF0B501BF
:1057E0008DE29FE00E9499F06EE27FE08DE29FE003
:1057F0000E94AFF0672D70E04AE050E08DE29FE03C
:105800000E9450F08DE29FE00E9443EF8CCF1F93E7
:10581000CF93DF9300D000D0CDB7DEB761307105F4
:1058200009F46BC05CF4672B09F45DC06DEB7CE0A0
:1058300082ED9FE00E94AFF080E04BC062307105C6
:1058400071F06330710591F79093D70D8093D60D69
:1058500055275093D90D4093D80D84E009C09093FB
:10586000D70D8093D60D5093D90D4093D80D83E07A
:105870000F945829182F4FEF5FEFBA0180E00F9473
:10588000C30F6093CF097093D0098093D10990938F
:10589000D2091123D9F068EA7CE08DE29FE00E94F2
:1058A000AFF0812F90E0B0E0A0E089839A83AB83D2
:1058B000BC8380E190E09E838D83BE016F5F7F4F4C
:1058C0008DE29FE00E94FECF0E9443EF81E0111124
:1058D000B3CF26960FB6F894DEBF0FBECDBFDF91D3
:1058E000CF911F9108959093D70D8093D60D50932B
:1058F000D90D4093D80D81E0BBCF9093D70D809305
:10590000D60D5093D90D4093D80D82E0B1CFCF93EF
:10591000DF93EC01EC81FD8140815181052E000C6B
:10592000660B770B22818DE39CE00E94FCF170E016
:1059300060E08A819B810E94D9B0E2EDFDE0828324
:105940008DE39CE0918380831092E20E1092E40E2E
:105950001092E30EDF91CF910895CF93DF936115FD
:10596000710589F0EB01DC011296ED91FC9162E08A
:10597000848195810F94A913BE010F94F712DF91D2
:10598000CF910D94932290E080E0DF91CF91089524
:105990004F925F926F927F928F929F92AF92BF923F
:1059A000CF92DF92EF92FF920F931F93CF93DF93EB
:1059B000CDB7DEB768970FB6F894DEBF0FBECDBF88
:1059C000098B1A8B2B8B3C8B4D8B5E8B6F8B788F5F
:1059D000DC0112962D913C911397232B09F4DEC024
:1059E000CC2009F4DBC06C01ED91FC91008CF18DB1
:1059F000E02D19955C0167E17BE082ED9FE00E945C
:105A0000AFF0CE0141960E94A87BA114B10471F4BD
:105A100060E0CE0141960E947377682FF601848181
:105A200095810F94AF0981E090E0BAC0CE01419614
:105A30000E9467794C0194E0F2E0AF16B10459F08E
:105A400081E1A816B10409F445C091E0A1E0AA16CD
:105A5000B10409F495E019861A861B861C861D86FA
:105A60001E861F86188A8A85807F892B8A87EE2466
:105A7000EA94FE2C09891A892B893C894D895E8913
:105A80006F89788DCE0109960E945DA56DE07BE05F
:105A900082ED9FE00E94AFF0CE0109960E94A87BA4
:105AA000B2E0AB16B10489F0E1E1AE16B104B1F099
:105AB000AA94AB2809F0B7CF188963E070E0C6015B
:105AC0000E9426E6612F0F94AF096F85F60184814D
:105AD000958151C0888D8170888FBCCF0FE710E011
:105AE0008FEF88169806A9F0092C000CAA08BB08AD
:105AF000A50194012959310941095109AFEFB0E0DD
:105B00000F9428472BE531E040E050E00F9409471F
:105B1000890163E070E0C6010E9426E65C012889E5
:105B200030E0D8010F947547412C512C32014A9432
:105B3000A30192010F940947622FC5010F94AF0989
:105B400064E070E0C6010E9426E65C01AFEFB0E0C1
:105B5000A01BB10B288930E00F947547A301920177
:105B60000F940947622FC5010F94AF096F85D601C5
:105B700014968D919C910F94AF091E8561E070E0A1
:105B8000C6010E9426E6612F0F94AF091D8562E0D1
:105B900070E0C6010E9426E6612F43CF90E080E0CE
:105BA00068960FB6F894DEBF0FBECDBFDF91CF91E0
:105BB0001F910F91FF90EF90DF90CF90BF90AF902B
:105BC0009F908F907F906F905F904F9008958F92ED
:105BD0009F92AF92BF92CF92DF92EF92FF920F937C
:105BE0001F93CF93DF9300D000D01F921F92CDB7A9
:105BF000DEB76D7F6130710509F4BDC0FC01E28044
:105C0000F380E114F10409F4B6C08C01C7010E94CD
:105C10004DB04B015C0161E070E0C7010E9493B0A0
:105C200081149104A104B10409F4A5C020E030E07E
:105C30004AE754E40F9403460F9476486B017C01C5
:105C4000C114D104E104F10409F495C00F94C927EB
:105C5000681979098A099B096C157D058E059F05D0
:105C600008F489C0F801A280B38070E060E0C5014B
:105C70000E9493B020E030E048EC52E40F940346D9
:105C80000F9476486B017C014FEF5FEFBA0180E023
:105C90000F94C30FAB01BC01C5010E940CB0198267
:105CA0001A821B821C821D821E821F8218868A8194
:105CB000807F8A83F8016281738140E050E3CE01E6
:105CC00001960E94B076CE0101960E941C794B018C
:105CD0005C0163E775E082ED9FE00E9499F02AE0A5
:105CE00030E0B501A40182ED9FE00E945EEF62E822
:105CF00075E082ED9FE00E9499F02AE030E0B70164
:105D0000A60182ED9FE00E945EEF82ED9FE00E947F
:105D100043EFC80CD91CEA1CFB1C8A81807F86607B
:105D20008A83CD82DE82EF82F886F80162817381F8
:105D300040E050E2CE0101960E949D7566E875E054
:105D400082ED9FE00E9499F02AE030E0B701A601C1
:105D500082ED9FE00E945EEF82ED9FE00E9443EFA4
:105D600030E020E040E050E260E070E0F801828145
:105D700093810E9491B590E080E028960FB6F89448
:105D8000DEBF0FBECDBFDF91CF911F910F91FF906E
:105D9000EF90DF90CF90BF90AF909F908F9008953D
:105DA000CF92DF92EF92FF920F931F93CF93DF93E7
:105DB000CDB7DEB762970FB6F894DEBF0FBECDBF8A
:105DC0006C010B871C872D873E874F87588B698B0B
:105DD0007A8B63EC7AE0C7010F94CD3FEEE0F0E000
:105DE000892BF1F06DEB7AE0C7010F94CD3FE0E134
:105DF000F0E0892BA9F067EB7AE0C7010F94CD3F63
:105E0000EFE0F0E0892B61F01D8563EB7AE0C701DC
:105E10000F94CD3FE12FF0E0892B11F4EDE0F0E09D
:105E20009B85992341F0309731F4EF2809F45CC049
:105E30008FEF9FEFCAC0E131F10508F037C0882726
:105E4000EB5DF04D8F4F0D945E47182F742F362F5A
:105E5000562F562F562F562F2630DD30562F562FC1
:105E6000562F562F562FE7302031F530CE010B96A6
:105E70000E94D87820EF260F2931D0F6D60114964B
:105E8000ED91FC91159723A39B01AC013327442787
:105E900055271296ED91FC910280F381E02D6081EF
:105EA00071810BE915E0C6010E9490E6D6011496B7
:105EB000ED91FC911597118A1496ED91FC9115972F
:105EC00081E081871496ED91FC9115978DE482878E
:105ED0001496ED91FC9115978FE5838714966D913B
:105EE0007C9145E250E04CC0F601048115814FEFF2
:105EF0005FEFBA0180E00F94C30FD80198966D93BD
:105F00007D938D939C939B97D601ED91FC91048496
:105F1000F585E02D64E0C6011995EB85E150E63189
:105F200028F6F0E0D60114962D913C91159788271C
:105F3000E356F04D8F4F0D945E47B32FC42F562F6D
:105F4000562FC42FB32F562F562F562F562F562F5E
:105F5000562F562FF42F0C30562F562F562F562FC4
:105F6000083004300A30F90185A1858F1496ED912F
:105F7000FC91858D8160858F4DE050E06AE172E093
:105F8000C6010E9412211FC0F90185A1858F1496B8
:105F9000ED91FC91858D8E7F858F4DE050E06DE019
:105FA00072E0C6010E941221D6011296ED91FC9179
:105FB0000280F381E02D40EA55E06BE776E08081D6
:105FC00091810F94842881E090E062960FB6F89456
:105FD000DEBF0FBECDBFDF91CF911F910F91FF901C
:105FE000EF90DF90CF900895F901178AD6011496AB
:105FF000ED91FC91159785A1858F1496ED91FC91FB
:10600000858D8160858F52CF81E0F901878BEECF3E
:1060100082E0FBCF84E0F9CF83E0F901878B14960F
:10602000ED91FC91159785A1858F1496ED91FC91CA
:106030001597858D8160858F1496ED91FC91818DEA
:10604000833009F033CF82E0818F30CF1982F6019F
:10605000048115819031C1F190F4923009F440C06F
:106060009E30B9F0CE010B960E94D878611571056B
:106070008105910509F058C0F80117A243C091317C
:1060800041F1923179F782E0F801818F6DE67AE093
:1060900006C083E0D80159968C9365E47AE0CE017E
:1060A00001960F94D63FD6011296ED91FC91028095
:1060B000F381E02D45EA55E0BE016F5F7F4F80819F
:1060C00091810F948428F2CEF801118E69E57AE06F
:1060D000E6CF81E0D80159968C9363E67AE0DFCF72
:1060E000D80197961C92048115814FEF5FEFBA019A
:1060F00080E00F94C30FD80198966D937D938D9394
:106100009C939B97D6011496ED91FC91159785A1D0
:10611000858F1496ED91FC91858D8E7F858F4DE056
:1061200050E06DE072E02CCFD80197961C92615040
:10613000710981099109660F771F881F991F2EEF3A
:1061400030E040E050E00F940947DA01C9010196C0
:10615000A11DB11D813071F0A8F2823029F1833088
:1061600009F0A1CFD6011496ED91FC91118E69E54D
:106170007AE008C0D6011496ED91FC9182E0818FFF
:106180006DE67AE0CE0101960F94D63FD6011496C3
:10619000ED91FC91159785A1858F1496ED91FC9159
:1061A000858D8160858F7FCFD6011496ED91FC910E
:1061B00081E0818F63E67AE0E5CFCE010B960E9405
:1061C000D878D6011496ED91FC91678B6FCED601ED
:1061D0001496ED91FC91913029F0923009F066CE41
:1061E000148E64CE80E5848F61CEF6010481158122
:1061F000913049F09230B1F0CE010B960E94D878E0
:10620000F801638F53CE83E0D8015B968C930280B4
:10621000F381E02D0280F381E02D4AEA55E06AE641
:1062200076E04DCFF801138ED6011296ED91FC91D8
:106230000280F381E02D4AEA55E06BE776E03FCF3C
:10624000D6011496ED91FC91913031F0923009F025
:106250002DCE858D877FD6CE858D8860D3CE8F92CB
:106260009F92AF92BF92CF92DF92EF92FF920F93E5
:106270001F93CF93DF937C014A015901C091CD094F
:10628000D091CE09062F660F110B209709F45CC040
:1062900088858F70863009F055C061EB75E0CE01BE
:1062A0000F94F7126C0182E08816910449F066EBB6
:1062B00075E0E3E08E16910429F0D0E0C0E006C05E
:1062C0006AEB75E0CE010F94F712EC01C114D10412
:1062D000D9F1F60180858F708430B1F561857285C2
:1062E000A801C7010F94F94BA8016DE578E0C7013B
:1062F0000F94DB4B209779F188858F70843059F5A6
:1063000069857A85A801C7010F94DB4BA8016DE56B
:1063100078E0C7010F94DB4BA114B10429F0A80168
:10632000B501C7010F94DB4BC701DF91CF911F91DE
:106330000F91FF90EF90DF90CF90BF90AF909F9024
:106340008F900895D0E0C0E0A8016BE873E1C70129
:106350000F940440C9CFF2E08F16910481F083E0DE
:106360008816910429F06091CB097091CC09CACFAD
:10637000A80165E873E1C7010F94E63FC7CFA80104
:1063800062E873E1F8CFAF92BF92CF92DF92EF92C3
:10639000FF921F93CF93DF9300D000D0CDB7DEB72D
:1063A0006C017C0110E08AE0A82EB12C133061F161
:1063B000F701828190E0B0E0A0E089839A83AB830B
:1063C000BC83BE82AD82BE016F5F7F4F85E29FE0DE
:1063D0000E94FECF60E873E10E94AFF01F5FFFEF05
:1063E000EF1AFF0A143011F726960FB6F894DEBFA5
:1063F0000FBECDBFDF91CF911F91FF90EF90DF9047
:10640000CF90BF90AF900895F601858190E0B0E005
:10641000A0E089839A83AB83BC83BE82AD82BE0138
:106420006F5F7F4F85E29FE00E94FECF6EE773E1D2
:10643000D3CFFC01DC018D918111FDCF30E020E054
:1064400050E040E08AE09191992301F144305105F8
:106450005CF59E3271F42F3F310509F02CF5DB011C
:10646000A40FB51F12962C934F5F5F4F30E020E0D2
:10647000EACF829FD001839FB00D1124292F990F5D
:10648000330B205331092A0F3B1FDDCF2F3F31053E
:1064900009F054F4443051053CF4640F751FFB01BE
:1064A000228381E090E0089590E080E00895CF920B
:1064B000DF92EF92FF920F931F93CF93DF93EC0144
:1064C0006A017B01CB01BA010F946F488B011F93C6
:1064D0006F9381ED97E09F938F93DF93CF930F940A
:1064E000504C0F900F900F900F900F900F9020E056
:1064F00030E0A901C701B6010F94A548181624F091
:10650000F7FAF094F7F8F09409900020E9F7219752
:106510008EE28883B80117FF03C0719561957109F8
:10652000072E000C880B990B0F94A4459B01AC011E
:10653000C701B6010F94904720E030E040E251E4FB
:106540000F9403460F946F48605D69831A82DF9150
:10655000CF911F910F91FF90EF90DF90CF90089512
:10656000CF93DF931F921F92CDB7DEB78091F210C9
:106570009091F310009711F48EEF90E1BE016F5FE0
:106580007F4F681B790B072E000C880B990B0F901F
:106590000F90DF91CF9108954F925F926F927F920B
:1065A0009F92AF92BF92CF92DF92EF92FF920F93A2
:1065B0001F93CF93DF93CDB7DEB768970FB6F894EC
:1065C000DEBF0FBECDBFFC01198A1A8A1B8A1C8A46
:1065D0001D8A1E8A1F8A188E8A89807F8A8BA081D5
:1065E000B181109709F47AC08C91882309F476C0A0
:1065F00000811181D8019C91992309F443C09D32F7
:1066000009F4DAC090539A3028F00F5F1F4F1183BE
:106610000083EECFC801912CDC016D01C81AD90AA4
:106620002D91022E000C330B205331092A303105F5
:10663000A0F37F016EE270E0C8010F94C04BFC0133
:10664000009709F448C0DC015D01AE1ABF0A11963B
:106650008C911197082E000C990BC09711960A97F0
:1066600098F38181282F082E000C330B2053310919
:106670002A30310518F480330CF057C020E030E0A8
:10668000A90108C0912CD12CC12CD3CF29E030E036
:1066900040E050E0AAE0B0E00F9428472B013C0115
:1066A0002281822F022E000C990BC0978A3091050F
:1066B00070F420330CF441C02A330CF042C0092E90
:1066C000000CAA0BBB0B480E591E6A1E7B1EA114A0
:1066D000B10409F088C0CD2809F073C088E0FE013C
:1066E0007196DE01199601900D928A95E1F7298540
:1066F0003A854B855C856D857E858F859889689602
:106700000FB6F894DEBF0FBECDBFDF91CF911F91C2
:106710000F91FF90EF90DF90CF90BF90AF909F9040
:106720007F906F905F904F9008958A330CF0AECFBA
:10673000032E000C440B550BADCF80E090E0DC0144
:10674000C2CF89E090E0A0E0B0E0BDCFB8E0CB16CA
:10675000D1040CF04DC0C8010F947F3F9B01AC01E8
:10676000A4E6B0E00F942847992041F0709460941B
:1067700050944094411C511C611C711C2A89207F3B
:1067800026602A8B460E571E681E791E4D8A5E8A29
:106790006F8A788E6CE270E0F701808191810F94AE
:1067A000C04B009721F4D7011D921C9297CF019600
:1067B000F7019183808392CFC80101969924939425
:1067C0002BCFC8010F947F3FAB01BC01CE01419696
:1067D0000E94877629833A834B835C836D837E8313
:1067E0008F839887D7CFF3E0AF16B1040CF4AECF08
:1067F000C8010F945D3F2A89207F27602A8B6D8B0B
:106800007E8B8F8B988FC6CFCF92DF92EF92FF92C5
:106810000F931F93CF93DF93EC01A881B981109759
:1068200081F18C91882369F108811981F8019081A7
:10683000992351F09D3241F090539A3028F00F5F28
:106840001F4F19830883F0CFC8010F947F3F6B015E
:106850007C016CE270E0C8010F94C04B009769F4B2
:1068600019821882C701B601DF91CF911F910F9154
:10687000FF90EF90DF90CF900895019699838883E1
:10688000F1CFC12CD12C7601EDCF0097B1F1FC01F5
:10689000DB01AC01405F5F4F80E090812FE9290F61
:1068A000263098F497559295907F9C9321813FE9EB
:1068B000320F3630B0F42755922B9D933296E41761
:1068C000F50759F791E0892708952FEB290F263016
:1068D00010F49753E8CF90539A3028F381E090E07A
:1068E000E2CF3FEB320F363010F42753E5CF205381
:1068F0002A3010F381E020E0DFCF80E00895009798
:10690000D1F0DC011696ED91FC913097A1F08085D5
:106910008F70843021F481859285009771F4068010
:10692000F781E02D309739F080858F70843019F42D
:1069300081859285089590E080E0089508950F93F1
:106940001F93CF93DF93EC010A811B8170E060E01D
:10695000C8010E94D9B01816D4F48A8761E070E0AB
:10696000C8010E94D9B0181619069CF49987888727
:1069700062E070E0C8010E94D9B01816190664F4EC
:106980009C878B87DF91CF911F910F91089583E0B2
:10699000E4CF8BE290E0EACF88E590E0F1CF089574
:1069A0000895089508950F931F93CF93DF93EC01FB
:1069B0001D860A811B8170E060E0C8010E94D9B089
:1069C00087FD44C08C838C818150853410F080E237
:1069D0008C8361E070E0C8010E94D9B087FD3BC0A4
:1069E0008D838D818150853410F081E28D8362E04A
:1069F00070E0C8010E94D9B0863490F58E8363E0C0
:106A000070E0C8010E94D9B09C01215031092115C4
:106A1000344040F59A87898764E070E0C8010E949D
:106A2000D9B0813024E0920700F59C878B8765E020
:106A300070E0C8010E94D9B018161906CCF49887E6
:106A40008F83DF91CF911F910F91089581958C8352
:106A500081E08D87B8CF81958D8381E08D87C1CF0F
:106A60001E82CDCF1A861986D7CF80E094E0DDCF85
:106A700080E197E2E4CF08950895CF93DF93EC018E
:106A80006EE772E182ED9FE00E94AFF069E772E18C
:106A900082ED9FE00E94AFF06C817D814AE050E082
:106AA00082ED9FE00E9450F063E772E182ED9FE08B
:106AB0000E94AFF082ED9FE00E9443EF61E08C8185
:106AC0000F9484236E818C810F9456238A819B813D
:106AD000009729F040E050E0BA010E940CB0E88134
:106AE000F9810484F585E02D62E0CE0119958A8153
:106AF0009B81009799F00E9471BA1816190674F4D8
:106B00000A80DB81C02D4FEF5FEFBA0180E00F9468
:106B1000C30FAB01BC01CE010E940CB081E090E03C
:106B2000DF91CF910895CF93DF93EC0160E572E19F
:106B300082ED9FE00E94AFF06C817D814AE050E0E1
:106B400082ED9FE00E9450F06EE472E182ED9FE0E2
:106B50000E94AFF0EA81FB810280F381E02D608129
:106B6000718182ED9FE00E9499F068E472E182ED0C
:106B70009FE00E94AFF082ED9FE00E9443EF8A8188
:106B80009B81892B09F451C08C819D81892B09F04F
:106B90004CC0E881F981008CF18DE02DCE01199572
:106BA0008130910529F0029759F061E08C811AC07B
:106BB00063E070E0CE010E9426E661E00F9484233A
:106BC00061E08C810F94842361E070E0CE010E942B
:106BD00026E661E00F94842362E070E0CE010E941B
:106BE00026E661E00F9484238091A100887F809342
:106BF000A10080919100887F809391008091A100F5
:106C000082608093A10080919100826080939100C6
:106C1000E881F9810484F585E02D62E0CE011995C3
:106C200081E090E0DF91CF91089590E080E0FACF8D
:106C30002F923F924F925F926F927F928F929F928C
:106C4000AF92BF92CF92DF92EF92FF920F931F937A
:106C5000CF93DF93CDB7DEB760970FB6F894DEBF62
:106C60000FBECDBF9A838983DC011496ED91FC9110
:106C7000309709F45DC1868097808114910409F4EE
:106C80001DC1D401ED91FC91309709F413C18081AD
:106C9000882309F40FC12FEF3FEFA90166EA75E0E1
:106CA000C4010E943D2722E030E040E050E061EA6C
:106CB00075E0C4010E943D272FEF3FEFA90166EB6D
:106CC00075E0C4010E943D276BE175E0C4010F949B
:106CD000F712988B8F87009709F4ECC0FC01808530
:106CE0008F70853009F0E6C0CF010F943A148330DD
:106CF00008F4E0C020E030E040EA51E46CE975E0DF
:106D0000C4010E9408278C010E94A11B20E030E0F2
:106D100040EA51E46FEB75E0C4010E9408276C0162
:106D20000E94A11B20E030E040E050EC63EC75E0F5
:106D3000C4010E9408277C010E94A11B20E030E0D2
:106D400040E85FE370E060E08F8598890F94D20E91
:106D50002B013C0120E030E0A9010F949D45B12CAE
:106D600087FF06C077FA709477F87094BB24B394C9
:106D700020E030E0A90161E070E08F8598890F94F0
:106D8000D20E6B837C838D839E8320E030E0A9014B
:106D900062E070E08F8598890F94D20E6F837887B8
:106DA00089879A8720E030E040EA50E463E070E0B1
:106DB0008F8598890F94D20E6B877C878D879E87ED
:106DC0008CE390E00F94913C1C019801275F3F4FAA
:106DD000A701475F5F4FB601675F7F4F1F92BF926A
:106DE000FA85FF9389858F9398859F93AF81AF93A1
:106DF000AB80BC80CD80DE8083017201C1010E9426
:106E00009BF4C101032C000CAA0BBB0BEF85F88986
:106E100081879287A387B48761E070E0C1010E94F7
:106E2000FCF320E030E04AE754E46B857C858D85F7
:106E30009E850F9403460F946F48AF85B8891996C5
:106E40008D919C910E944EF463EA7FE082ED9FE079
:106E50000E94AFF0B301A20182ED9FE00F943D18B4
:106E600066EC75E082ED9FE00E9499F04B815C81B9
:106E70006D817E8182ED9FE00F943D186AEC75E094
:106E800082ED9FE00E9499F03F81288599858A854F
:106E9000432F522F692F782F82ED9FE00F943D18DA
:106EA00082ED9FE00E9443EF0F900F900F900F90A4
:106EB0000F900F90F40182809380DFCE68E97FE02D
:106EC00082ED9FE00E94AFF082ED9FE00E9443EFD1
:106ED00040E050E0BA01A981BA8112968D919C914F
:106EE0000E940CB0A981BA81ED91FC9111970484A4
:106EF000F585E02D62E0CD01199581E090E0609686
:106F00000FB6F894DEBF0FBECDBFDF91CF911F91BA
:106F10000F91FF90EF90DF90CF90BF90AF909F9038
:106F20008F907F906F905F904F903F902F9008953B
:106F300064E87FE082ED9FE00E94AFF082ED9FE089
:106F40000E9443EF90E080E0DACFCF93DF93EC0133
:106F50000E94D3346EEC75E082ED9FE00E9447EF13
:106F600061E08C810F94842361E08D810F948423F0
:106F70006D858C810F9456236D858D810F945623DA
:106F800060E08E810F94842340E050E0BA018A8152
:106F90009B810E940CB040E050E061E070E08A818B
:106FA0009B810E94B8B140E050E062E070E08A81CD
:106FB0009B810E94B8B1E881F9810484F585E02DB8
:106FC00062E0CE01199582E08093270281E090E093
:106FD000DF91CF9108956F927F928F929F92AF929F
:106FE000BF92CF92DF92EF92FF920F931F93CF93B6
:106FF000DF933C01DC0114968D919C911597892BB0
:1070000071F41296CD91DC9184E190E00F94913C63
:10701000BC01CE010E94C9AFE3019D838C83F301C3
:10702000C481D581209769F464E97CE08DE29FE01A
:107030000E94AFF08DE29FE00E9443EF90E080E07D
:10704000B4C24FEF5FEFBA0180E00F94C30F6E83BD
:107050007F8388879987D3011496ED90FC901597CC
:10706000E114F104D1F01296ED91FC913097A9F062
:10707000C481D581209789F088858F70853069F427
:10708000CE010F943A14823040F00091C70910915C
:10709000C8090115110509F096C067E57CE08DE28D
:1070A0009FE00E94AFF061E070E0E3018C819D8180
:1070B000892B11F470E060E04AE050E08DE29FE03F
:1070C0000E9450F065E57CE08DE29FE00E94AFF009
:1070D00061E070E0F30182819381892B11F470E00B
:1070E00060E04AE050E08DE29FE00E9450F063E5EE
:1070F0007CE08DE29FE00E94AFF0D3011296ED910B
:10710000FC9161E070E084819581892B11F470E03D
:1071100060E04AE050E08DE29FE00E9450F061E5BF
:107120007CE08DE29FE00E94AFF0E301EA81FB8109
:107130000480F581E02D80858F7061E070E08530FE
:1071400011F470E060E04AE050E08DE29FE00E94C0
:1071500050F06FE47CE08DE29FE00E94AFF0D3013D
:107160001296ED91FC91848195810F943A1461E01F
:1071700070E0823010F070E060E04AE050E08DE2B4
:107180009FE00E9450F08DE29FE00E9443EF6CE68A
:107190007CE08DE29FE00E94AFF08DE29FE00E94D4
:1071A00043EFD301ED91FC910484F585E02D61E07E
:1071B000C3011995E301E881F9810084F185E02D8F
:1071C000C30119953BCF61E0CE010F94A913EC01E7
:1071D00088858F70843029F469857A8561157105F9
:1071E00039F467E37CE08DE29FE00E94AFF0CBCF03
:1071F000C8010F94F7128C01009769F465E17CE0F7
:107200008DE29FE00E94AFF069857A858DE29FE074
:107210000E9499F0B8CF6AED75E00F94F7120097CD
:1072200009F4D2C0EC0128852F70243009F0CCC0BD
:10723000C984DA84D0E0C0E0C114D10409F4B7C035
:10724000BE016F58744FC6010F94CD3F892B09F0D2
:10725000A9C0FE01EB58F44F25913491922F832F52
:10726000F7019283838361EE75E0C8010F94F712F2
:10727000E301EC81FD81009709F4AEC0DC011896B2
:107280002C9118972F70223009F0A6C019968D9175
:107290009D910D90BC91A02D0097A105B10509F419
:1072A0009BC09183808340815181052E000C660B29
:1072B000770B22818DE39CE00E94FCF166EE75E085
:1072C000C8010F94F7127C01F301C481D5810097A6
:1072D00009F488C0DC0118968C918F70863009F013
:1072E00081C06BEE75E0C7010F94F7129B878A8708
:1072F00060EF75E0C7010F94F7129D878C8764EFEC
:1073000075E0C7010F94F7129F878E876AEF75E0CB
:10731000C7010F94F712998B888B6FEF75E0C70147
:107320000F94F712009709F45AC0FC0181859285E9
:107330009D838C8365E076E0C8010F94F7129B8BE8
:107340008A8B892B09F40FC16FEF7BE082ED9FE000
:107350000E94AFF082ED9FE00E9443EFD3011496AC
:10736000ED91FC910288F389E02DC681D7812097A9
:1073700009F441C069E076E0CE010F94F71200975E
:1073800069F0FC0120852F70213041F4818588232C
:1073900029F068817981C3010E94AD2C0A80DB81CC
:1073A000C02DE5CF2696C834D10509F045CF64E558
:1073B0007BE082ED9FE00E94AFF082ED9FE00E94B3
:1073C00043EF96E080E04CCF86E090E0D701139643
:1073D0009C938E93129747CF80E895E262CF88EE18
:1073E00093E0A6CF1B861A8688EE93E09D838C835C
:1073F0001D861C869FCF69EE7BE082ED9FE00E9498
:10740000AFF082ED9FE00E9443EFD3011496ED911F
:10741000FC910288F389E02DE680F780E114F10405
:1074200009F47BC06CE675E0C7010F94F712009772
:1074300009F468C062E176E00F94F7128C010097BE
:1074400009F460C0EC0188858F70823009F04EC06D
:10745000C984DA84D3011496ED91FC910288F389F2
:10746000E02D309709F456C0C681D78146010D2C16
:10747000000CAA08BB08209709F44CC066E176E02E
:10748000CE010F94F712009709F440C0FC0120854B
:107490002F702230D9F581859285A385B485881512
:1074A0009905AA05BB0591F568EC7BE082ED9FE0AC
:1074B0000E94AFF06881798182ED9FE00E9499F08F
:1074C00069EB7BE082ED9FE00E94AFF04AE050E084
:1074D000B60182ED9FE00E9450F082ED9FE00E9495
:1074E00043EF68817981C3010E94AD2CF80180854A
:1074F0008F70843039F4D80119966D917C91C30155
:107500000E94AD2CE701EA80FB8088CF0A80DB81F6
:10751000C02DB1CF70E060E0E6CF6FEC7BE082ED94
:107520009FE00E94AFF082ED9FE00E9443EFD30105
:107530001296ED91FC9162E0848195810F94A913DC
:10754000009789F0FC01C681D781209761F0CE01B8
:107550000E94C11B882319F0CE010F9493220A8048
:10756000DB81C02DF2CF6FE77CE085E29FE00E94D7
:10757000AFF0D3011296ED91FC910280F381E02DE2
:107580006081718185E29FE00E9499F085E29FE031
:107590000E9443EFE301E881F9810484F585E02D41
:1075A00062E0C301199581E090E0DF91CF911F91D6
:1075B0000F91FF90EF90DF90CF90BF90AF909F9092
:1075C0008F907F906F900895CF93DF93EC016FEED3
:1075D0007AE082ED9FE00E94AFF0EA81FB810280B9
:1075E000F381E02D6081718182ED9FE00E9499F02E
:1075F00082ED9FE00E9443EFE881F9810484F585E4
:10760000E02D62E0CE01199581E090E0DF91CF910D
:107610000895DC01ED91FC910484F585E02D62E094
:10762000199581E090E008950F931F93CF93DF9316
:10763000DC0112962D913C91232B81F1EC0169E63E
:1076400079E082ED9FE00E94AFF04AE050E06E8169
:1076500082ED9FE00E9466EF82ED9FE00E9443EF83
:107660008C819D81892B61F40A811B818CE290E0E1
:107670000F94913CBC01C8010E94C9AF9D838C83CB
:10768000EC81FD81309769F467E579E08DE29FE058
:107690000E94AFF08DE29FE00E9443EF90E080E017
:1076A0004BC085E2DF011D928A95E9F7EC81FD81EF
:1076B00082E28283EC81FD8116A2EC81FD8115A21C
:1076C000EC81FD8117A20C811D814FEF5FEFBA01A4
:1076D00080E00F94C30FF80160A771A782A793A75A
:1076E0008E81811116C062E00F9484236EE179E0EF
:1076F00085E29FE00E94AFF085E29FE00E9443EFA9
:1077000085E39FE00E9445E81092310281E080937A
:10771000A90A26E040E855E260E070E08F81988594
:107720000E94FCF1E881F9810484F585E02D62E096
:10773000CE01199581E090E0DF91CF911F910F91DB
:1077400008952F923F924F925F926F927F928F9205
:107750009F92AF92BF92CF92DF92EF92FF920F93E0
:107760001F93CF93DF93CDB7DEB7CB57D1090FB6B9
:10777000F894DEBF0FBECDBFE296EFAEE297E39680
:10778000FFAEE397E4960FAFE497E5961FAFE5975A
:10779000E6962FAFE697E7963FAFE797E8964FAFAD
:1077A000E897E9965FAFE9970097B9F124012B2C90
:1077B000EC96AFAEEC97EB96DFAEEB97EA96CFAEDA
:1077C000EA97362E8C0180913102893020F4809125
:1077D00030028930C0F0C8010F94B41B7C01892BA2
:1077E00091F06AE176E082ED9FE00E9499F0B701A6
:1077F00082ED9FE00E9499F082ED9FE00E9443EFAE
:10780000C7010F942D3DF80180858F70843009F4F5
:1078100061C128F4882309F466C180E02FC0853057
:1078200009F446C08630C9F760E276E0C8010F94DB
:10783000F7123C01009709F476C0912C812CB12CF1
:10784000A12CD12CC12CE296EFACE297E396FFACD1
:10785000E397E4960FADE497E5961FADE597E696BE
:107860002FADE697E7963FADE797E8964FADE897DF
:10787000E9965FADE997632D0E94A13BC558DF4FA4
:107880000FB6F894DEBF0FBECDBFDF91CF911F9131
:107890000F91FF90EF90DF90CF90BF90AF909F90AF
:1078A0008F907F906F905F904F903F902F900895B2
:1078B0008091C10A8F5F8093C10A668077806114CE
:1078C000710459F14201EC96AFACEC97B22CEA96F8
:1078D000CFACEA97EB96DFACEB97E296EFACE29792
:1078E000E396FFACE397E4960FADE497E5961FAD02
:1078F000E597E6962FADE697E7963FADE797E896D2
:107900004FADE897E9965FADE997632DC3010E94FB
:10791000A13BF30162807380D2CF8091C10A815074
:107920008093C10A7ACF64E276E0C8010F94F7121F
:107930002C0169E276E0C8010F94F7127C016EE237
:1079400076E0C8010F94F712332039F0F1E03F16CA
:1079500009F4A1C0D12CC12C0CC062E376E0C801AF
:107960000F94F7123C0167E376E0C8010F94F71219
:107970006C016114710409F43801C114D10409F4D3
:1079800068014114510431F4EA964FACEA97EB9642
:107990005FACEB97E114F10421F4EC96EFACEC97BB
:1079A000F22C6114710409F4A7C0F30180858F7073
:1079B000843009F0A1C061847284C114D10409F437
:1079C0009EC0F60180858F70843009F098C0C18414
:1079D000D28410E000E04114510409F4F5C06114B0
:1079E000710409F4B3C068ED73E182ED9FE00E9479
:1079F000AFF0F2016185728582ED9FE00E9499F0FF
:107A000063ED73E182ED9FE00E94AFF0B30182ED80
:107A10009FE00E9499F082ED9FE00E9443EFCE012B
:107A20008F589F4F0E94A87BE114F10409F0D5C044
:107A3000F20180858F70843009F085C14091C50ABC
:107A40005091C60A61857285CE0101960E9498B850
:107A5000CE0101960E94BCAF8823C1F00E94B032D3
:107A60006B01683C71050CF085C062E973E18DE241
:107A70009FE00E94AFF04AE050E0B6018DE29FE047
:107A80000E9450F08DE29FE00E9443EFCE010196EC
:107A90000E9435B958C16CE376E0C8010F94F71223
:107AA0003C0161E476E0C8010F94F7126C016114A7
:107AB000710409F04AC162E376E0C8010F94F7123D
:107AC0003C01C114D10409F44ECF892B09F059CFE0
:107AD000380157CFD12CC12C712C612CF12CE12C09
:107AE000512C412C46CFD12CC12C712C612CF12C66
:107AF000E12C512C412C45CF712C612C5ECF00E044
:107B000020E030E340E150E0BE016F597F4FCE01ED
:107B10008F589F4F0E9488796C01E4960FADE497CF
:107B200010E00115110509F056CFE2968FADE297EE
:107B3000811109C0E3968FADE3978F7009F44BCFA5
:107B400002E010E048CF01E010E045CF69EC73E1BE
:107B500082ED9FE00E94AFF0F2016185728582EDB7
:107B60009FE00E9499F064EC73E182ED9FE00E9437
:107B7000AFF055CF6114710431F0B301CE0101961D
:107B80000F94F31B83CFA12CC12CF12CE12CE29696
:107B90000FADE297E3961FADE397E4962FADE49720
:107BA000E5963FADE597E6964FADE697E7965FAD74
:107BB000E797E8966FADE897E9967FADE997CE0134
:107BC00001960E9483BB62CFE114F10409F4BBC0AB
:107BD000C114D10409F4B7C004C0C114D10409F41C
:107BE00027CFF70180858F70843009F0A8C0818588
:107BF000928525961FAE1EAE259748EE53E060E0B5
:107C000070E029964CAF5DAF6EAF7FAF299720E54E
:107C100032E023963FAF2EAF23972F969FAF8EAFC4
:107C20002F9761961FAE1EAE619763961FAE1EAE74
:107C3000639765961FAE1EAE659767961FAE1EAE24
:107C4000679769961FAF0EAF69976A961FAE6A97DE
:107C500040E450E0BE016F5F7F4FCE018F5B9F4FCE
:107C60000F949F1421E030E02C0F3D1F820F931FD3
:107C7000FC0110826CEB73E182ED9FE00E94AFF09B
:107C8000F7016185728582ED9FE00E9499F066E4BC
:107C900076E082ED9FE00E9499F0BE016F5F7F4F1A
:107CA00082ED9FE00E9499F067EB73E182ED9FE027
:107CB0000E94AFF0B60182ED9FE00E9499F082ED44
:107CC0009FE00E9443EF0F9415138823C1F1809128
:107CD000390C811134C06FE270E0CE0101960F942F
:107CE000C04B892B51F4F7012185328543E050E0E8
:107CF00060E4CE0101960E942F3160EB73E182EDCA
:107D00009FE00E94AFF0BE016F5F7F4F82ED9FE06A
:107D10000E9499F06BEA73E182ED9FE00E94AFF060
:107D2000B60182ED9FE00E9499F082ED9FE00E94F3
:107D300043EF41E0B601CE0101960F94662841144D
:107D4000510409F075CE81E099CD892B09F019CE47
:107D50000ACE8F929F92AF92BF92CF92DF92EF9214
:107D6000FF920F931F93CF93DF9300D000D01F9209
:107D70001F92CDB7DEB7DC011296ED91FC913097E2
:107D800009F468C024813581232B09F463C08C0178
:107D9000662309F472C00E94CC25E62EB72E6C0132
:107DA000D8011296ED91FC910280F381E02D608163
:107DB00071818DE29FE00E9499F06CED71E18DE29E
:107DC0009FE00E94AFF08DE29FE00E9443EF20E031
:107DD00030E0A9016E2D7B2DC6010F94A54887FDCB
:107DE00039C060ED71E18DE29FE00E94AFF04E2D51
:107DF0005B2DB6018DE29FE00F943D188DE29FE070
:107E00000E9443EFD8011296ED91FC9161E08481CC
:107E100095810F94A91319821A821B821C822A81D0
:107E2000207F2760F22E2E2D4E2D5B2DB6014D8327
:107E30005E836F837887912C812CB12CA12CD12C5F
:107E4000C12CE9800B811C813E814F8158856FEFE9
:107E50000E94A13B28960FB6F894DEBF0FBECDBF9F
:107E6000DF91CF911F910F91FF90EF90DF90CF9016
:107E7000BF90AF909F908F9008950280F381E02D86
:107E80006081718185E29FE00E9499F069EE71E165
:107E900085E29FE00E94AFF085E29FE028960FB652
:107EA000F894DEBF0FBECDBFDF91CF911F910F9130
:107EB000FF90EF90DF90CF90BF90AF909F908F900A
:107EC0000C9443EF4F925F926F927F928F929F92AA
:107ED000AF92BF92CF92DF92EF92FF920F931F93D8
:107EE000CF93DF93CDB7DEB7E8970FB6F894DEBF38
:107EF0000FBECDBF09AB1AAB2BAB3CAB4DAB5EABF2
:107F00006FAB78AFDC011496ED91FC91309719F4CA
:107F100090E080E0CBC020813181232BC9F33C016C
:107F2000DC01ED91FC910284F385E02D1995029717
:107F300079F78BA9E82EF12C19A9112321F0E1146E
:107F4000F10409F433C1823009F4D9C0B8F48823AC
:107F500009F4D5C08130B9F06CEF71E182ED9FE09A
:107F60000E94AFF04AE050E0B70182ED9FE00E942E
:107F700050F082ED9FE00E9443EFCACF833009F4B6
:107F800047C0893049F7D3011296ED91FC9161E029
:107F9000848195810F94A9132C0119A61AA61BA6FA
:107FA0001CA61DA61EA61FA618AA8AA5807F8AA7A2
:107FB00019A761E0CE0189960E94437629A33AA3CE
:107FC0004BA35CA36DA37EA38FA398A7115016317A
:107FD00008F0FDC1E12FF0E08827EE50F04C8F4F04
:107FE0000D945E471C41DA40E741E741E741E74134
:107FF000E741E741E7414B41AB41E741E7411C41E4
:108000001C41E741E741E7411C411C411C411C4127
:108010008AA98F7009F47CCFCE01C1960E94927814
:10802000D3011496ED91FC916683778380879187C5
:1080300062E472E182ED9FE00E94AFF0D3011296FC
:10804000ED91FC910280F381E02D6081718182EDE0
:108050009FE00E9499F064E372E182ED9FE00E944C
:10806000AFF0D3011496ED91FC9146815781608564
:10807000718582ED9FE00F943D1882ED9FE00E9494
:1080800043EFF301E480F5800F94C927D70152969E
:108090006D937D938D939C935597D3011496ED9199
:1080A000FC918689811119C081E090E0E8960FB6B5
:1080B000F894DEBF0FBECDBFDF91CF911F910F911E
:1080C000FF90EF90DF90CF90BF90AF909F908F90F8
:1080D0007F906F905F904F900895168A60E0C30183
:1080E0000E94A93ED3011496ED91FC9180E090E0AE
:1080F000A0E0B0EC86879787A08BB18BD5CF8AA9FB
:108100008F7009F405CFCE01C1960E949278D301F9
:108110001496ED91FC9162877387848795876EE250
:1081200072E182ED9FE00E94AFF0D3011296ED91D3
:10813000FC910280F381E02D6081718182ED9FE0EE
:108140000E9499F063E272E182ED9FE00E94AFF03D
:10815000D3011496ED91FC91428553856485758514
:1081600082ED9FE00F943D1882ED9FE00E9443EF67
:10817000D3011296ED91FC9162E0848195810F9478
:10818000A913009709F490CF912C812CB12CA12C2C
:10819000D12CC12CE9A8FAA80BA91CA92DA93EA98C
:1081A0004FA958AD6FEF0E94A13B7ECFEE24E39420
:1081B000F12CE9CE80913A0C90913B0C0597F1F0AF
:1081C00019821A821B821C821D821E821F821886BF
:1081D0008A81807F8A836BE0CE0101960E9465765A
:1081E000912C812CB12CA12CD12CC12C79018A018C
:1081F0009B01AC016FEFC2010E94A13B912C812C2D
:10820000B12CA12CD12CC12CE9A4FAA40BA51CA53E
:108210002DA53EA54FA558A96FEFC2010E94A13B15
:1082200030E020E040E050E460E070E0F301828163
:1082300093810E9491B538CF19821A821B821C82C9
:108240001D821E821F8218868A81807F8A8340E079
:1082500051E060E070E0D30112968D919C910E94F4
:108260000AB2672B682B692BA1F06BE0CE01019657
:108270000E946576912C812CB12CA12CD12CC12C83
:1082800079018A019B01AC016FEFC2010E94A13B01
:10829000BBCF6AE0EBCF80913A0C90913B0C0597F5
:1082A00091F061E0D30112968D919C910E942DB8BE
:1082B00030E020E040E050E160E070E0F3018281D6
:1082C00093810E9491B540E050E061E070E0D301FD
:1082D00012968D919C910E94E1B1912C812CB12C30
:1082E000A12CD12CC12CE9A4FAA40BA51CA52DA569
:1082F0003EA54FA558A96FEFC2010E94A13BD30133
:10830000ED91FC910288F389E02DC3011995892B29
:1083100009F4E8CE19821A821B821C821D821E82F9
:108320001F8218868A81807F8A8361E0CE01019650
:108330000E94657629873A874B875C876D877E87A1
:108340008F87988B79018A019B01AC016FEFC20185
:108350000E94A13BC7CE912C812CB12CA12CD12CF9
:10836000C12CE9A4FAA40BA51CA52DA53EA54FA5DB
:1083700058A96FEFC2010E94A13BD301ED91FC917E
:108380000288F389E02DC3011995892B09F08CCE61
:1083900019861A861B861C861D861E861F86188ACD
:1083A0008A85807F8A8762E0CE0109960E94657681
:1083B00029833A834B835C836D837E838F83988785
:1083C00079018A019B01AC016FEFC201ECCE61E142
:1083D00072E182ED9FE00E94AFF04AE050E069A9AF
:1083E00082ED9FE00E9466EF82ED9FE00E9443EFE6
:1083F000B3CD2F923F924F925F926F927F928F9266
:108400009F92AF92BF92CF92DF92EF92FF920F9323
:108410001F93CF93DF93CDB7DEB764970FB6F89471
:10842000DEBF0FBECDBF1C01DC0114968D919C9167
:108430001597892B99F41296ED91FC91FA83E983B3
:1084400089E190E00F94913CBC0189819A810E945E
:10845000C9AFD10115969C938E931497F1010481B5
:1084600015810115110569F461E771E18DE29FE065
:108470000E94AFF08DE29FE00E9443EF90E080E029
:108480009CC3D8011D921C920280F381E02DFC8BCD
:10849000EB8B309791F0848195819A838983009743
:1084A00061F0DC0118968C9118978F70853029F453
:1084B000CD010F943A14811190C067E371E18DE210
:1084C0009FE00E94AFF061E070E0F101848195814E
:1084D000892B11F470E060E04AE050E08DE29FE00B
:1084E0000E9450F065E371E18DE29FE00E94AFF0E1
:1084F00061E070E0D10112968D919C91892B11F46D
:1085000070E060E04AE050E08DE29FE00E9450F0B1
:1085100063E371E18DE29FE00E94AFF0D10112961A
:10852000ED91FC9161E070E084819581892B11F4DB
:1085300070E060E04AE050E08DE29FE00E9450F081
:1085400061E371E18DE29FE00E94AFF0D1011296EC
:10855000ED91FC910480F581E02D80858F7061E0C4
:1085600070E0853011F470E060E04AE050E08DE2A8
:108570009FE00E9450F06FE271E18DE29FE00E9467
:10858000AFF0D1011296ED91FC91848195810F9409
:108590003A1461E070E0823010F070E060E04AE090
:1085A00050E08DE29FE00E9450F08DE29FE00E943B
:1085B00043EF6BE471E18DE29FE00E94AFF08DE24A
:1085C0009FE00E9443EFD101ED91FC910484F58579
:1085D000E02D61E0C101199551CF60E089819A8158
:1085E0000F94A9139F838E83009729F0FC01808547
:1085F0008F70853039F065E171E18DE29FE00E9476
:10860000AFF0D3CF8E819F810F943A148150883080
:1086100008F0A3C1E82FF0E08827EE5EFC4B8F4FF7
:108620000D945E477E4454442744A2438A438A43C0
:1086300073431A4367E08E819F810F94A913FC0155
:1086400090859F70933009F041C0418452846384C7
:108650007484F1E0FD8366E08E819F810F94A913FD
:10866000FC0190859F70933009F045C0818592850B
:10867000A385B48589839A83AB83BC8391E09D8372
:1086800064E08E819F810F94A913FC0190859F70F7
:10869000933009F050C061857285838594850F946D
:1086A00076484B0163E08E819F810F94A913FC01F2
:1086B00080858F70833009F060C081859285A385A5
:1086C000B4858A879B87AC87BD8764C0923059F494
:1086D00061857285838594850F94A4452B013C01A7
:1086E00081E08D83B8CF412C512C8FE7682E83E435
:1086F000782E1D82B0CF9230C9F461857285838552
:1087000094850F94A44569837A838B839C83A1E02D
:10871000AD83B6CF412C512CBFE76B2EB3E47B2E3B
:1087200019821A821B821C821D82AACF19821A8288
:108730001B821C82A5CF9230C1F481849284A384D1
:10874000B484B0CFF0EC8F2EF7E29F2EF9E0AF2E7D
:10875000B12C412C512CAFE76A2EA3E47A2E19825A
:108760001A821B821C821D829DCFE0EC8E2EE7E2D6
:108770009E2EE9E0AE2EB12C95CF823009F082C05A
:1087800061857285838594850F94A4456A877B876C
:108790008C879D8762E08E819F810F94A913FC01D5
:1087A00080858F70833009F072C091859E87A28585
:1087B000AF87B385B88B8485898B61E08E819F817B
:1087C0000F94A913FC0180858F70833009F08BC052
:1087D000C184D284E384F48460E08E819F810F940D
:1087E000A913FC0180858F70833009F0A9C08185B1
:1087F0009285A385B4858E839F83A887B98720E05F
:1088000030E0A9016E817F81888599850F949D450F
:1088100087FFD0C08E819F81A885B985B0588E838F
:108820009F83A887B98791E09A8BAB89BC891696FC
:10883000ED91FC9180858F70823009F4BDC083304A
:1088400009F4D4C180E090E0A0EAB1E4D3C160ECC7
:10885000862E67E2962E69E0A62EB12C80E090E08D
:10886000A0EAB0E48A879B87AC87BD87412C512C56
:108870007FE7672E73E4772E19821A821B821C828F
:108880001D8288CF80E090E0A0EAB0E41ACF823069
:1088900029F561857285838594850F94A4456E873B
:1088A0007F87888B998B89CF40EC842E47E2942E6A
:1088B00049E0A42EB12C80E090E0A0EAB0E48A87E1
:1088C0009B87AC87BD87412C512C5FE7652E53E415
:1088D000752E19821A821B821C821D821E861F869B
:1088E000188A198A6ACF823039F561857285838545
:1088F00094850F94A4456B017C016ECF20EC822EF1
:1089000027E2922E29E0A22EB12C80E090E0A0EA8E
:10891000B0E48A879B87AC87BD87412C512C3FE709
:10892000632E33E4732E19821A821B821C821D82ED
:108930001E861F86188A198AC12CD12C76014CCF2D
:10894000823091F561857285838594850F94A44565
:108950006E837F838887998752CF80EC882E87E249
:10896000982E89E0A82EB12C80E090E0A0EAB0E437
:108970008A879B87AC87BD87412C512C9FE7692E46
:1089800093E4792E19821A821B821C821D821A8A14
:108990001E861F86188A198AC12CD12C7601CE8298
:1089A000DF82E886F98641CF1A8A1E821F821886E6
:1089B00019863BCF1A8A39CF618572858385948564
:1089C0000F94A445F8016287738784879587D8013F
:1089D00016961D921D921D921C921997F8011282F3
:1089E0001382148215820F94C927D80152966D9371
:1089F0007D938D939C935597D1011496ED91FC91A5
:108A000081E0868B908E878A61E0C1010E94A93E39
:108A1000F10104811581D8018D919C916CEF70E179
:108A2000892B09F0EACD8CE390E00F94913C9C8B6C
:108A30008B8B9801265F3F4FA8014E5F5F4FB801B7
:108A40006A5F7F4F1F92BA89BF93E989EF93F889D4
:108A5000FF938F858F939E859F9356016701EE80CC
:108A6000FF80088519858B899C890E949BF4D10120
:108A70001496ED91FC918B899C89918380830F9052
:108A80000F900F900F900F900F90009709F491CDD9
:108A900061E070E00E94FCF3D1011496ED90FC902F
:108AA000BD81BB2309F44AC0A301920169817A8187
:108AB0008B819C810F94A54887FF40C0F7010190EE
:108AC000F081E02DFF83EE8389819A81AB81BC81A7
:108AD00082AB93ABA4ABB5AB46AA57AA60AE71AE5E
:108AE00082AD882359F1068D178DF8018080918021
:108AF000A280B380A5019401C301B2010F949D45EA
:108B000087FF7EC0D8014D925D926D927C92139743
:108B1000AE81BF8196968D909D90AD90BC909997B7
:108B2000A5019401C301B2010F949D4587FF7DC04B
:108B3000EE81FF8146A257A260A671A620E030E038
:108B40004AE754E46A857B858C859D850F940346AE
:108B50000F946F48D7018D919C910E944EF46DE562
:108B600071E185E29FE00E94AFF0D1011296ED9194
:108B7000FC910280F381E02D6081718185E29FE0AC
:108B80000E9499F085E29FE00E9443EFD101149684
:108B9000ED91FC9180E090E0A0E0B0EC86879787B3
:108BA000A08BB18BD101ED91FC910484F585E02D72
:108BB00062E0C101199581E090E064960FB6F894E7
:108BC000DEBF0FBECDBFDF91CF911F910F91FF9000
:108BD000EF90DF90CF90BF90AF909F908F907F905D
:108BE0006F905F904F903F902F9008958185928570
:108BF000A385B485F80182879387A487B587E7CEDC
:108C0000A501940169817A818B819C810F94A5488B
:108C100018160CF07DCF89819A81AB81BC81F80157
:108C200080839183A283B38373CFA501940169816B
:108C30007A818B819C810F94A54818160CF07ECF09
:108C400089819A81AB81BC81EE81FF8186A397A344
:108C5000A0A7B1A773CF4F925F926F927F928F922E
:108C60009F92AF92BF92CF92DF92EF92FF920F93BB
:108C70001F93CF93DF93CDB7DEB760970FB6F8940D
:108C8000DEBF0FBECDBF6130710509F4DBC1DC0171
:108C90001496ED91FC913097C9F481E090E06096D4
:108CA0000FB6F894DEBF0FBECDBFDF91CF911F91FD
:108CB0000F91FF90EF90DF90CF90BF90AF909F907B
:108CC0008F907F906F905F904F90089520813181B9
:108CD000232B19F33C01DC01ED91FC910284F38517
:108CE000E02D19950297C9F6F301E280F380E114B3
:108CF000F10499F2C7010E944CB8823071F240E051
:108D000051E060E070E0C7010E940AB2672B682B57
:108D1000692B19F6D3011496ED91FC918081918114
:108D2000FC0122AD222309F455C10E945EF2882382
:108D300009F450C1D3011496ED91FC9186898823E2
:108D4000A1F0C3010E94CC256B017C0120E030E042
:108D5000A9010F94A54887FD08C0D3011496ED9191
:108D6000FC91C282D382E482F58260EB71E182EDF4
:108D70009FE00E94AFF0D3011296ED91FC9102802A
:108D8000F381E02D6081718182ED9FE00E9499F076
:108D90006AEA71E182ED9FE00E94AFF0D301149680
:108DA000ED91FC91428553856485758582ED9FE048
:108DB0000F943D1865EA71E182ED9FE00E94AFF0EB
:108DC000D3011496ED91FC914681578160857185A0
:108DD00082ED9FE00F943D1869E476E082ED9FE01C
:108DE0000E9499F0D3011496ED91FC914281538138
:108DF0006481758182ED9FE00F943D1861EA71E115
:108E000082ED9FE00E94AFF0D3011496ED91FC91AA
:108E10000190F081E02D408151816281738182ED6A
:108E20009FE00F943D186DE971E182ED9FE00E9493
:108E3000AFF0D3011496ED91FC910190F081E02DFB
:108E4000448155816681778182ED9FE00F943D18C2
:108E500069E971E182ED9FE00E94AFF0D3011496C1
:108E6000ED91FC910190F081E02D40855185628566
:108E7000738582ED9FE00F943D18D3011496ED9118
:108E8000FC918689882331F062E971E182ED9FE0EF
:108E90000E94AFF082ED9FE00E9443EFF301E48077
:108EA000F580D70156968C918111F7CE02811381FE
:108EB00061E0F801848195810F94A9132C0120E0D1
:108EC00030E0A901D7011E966D917D918D919C9105
:108ED00051970F949D4581110CC020E030E0A9010D
:108EE000F70162817381848195810F94A5481816DA
:108EF0005CF040E050E061E070E0C8010E940AB21E
:108F0000672B682B692B31F119861A861B861C8604
:108F10001D861E861F86188A8A85807F8A8761E063
:108F2000CE0109960E94657629833A834B835C8340
:108F30006D837E838F839887912C812CB12CA12CFB
:108F4000D12CC12C79018A019B01AC016FEFC201C8
:108F50000E94A13B40E050E061E070E0D301129636
:108F60008D919C910E94B8B1D3011496ED91FC9122
:108F7000328163815481458119861A861B861C863D
:108F80008A85807F8760F82E8A87232F832F962FEC
:108F9000A52FB42F8D879E87AF87B88B912C812CFE
:108FA000B12CA12CD12CC12CE9840B851C853E85CC
:108FB0004F8558896FEFC2010E94A13BD3011496DF
:108FC000ED91FC9182819381A481B58186879787F9
:108FD000A08BB18BD3011496ED91FC918689811100
:108FE0005CCE8789908D009709F457CE28EE33E048
:108FF000829F2001839F500C929F500C11240F944C
:10900000C927D3011496ED91FC914114510499F0B4
:109010006201F12CE12C0289138924893589AB0185
:10902000BC01401B510B620B730B4C155D056E05AB
:109030007F0508F432CE81E0868B61E0C3010E9497
:10904000A93E2BCE90E080E02ACE2F923F924F9205
:109050005F926F927F928F929F92AF92BF92CF92C8
:10906000DF92EF92FF920F931F93CF93DF93CDB7D1
:10907000DEB7C458D1090FB6F894DEBF0FBECDBF1E
:10908000FC01902FA2960FAFA297A3961FAFA397B4
:10909000A4962FAFA497A5963FAFA597A6964FAFDE
:1090A000A697A7965FAFA797A8966FAFA897A99620
:1090B0007FAFA99786EF800F823008F4A0C6EB96A9
:1090C000FFAEEEAEEB97AD96FFAFEEAFAD97822F52
:1090D000422E512C002309F4A0C64114510409F476
:1090E00091C6EB96AEADBFADEB97AB2B09F49CC62A
:1090F000873051F5913109F429C2923109F446C201
:109100009031F9F46FEF70E0CE018F599F4F0E94BC
:109110003F776A962FAF6A976B963FAF6B976C96C7
:109120004FAF6C976D965FAF6D976E966FAF6E9702
:109130006F967FAF6F97A0968FAFA097A1969FAFC6
:10914000A19767E0462E512CAD96AEADBFADAD9761
:109150001496ED91FC91309709F474C46680778081
:10916000CF57DF4F19821882C158D040E9961FAE01
:109170001EAEE997E3961FAE1EAEE397312C212C6D
:10918000E7961FAE1EAEE7976114710409F468C438
:1091900066EA75E0C3010F94F712E1969FAF8EAFB8
:1091A000E19761EA75E0C3010F94F712AB969FAFA8
:1091B0008EAFAB9768E576E0C3010F94F712CD57F9
:1091C000DF4F99838883C358D0406BE175E0C301BA
:1091D0000F94F712ED969FAF8EAFED97E196EEAD3F
:1091E000FFADE197309709F4C0C0AB962EAD3FAD0F
:1091F000AB972115310509F4B8C080858F70823096
:1092000009F0B3C0D90118968C918F70823009F0A3
:10921000ACC02CE330E040E050E061E775E0C30112
:109220000F94FE0EC358DF4F688379838A839B8334
:10923000CD57D040EB96EEADFFADEB973097F1F107
:10924000BF01D3018D919C910F94CB4B892BB1F52C
:10925000B2E04B16510409F4ABC30CF09FC1F1E02E
:109260004F16510409F43CC2CD57DF4FE881F98114
:10927000C358D040309711F1912C812CB12CA12CE6
:10928000D12CC12CA296EFACA297A396FFACA397CA
:10929000A4960FADA497A5961FADA597A6962FAD42
:1092A000A697A7963FADA797A8964FADA897A99662
:1092B0005FADA9976FEFCF010E94A13BAB96EEADDA
:1092C000FFADAB9781859285A385B48582309105EA
:1092D000A105B10509F443C08F3F9F4FAF4FBF4F6A
:1092E000F1F1E196EEADFFADE19781859285A38521
:1092F000B485EF964EAD5FADEF97849F9001859F4B
:10930000300D949F300D1124E796EEADFFADE79739
:10931000E20FF31FE796FFAFEEAFE797CF57DF4FB0
:10932000E881F981C158D040AF01FF0F660B770B80
:10933000481759076A077B0794F4CF57DF4F998383
:109340008883C158D040E9963FAF2EAFE997EF969A
:109350002EAD3FADEF97E3963FAF2EAFE397EF967D
:109360004EAD5FADEF97240E351ED30112966D9072
:109370007C900ACFA3968FADA3978F70E1F481E024
:1093800090E0CC57DF4F0FB6F894DEBF0FBECDBFD5
:10939000DF91CF911F910F91FF90EF90DF90CF90D1
:1093A000BF90AF909F908F907F906F905F904F9005
:1093B0003F902F90089566EF70E182ED9FE00E944C
:1093C000AFF068EE70E182ED9FE00E94AFF0CE0159
:1093D0008F599F4F0E949278AB01BC0182ED9FE0B4
:1093E0000F943D1882ED9FE00E9443EFAD96AEAD25
:1093F000BFADAD9712960D911C914FEF5FEFBA0183
:1094000080E00F94C30FAB01BC01C8010E940CB0F7
:10941000CE018F599F4F0E9492786B017C016CE3C3
:1094200079E0AD96EEADFFADAD97848195810F9457
:10943000F712A70196016FEB75E00E94DA269FCF25
:1094400062EE70E182ED9FE00E94AFF068ED70E1A6
:1094500082ED9FE00E94AFF04AE050E0A2966FAD2F
:10946000A29782ED9FE00E9466EF82ED9FE00E944E
:1094700043EFA2960FADA2976CE379E0AD96AEAD47
:10948000BFADAD9714968D919C910F94F71262E544
:1094900077E00F94AB0E7C01009709F470CFFC01CC
:1094A0008085982F9F70923039F0933081F0911120
:1094B00066CF807F8260808710E030E020E0D701B7
:1094C00019960D931D932D933C931C9758CF602FA5
:1094D00070E090E080E00F94A245D70119966D935B
:1094E0007D938D939C931C974ACF62ED70E182ED42
:1094F0009FE00E94AFF060EC70E182ED9FE00E947F
:10950000AFF0CE018F599F4F0E949278AB01BC0102
:1095100082ED9FE00F943D1882ED9FE00E9443EFA3
:10952000CE018F599F4F0E9492786B017C016CE3B2
:1095300079E0AD96EEADFFADAD97848195810F9446
:10954000F712A70196016FE476E077CF60E870E04C
:10955000CE018F599F4F0E943F7762962FAF62973F
:1095600063963FAF639764964FAF649765965FAF1E
:10957000659766966FAF669767967FAF67976896B1
:109580008FAF689769969FAF6997DBCD6AE070E00F
:10959000CE018F599F4F0E943F78D3CD23E04216D2
:1095A000510409F429C237E04316510409F05CCE96
:1095B000A3968FADA3978F7009F48CC0CE018F59FD
:1095C0009F4F0E94D878AB96AEADBFADAB971996C2
:1095D0000D911D912D913C911C97672B682B692B48
:1095E00009F4A6C00230110521053105B1F56CE57D
:1095F00076E082ED9FE00E9499F082ED9FE00E946C
:1096000043EF21E030E040E050E0AB96AEADBFADBF
:10961000AB9719962D933D934D935C931C9761E006
:10962000CE018F599F4F0E9465762A962FAF2A97B9
:109630002B963FAF2B972C964FAF2C972D965FAF65
:109640002D972E966FAF2E972F967FAF2F97609600
:109650008FAF609761969FAF6197CE018F599F4FF3
:109660000E94D878E196EEADFFADE19761877287F1
:109670008387948780913A0C90913B0C059751F128
:10968000D301AD90BC9088248394C12C50E3D52E97
:10969000E12CF12CA2960FADA297A3961FADA39734
:1096A000A4962FADA497A5963FADA597A6964FADCE
:1096B000A697A7965FADA797A8966FADA897A9960E
:1096C0007FADA997AD96EEADFFADAD978281938149
:1096D0000E942EB2A2968FADA297882309F4C4CD22
:1096E000A2969FADA297992309F4BECDEFEFE90FA3
:1096F000E63108F059C1F0E08827EE57F44B8F4F60
:109700000D945E47DC4B764CD44CD44CD44CD44CAA
:10971000D44CD44CD44C944CAE4CD44CD44CC24CC1
:10972000C24CD44CD44CD44CC24CC24CC24CC24C93
:109730000130110521053105B1F56DE676E082EDC8
:109740009FE00E9499F082ED9FE00E9443EF22E0AB
:1097500030E040E050E0AB96AEADBFADAB971996B0
:109760002D933D934D935C931C9762E0CE018F59EE
:109770009F4F0E94657622962FAF229723963FAF88
:10978000239724964FAF249725965FAF259726966B
:109790006FAF269727967FAF279728968FAF28978A
:1097A00029969FAF2997E196EEADFFADE19711861F
:1097B0001286138614865ECFE196AEADBFADE197FB
:1097C00019966D917C91CE018F599F4F0E943F77E2
:1097D00029AF3AAF4BAF5CAF6DAF7EAF8FAF219685
:1097E0009FAF219767E0CE018F599F4F0E9443762C
:1097F00029AB3AAB4BAB5CAB6DAB7EAB8FAB98AFF1
:10980000A2968FADA29790E0B0E0A0E0AB96EEAD4F
:10981000FFADAB9781879287A387B487C12C40E3C4
:10982000D42EE12CF12C80913A0C90913B0C0597B1
:1098300079F1AB96EEADFFADAB9781859285A385AF
:10984000B4850197A105B10519F5E196EEADFFAD1F
:10985000E19781859285A385B4854497A105B105DB
:10986000BCF42EE130E040E050E0218732874387AE
:1098700054876EE170E0CE018F599F4F0E943F7771
:10988000298F3A8F4B8F5C8F6D8F7E8F8F8F98A330
:1098900080913A0C90913B0C059709F4E5CCF301CB
:1098A000A080B18088248394A2960FADA297A3963E
:1098B0001FADA397A4962FADA497A5963FADA597EE
:1098C000A6964FADA697A7965FADA797A8966FAD42
:1098D000A897A9967FADA997AD96AEADBFADAD9750
:1098E00012968D919C910E942EB2BECC70E060E0E9
:1098F000CE018F599F4F0E943F7729A73AA74BA7C8
:109900005CA76DA77EA78FA798AB67E0CE018F59A4
:109910009F4F0E94437629A33AA34BA35CA36DA358
:109920007EA38FA398A76CCFED962EAD3FADED979C
:109930002115310569F0F90181859285A385B485EA
:109940000097A105B10521F061E070E00E94FCF3F1
:10995000C12C20E4D22EE12CF12C65CFED962EAD5A
:109960003FADED972115310599F3F9018185928578
:10997000A385B4850097A105B10551F3DC01DA9602
:109980001C92E6CF892F90E0B0E0A0E0AB96EEAD60
:10999000FFADAB9781879287A387B487C12C30E155
:1099A000D32EE12CF12C3FCFC12CD12C76013BCF13
:1099B000A3968FADA3978F7009F456CCCE018F5923
:1099C0009F4F0E9492789B01AC016CE975E0C30146
:1099D0000E94DA2680913A0C90913B0C059709F48D
:1099E00043CCF301A080B18088248394C12C90E201
:1099F000D92EE12CF12C58CFA3968FADA3978F7061
:109A000009F4BDCC63EB70E182ED9FE00E94AFF002
:109A1000CE018F599F4F0E949278AB01BC0182ED1D
:109A20009FE00F943D1882ED9FE00E9443EFCE012E
:109A30008F599F4F0E9492789B01AC016FEB75E0AC
:109A4000C301FBCCE9961FAE1EAEE997E3961FAEAD
:109A50001EAEE397312C212CE7961FAE1EAEE79782
:109A60002114310409F4CBC1E7968EAD9FADE79781
:109A7000B1010F944A473B0164EA70E182ED9FE037
:109A80000E94AFF04AE050E0B10182ED9FE00E94F9
:109A900050F069E970E182ED9FE00E94AFF00FEFB6
:109AA00010E0E7968EAD9FADE797B8010F944A4757
:109AB0004AE050E082ED9FE00E9450F062E970E1E0
:109AC00082ED9FE00E94AFF04AE050E0B30182EDEA
:109AD0009FE00E9450F068E870E182ED9FE00E94F4
:109AE000AFF0E9968EAD9FADE997B8010F944A4764
:109AF0004AE050E082ED9FE00E9450F061E870E1A2
:109B000082ED9FE00E94AFF04AE050E0E3966EAD38
:109B10007FADE39782ED9FE00E9450F06DE770E12A
:109B200082ED9FE00E94AFF082ED9FE00E9443EF44
:109B300019821A821B821C821D821E821F82188635
:109B40008A81807F8A83B301CE0101960E943F778C
:109B500029873A874B875C876D877E878F87988BAD
:109B600067E0CE0109960E94437679018A011B01C4
:109B70002C01298BFA8A4B8B1C8B6D8B3E8A8F8B29
:109B8000588E6CE379E0AD96EEADFFADAD97848174
:109B900095810F94F712912C812CB12CA12CD12CF2
:109BA000C12C9101A2016FEF0E94A13B672809F42B
:109BB000E6CBAD96AEADBFADAD971496ED91FC91F1
:109BC000309709F4DCCB66807780E3962EAD3FAD0D
:109BD000E397032E000C440B550BE5962CAF3DAFDD
:109BE0004EAF5FAFE597E9968EAD9FADE997092E31
:109BF000000CAA0BBB0BAF968CAF9DAFAEAFBFAF47
:109C0000AF976114710409F4BACB2CE330E040E063
:109C100050E061E775E0C3010F94FE0E6B0166EB47
:109C200075E0C3010F94F712AB969FAF8EAFAB9761
:109C300066EA75E0C3010F94F7128C0161EA75E0E2
:109C4000C3010F94F712AB96AEADBFADAB971097B3
:109C500009F4CDC00115110509F4C9C0009709F434
:109C6000C6C018962C912F70223009F0C0C0F801A0
:109C700020852F70223009F0BAC0DC0118962C9193
:109C800018972F70223009F0B2C0C114D10409F422
:109C9000AEC019968D919D910D90BC91A02D8230F2
:109CA0009105A105B10509F4A6C08F3F9F4FAF4FA5
:109CB000BF4F09F4A0C0E9962EAD3FADE997232B25
:109CC00009F499C0D80119968D919C918C9D8001C1
:109CD0008D9D100D9C9D100D11242FEF30E0D801AB
:109CE0000F9475479601DD0C440B550B0F940947F3
:109CF000E5966CAD7DAD8EAD9FADE5970F94D746E3
:109D0000AF962CAD3DAD4EAD5FADAF970F9409470B
:109D100019012A0166E770E182ED9FE00E94AFF031
:109D2000F3016081718182ED9FE00E9499F060E70C
:109D300070E182ED9FE00E94AFF0C8016FEF70E02C
:109D40000F944A474AE050E082ED9FE00E9450F0B5
:109D50006AE670E182ED9FE00E94AFF02AE030E019
:109D6000B201A10182ED9FE00E9408F082ED9FE028
:109D70000E9443EFAB96EEADFFADAB978185928528
:109D8000A385B48582159305A405B50581F11986CF
:109D90001A861B861C861D861E861F86188A8A8543
:109DA000807F8A87B101CE0109960E943F7729837F
:109DB0003A834B835C836D837E838F839887912C5A
:109DC000812CB12CA12CD12CC12C79018A019B01B1
:109DD000AC016FEFC3010E94A13BAB96AEADBFAD2E
:109DE000AB9719962D923D924D925C921C97F30180
:109DF0006280738006CF212C312C2101BBCF90E0F3
:109E000080E0BFCAEB962EAD3FADEB974424439460
:109E1000512C232B09F098C9B2CAEB964EAD5FAD19
:109E2000EB97452B09F090C9833009F4A3CA20F4BD
:109E3000813008F489C9A3CA883009F401CB8C3079
:109E400009F453CB873009F07FC999CA4F925F92CA
:109E50006F927F928F929F92AF92BF92CF92DF923A
:109E6000EF92FF920F931F93CF93DF93CDB7DEB79F
:109E700068970FB6F894DEBF0FBECDBF3B016CE311
:109E800079E0FC01848195810F94F7122C010097F1
:109E900009F47BC020E030E0A9016FE776E00F9481
:109EA000FE0E8B0120E030E0A90162E577E0C201FF
:109EB0000F94FE0E0115110541F00617170709F062
:109EC00064C00615170509F460C019861A861B863A
:109ED0001C861D861E861F86188A8A85807F8A8733
:109EE000662DCE0109960E946576298B3A8B4B8BA5
:109EF0005C8B6D8B7E8B8F8B988F61E0CE01419652
:109F00000E94437629833A834B835C836D837E83EF
:109F10008F839887912C812CB12CA12CD12CC12C12
:109F200079018A019B01AC016FEFC2010E94A13B44
:109F30006FE776E0C2010F94AB0E8C01009711F130
:109F4000FC018085982F9F70923039F0933079F022
:109F5000911118C0807F82608087C301770CAA0BA3
:109F6000BB0BF80181879287A387B4870BC0B3012D
:109F7000770C880B990B0F94A445F80161877287C1
:109F80008387948781E090E002C090E080E068964B
:109F90000FB6F894DEBF0FBECDBFDF91CF911F91FA
:109FA0000F91FF90EF90DF90CF90BF90AF909F9078
:109FB0008F907F906F905F904F9008952F923F9277
:109FC0004F925F926F927F928F929F92AF92BF92C9
:109FD000CF92DF92EF92FF920F931F93CF93DF9375
:109FE000CDB7DEB7E6970FB6F894DEBF0FBECDBF94
:109FF0004C0161307105D9F5DC0112968D919C916F
:10A000000E944DB0672B682B692B89F14FEF5FEFF2
:10A01000BA0180E00F94C30F6B017C01F40102814F
:10A020001381C8010E944DB0C61AD70AE80AF90A7E
:10A03000F0E6CF16FAEEDF06E104F104C0F040E0EE
:10A0400050E0BA01C8010E940CB06CE379E0D40181
:10A0500014968D919C910F94F7126FEB75E00F940D
:10A06000F712009721F0FC012085207F2087D40182
:10A0700014960D911C910115110509F4C0C36CE3F0
:10A0800079E0C8010F94F7123C01009709F4DAC394
:10A09000FC0180858F70863009F0D4C36FEB75E0CA
:10A0A000C3010F94F712FC01892B09F4CBC39085EF
:10A0B0009F70933009F0C3C3C184D284E384F484D5
:10A0C00020E030E0A90162E577E0C3010F94FE0EC5
:10A0D0007EAB6DAB20E030E040EF51E4C701B6014C
:10A0E0000F94A54818160CF43FC120E030E040E77B
:10A0F00051E4C701B6010F949D4587FF3AC125E1A0
:10A1000030E03CAB2BABF80166807780B12C1AAA0B
:10A1100019AA6114710409F450C3D301ED91FC91A3
:10A12000309709F414C18081882309F410C120E01C
:10A1300030E0A90161EA75E0C3010F94FE0E8B01C6
:10A1400020E030E0A9016CE975E0C3010F94FE0E38
:10A150001B012C0120E030E0A9016FEB75E0C30189
:10A160000F94FE0E6B017C010F30110509F434C110
:10A170000CF004C10230110521F00E30110509F078
:10A1800005C16BE175E0C3010F94F7126C010097F4
:10A1900009F4DDC0FC0181859285A385B485009713
:10A1A000A105B10509F4D3C07C01FC0122AD222335
:10A1B00009F4CDC00E945EF2882309F4C8C063ECA4
:10A1C00075E0C3010F94F7122C01009709F4BFC08A
:10A1D000DC0118968C918F70833009F0B8C063E66B
:10A1E00070E182ED9FE00E94AFF0D4011296ED91F4
:10A1F000FC910280F381E02D6081718182ED9FE00E
:10A200000E9499F06DE578E082ED9FE00E9499F060
:10A21000F3016081718182ED9FE00E9499F06EE50B
:10A2200070E182ED9FE00E94AFF0D7015C96ED9166
:10A23000FC91408151816281738182ED9FE00F9496
:10A240003D1868E570E182ED9FE00E94AFF0D70114
:10A250009096ED91FC91408151816281738182EDF4
:10A260009FE00F943D1862E570E182ED9FE00E944F
:10A27000AFF0D7015E96ED91FC91408151816281F2
:10A28000738182ED9FE00F943D1866E976E082EDE0
:10A290009FE00E9499F0F7014081518162817381B2
:10A2A00082ED9FE00F943D186AE976E082ED9FE031
:10A2B0000E9499F0D70114964D915D916D917C911A
:10A2C000179782ED9FE00F943D186EE976E082EDDE
:10A2D0009FE00E9499F0F701408551856285738562
:10A2E00082ED9FE00F943D18D70158968D919C9177
:10A2F0006EE876E0892B11F068E876E082ED9FE069
:10A300000E9499F0F70182AD64E976E0811102C004
:10A310006AEA78E082ED9FE00E9499F082ED9FE08A
:10A320000E9443EF0431110509F443C105311105C1
:10A3300009F4CEC10E30110551F42BA93CA92431EA
:10A34000310509F44CC02531310509F4C2C0F301CF
:10A3500062807380DECE61857285838594850F94DB
:10A36000A4456B017C01ACCE84E190E09CAB8BAB4F
:10A37000CACEAFE0B0E0BCABABABC5CE033111058C
:10A3800041F024F0063111050CF4FBCE10E000E0A2
:10A39000F8CEC201B1010F94A4451B012C01C701E5
:10A3A000B6010F94A4456B017C01AC019B01C20175
:10A3B000B1010F94A54804E110E0181614F010E064
:10A3C00000E0A7019601C201B1010F949D4587FFEE
:10A3D000D8CE05E110E0D5CEBB24B394D2CE70E048
:10A3E00060E0D60119968D919C910E94C0F361E4C2
:10A3F00070E182ED9FE00E94AFF0D4011296ED91E2
:10A40000FC910280F381E02D6081718182ED9FE0FB
:10A410000E9499F06DE578E082ED9FE00E9499F04E
:10A42000F3016081718182ED9FE00E9499F060E309
:10A4300070E182ED9FE00E94AFF082ED9FE00E940C
:10A4400043EF2DA93EA92230310509F480CFD40174
:10A45000ED91FC9120883188F301E080F180198230
:10A460001A821B821C821D821E821F8218868A818C
:10A47000807F8A83D20119966D917D918D919C91F7
:10A480001C970F946F48CE0101960E943F77298751
:10A490003A874B875C876D877E878F87988B67E0CD
:10A4A000CE0109960E944376022F242F09A73AA7CE
:10A4B0004BA75CA76DA77EA78FA798ABA12CCC2438
:10A4C000C394132F352FAB01BC01C401F1011995C1
:10A4D0003ECF61E070E0D60119968D919C910E946B
:10A4E000C0F36FE170E182ED9FE00E94AFF0D40114
:10A4F0001296ED91FC910280F381E02D60817181D3
:10A5000082ED9FE00E9499F06DE578E082ED9FE09A
:10A510000E9499F0F3016081718182ED9FE00E94B9
:10A5200099F06DE070E182ED9FE00E94AFF082ED66
:10A530009FE00E9443EF2DA93EA92230310509F486
:10A5400006CFD401ED91FC9120883188F301E080A1
:10A55000F18019821A821B821C821D821E821F8238
:10A5600018868A81807F8A83D20119966D917D91A8
:10A570008D919C911C970F946F48CE0101960E947B
:10A580003F7729873A874B875C876D877E878F87E0
:10A59000988B67E0CE0109960E944376022F242F04
:10A5A00009A33AA34BA35CA36DA37EA38FA398A793
:10A5B00085CF70E060E0D60119968D919C910E9444
:10A5C000C0F361E070E182ED9FE00E94AFF0D40142
:10A5D0001296ED91FC910280F381E02D60817181F2
:10A5E00082ED9FE00E9499F06DE578E082ED9FE0BA
:10A5F0000E9499F0F3016081718182ED9FE00E94D9
:10A6000099F060EF7FE082ED9FE00E94AFF082ED75
:10A610009FE00E9443EF2DA93EA92431310509F0A6
:10A6200041C0D401ED91FC9120883188F301E08094
:10A63000F18019821A821B821C821D821E821F8257
:10A6400018868A81807F8A83D20119966D917D91C7
:10A650008D919C911C970F946F48CE0101960E949A
:10A660003F7729873A874B875C876D877E878F87FF
:10A67000988B67E0CE0109960E944376022F242F23
:10A68000098F3A8F4B8F5C8F6D8F7E8F8F8F98A342
:10A69000A12CCC24C394132F352FAB01BC01C401D2
:10A6A000F101199529A93AA9B901330F880B990B22
:10A6B0000F94A445D20119962D913D914D915C9135
:10A6C0001C970F9491470F946F487AAB69AB3FCEBC
:10A6D00061E070E0F601818592850E94C0F364EE2E
:10A6E0007FE082ED9FE00E94AFF0D4011296ED91E1
:10A6F000FC910280F381E02D6081718182ED9FE009
:10A700000E9499F06DE578E082ED9FE00E9499F05B
:10A71000F3016081718182ED9FE00E9499F062ED0A
:10A720007FE082ED9FE00E94AFF082ED9FE00E940B
:10A7300043EF2DA93EA92531310569F519821A8209
:10A740001B821C821D821E821F8218868A81807F46
:10A750008A83D20119966D917D918D919C911C9760
:10A760000F946F48CE0101960E943F7729873A8760
:10A770004B875C876D877E878F87988B67E0CE01DC
:10A7800009960E944376298B3A8B4B8B5C8B6D8BA1
:10A790007E8B8F8B988FE9A9FAA9BF01FF0F880BD9
:10A7A000990B0F94A445D20119962D913D914D918D
:10A7B0005C911C970F94904786CF29A93AA9232B27
:10A7C000C9F16EEB7FE082ED9FE00E94AFF04AE0BE
:10A7D00050E069A97AA982ED9FE00E9450F082EDD5
:10A7E0009FE00E9443EF89A99AA964E170E01816DE
:10A7F000190614F065E170E0C4010E94264F81E063
:10A8000090E0E6960FB6F894DEBF0FBECDBFDF91A5
:10A81000CF911F910F91FF90EF90DF90CF90BF905D
:10A82000AF909F908F907F906F905F904F903F90F0
:10A830002F900895BB2019F36FE070E0DDCF9230C8
:10A8400009F489CDC12CD12C80ECE82E8FE7F82EAD
:10A8500037CC2F923F924F925F926F927F928F925E
:10A860009F92AF92BF92CF92DF92EF92FF920F939F
:10A870001F93CF93DF93CDB7DEB7CF58D1090FB673
:10A88000F894DEBF0FBECDBF3C011A01CD57DF4F9C
:10A890002883C358D040C457DF4F19830883CC584E
:10A8A000D040C257DF4FF982E882CE58D040C95716
:10A8B000DF4FC882C758D040CB57DF4FB982A8823C
:10A8C000C558D040DC011496ED91FC910288F389C3
:10A8D000E02D86809780AB2849F4FE01EE57FF4FAC
:10A8E000CB57DF4FF983E883C558D04081E0CB5781
:10A8F000DF4FA881B981C558D0408C936B01F12CF2
:10A90000E12C8114910409F4F6C5CD57DF4FB881CD
:10A91000C358D040B13009F488C008F47FC0B230C9
:10A9200041F0B33009F477C0D40112968D909C9019
:10A93000E8CF66E176E0C4010F94F71211E00097CA
:10A9400099F3FC0181859285A385B4858C159D05BD
:10A95000AE05BF0549F76CE175E0C4010F94F7122D
:10A96000C857DF4F99838883C858D040D3011296C7
:10A97000ED91FC9162E0848195810F94A913C657F3
:10A98000DF4F99838883CA58D040822D0F9460206E
:10A990007C01CF57DF4F1882C158D04019AA1AAA9C
:10A9A0001BAA1CAA1DAA1EAA1FAA18AE8AA9807FCC
:10A9B0008AAB67E675E0C4010F94F7126C016CE690
:10A9C00075E0C4010F94F7125C01C114D10451F079
:10A9D000F60180858F70843029F4818592850E94EC
:10A9E000EF20182FEFEFE10FEB3008F09DC10E2E96
:10A9F000000CFF0B8827E050FB4A8F4F0D945E47F9
:10AA00001855A6558455CB55945694561356F05563
:10AA100037564856605662EA76E08DCF65EA76E0B2
:10AA2000C4010F94F7121BE08ACF6AEA76E0F8CFF0
:10AA30001701512C412CA701FF0C660B770BCE019F
:10AA4000C1960E948776EA962FAFEA97EB963FAFC2
:10AA5000EB97EC964FAFEC97ED965FAFED97EE96D8
:10AA60006FAFEE97EF967FAFEF97C158DF4F8883B8
:10AA7000CF57D040C058DF4F9883C058D040809106
:10AA80003102893020F4809130028930B8F165E9D3
:10AA90007DE082ED9FE00E94AFF000E020E030E337
:10AAA00040E150E0BE016F5F7F4FCE01C1960E9432
:10AAB0008879BC0182ED9FE00E9499F069E87DE011
:10AAC00082ED9FE00E94AFF0612F110F770B4AE0FB
:10AAD00050E082ED9FE00E9450F067E87DE082ED5B
:10AAE0009FE00E94AFF0D4016D917C9182ED9FE0D8
:10AAF0000E9499F082ED9FE00E9443EFA114B104FF
:10AB000009F016C1D12C71C31701512C412CB2018F
:10AB1000A701CE01C1960E948776E2962FAFE297F9
:10AB2000E3963FAFE397E4964FAFE497E5965FAFC8
:10AB3000E597E6966FAFE697E7967FAFE797E896DB
:10AB40008FAFE897E9969FAFE99799CFFE24EF245E
:10AB5000FE241701512C412CB201A101CE01C19656
:10AB60000E948776AA962FAFAA97AB963FAFAB9776
:10AB7000AC964FAFAC97AD965FAFAD97AE966FAF5B
:10AB8000AE97AF967FAFAF97E0968FAFE097E19625
:10AB90009FAFE19774CFFE24EF24FE241701512CC0
:10ABA000412CB201A101CE01C1960E948776A296E6
:10ABB0002FAFA297A3963FAFA397A4964FAFA497AA
:10ABC000A5965FAFA597A6966FAFA697A7967FAFFE
:10ABD000A797A8968FAFA897A9969FAFA9974FCF91
:10ABE000FF241701512C412CB201A701CE01C196BF
:10ABF0000E9487766A962FAF6A976B963FAF6B97E6
:10AC00006C964FAF6C976D965FAF6D976E966FAF0A
:10AC10006E976F967FAF6F97A0968FAFA097A19614
:10AC20009FAFA1972CCFEF2CFF241701512C412C63
:10AC3000B201A701CE01C1960E94877662962FAF1E
:10AC4000629763963FAF639764964FAF649765963C
:10AC50005FAF659766966FAF669767967FAF6797AA
:10AC600068968FAF689769969FAF699708CF17016D
:10AC7000512C412C8AA9807F86608AAB2AE030E083
:10AC8000D7010F9475476DAB7EAB8FAB98AFF7CE06
:10AC90001701512C412C8AA9807F87608AABB701AC
:10ACA000FF0C880B990B0F94A44520E030E048EC92
:10ACB00052E40F94FD476DAB7EAB8FAB98AFDFCE08
:10ACC000C10124E0969587952A95E1F70F946020BD
:10ACD000FFE02F22332402C0969587952A94E2F74D
:10ACE000817099271C01512C412CB201AC01CE017D
:10ACF000C1960E9487762A962FAF2A972B963FAF50
:10AD00002B972C964FAF2C972D965FAF2D972E96A5
:10AD10006FAF2E972F967FAF2F9760968FAF60976C
:10AD200061969FAF6197ABCE212C312C2101A7CE2C
:10AD3000F50180858F708550823008F0E3CEB50133
:10AD4000CE01C1960E94C57C29A33AA34BA35CA364
:10AD50006DA37EA38FA398A788E0FE01B196DE01C4
:10AD6000999601900D928A95E1F788E0FE01B996D7
:10AD7000DE01D19601900D928A95E1F789A98111A2
:10AD800003C08AA98F7009F180913102893008F4DB
:10AD9000B9C262E07DE082ED9FE00E94AFF000E08A
:10ADA00020E030E340E150E0BE016F5F7F4FCE0115
:10ADB000C1960E948879BC0182ED9FE00E9499F0C3
:10ADC00082ED9FE00E9443EF9DCE62E176E0C501F7
:10ADD0000F94F7127C01009709F494CEDC011896C9
:10ADE0008C918F70823009F41DC1843009F08ACEB5
:10ADF00080913102893020F480913002893090F0C6
:10AE000068E37DE082ED9FE00E94AFF0D7011996E4
:10AE10006D917C9182ED9FE00E9499F082ED9FE020
:10AE20000E9443EFC657DF4FE881F981CA58D040EE
:10AE3000309709F471C380858F70863009F06AC33A
:10AE4000D7011996CD90DC90C114D10409F462C3E6
:10AE5000D3011296ED91FC9162E0848195810F946B
:10AE6000A913B6010F94F7120F94D8226C01892B05
:10AE700009F450C380913102893020F4809130026E
:10AE80008930A8F066E27DE082ED9FE00E94AFF09D
:10AE9000F60141855285638574852AE030E082EDB4
:10AEA0009FE00E9408F082ED9FE00E9443EFD701EF
:10AEB00019966D917C91D3011496ED91FC91828944
:10AEC00093890F94F7127C01009709F423C367E676
:10AED00075E00F94F712009749F0FC0120852F7060
:10AEE000243021F4818592850E94EF20D6011996A5
:10AEF0004D915D916D917C911C97CE01C1960E9400
:10AF0000877622962FAF229723963FAF23972496DA
:10AF10004FAF249725965FAF259726966FAF26975C
:10AF200027967FAF279728968FAF289729969FAFB0
:10AF300029976CE675E0C7010F94F712BC010097E2
:10AF400021F1FC0190859F7095509230F0F4CE0174
:10AF5000C1960E94C57C298B3A8B4B8B5C8B6D8B89
:10AF60007E8B8F8B988F88E0FE017196DE0159965B
:10AF700001900D928A95E1F788E0FE017996DE0155
:10AF8000D19601900D928A95E1F780913102893036
:10AF900020F4809130028930D8F061E17DE082EDCB
:10AFA0009FE00E94AFF000E020E030E340E150E09D
:10AFB000BE016F5F7F4FCE01C1960E948879BC01B0
:10AFC00082ED9FE00E9499F082ED9FE00E9443EFA6
:10AFD000D60118968C911897982F92959F7090FD96
:10AFE00099C221E0CF57DF4F2883C158D0409160EC
:10AFF0009295907F8F70892B18968C93DD24D39433
:10B00000C957DF4FB881C758D040BB2309F406C1E8
:10B01000C857DF4F48815981C858D040452B09F4A3
:10B02000FDC08CC280913102893020F480913002C1
:10B030008930A8F061E77DE082ED9FE00E94AFF0EB
:10B04000F70141855285638574852AE030E082ED01
:10B050009FE00E9408F082ED9FE00E9443EFD7013D
:10B0600019966D917D918D919C911C97C457DF4FDE
:10B07000E881F981CC58D0408F0130E020E06017A2
:10B080007107820793070CF455C0C257DF4F488100
:10B090005981CE58D0408A0130E020E006171707CA
:10B0A000280739070CF446C0AB014E1B5F0BDE01CD
:10B0B000AF57BF4F5D01C12CC257DF4FE880F98009
:10B0C000CE58D0408F01CD57DF4F2881C358D04094
:10B0D000C3010E94295429AB3AAB4BAB5CAB6DABBF
:10B0E0007EAB8FAB98AF80913102893020F4809194
:10B0F00030028930E0F06EEA76E082ED9FE00E9457
:10B1000099F06BEC76E082ED9FE00E9499F0CF57CA
:10B11000DF4F6881C158D04070E04AE050E082EDD6
:10B120009FE00E9450F082ED9FE00E9443EFDD24FB
:10B13000D3945BC067E67DE082ED9FE00E94AFF0B4
:10B14000F70141855285638574852AE030E082ED00
:10B150009FE00E9408F068E47DE082ED9FE00E949D
:10B16000AFF082ED9FE00E9443EF81E08093D50D28
:10B17000CE01419690935B0E80935A0ECD57DF4FD0
:10B18000F881C358D0406F2F70E041E050E0D70104
:10B1900019968D919C910E94072CD82E8823E1F05E
:10B1A000F701618572859E012F573F4F5901C12CD0
:10B1B0007B018B01CD57DF4F2881C358D04050E031
:10B1C00040E0C3010E94295429AB3AAB4BAB5CABC6
:10B1D0006DAB7EAB8FAB98AF80E48093D50D8AEDDD
:10B1E0009DE090935B0E80935A0EC957DF4FB88154
:10B1F000C758D040BB2349F0C857DF4FE881F981D9
:10B20000C858D040EF2B09F099C1C657DF4FE881ED
:10B21000F981CA58D040EF2B09F447C0C657DF4F19
:10B22000A881B981CA58D04018968C9118978F7010
:10B230008630D9F5F40160817181CD010F94F71248
:10B240003C01009791F10F94D8227C01009709F4FA
:10B25000D6C0FC0181859285A385B48582159305AE
:10B26000A405B50509F09CC0C957DF4FF881C75840
:10B27000D040F11157C0D70118968C91189782953C
:10B280008F7080FD4FC091E0CB57DF4FE881F9818F
:10B29000C558D040908381608295807F18969C919C
:10B2A00018979F70892B18968C9388E0FE01F19671
:10B2B000DE01D99601900D928A95E1F729AD3AAD5C
:10B2C0004BAD5CAD6DAD7EAD8FAD21969FAD219741
:10B2D000C157DF4F0FB6F894DEBF0FBECDBFDF9171
:10B2E000CF911F910F91FF90EF90DF90CF90BF9083
:10B2F000AF909F908F907F906F905F904F903F9016
:10B300002F90089580913002893008F4FBCB41CD15
:10B31000F3016281738140E050E1CE01C1960E9449
:10B320009D7573CFCB57DF4FA881B981C558D040E9
:10B330001C92DD2009F4B9CFC957DF4FB881C75837
:10B34000D040BB2309F4B1CFCF57DF4F8881C1581C
:10B35000D04081110AC0CB57DF4FA881B981C558B1
:10B36000D0408C91882309F4A0CF912C812CB12C52
:10B37000A12CD12CC12CE9A8FAA80BA91CA92DA994
:10B380003EA94FA958AD6FEFC3010E94A13B81E0D8
:10B39000CB57DF4FE881F981C558D040808385CFF6
:10B3A000218632864386548680913102893020F48A
:10B3B000809130028930F8F060ED76E082ED9FE018
:10B3C0000E9499F02AE030E0B201A10182ED9FE0F5
:10B3D0000E945EEF6EED76E082ED9FE00E9499F0B4
:10B3E000D4016D917C9182ED9FE00E9499F082EDF5
:10B3F0009FE00E9443EFF70180858F7E8087D11008
:10B400009BCFCB57DF4FA881B981C558D0408C91D5
:10B41000882309F44ACFC957DF4FB881C758D040B5
:10B42000BB2309F442CFF30180858F708530D1F5BD
:10B430008681978160E775E00F94F712CD57DF4F53
:10B4400099838883C358D040009771F1DC01189626
:10B450008C9118978F70823039F519968D919D9146
:10B460000D90BC91A02D82159305A405B505E1F4BE
:10B4700080913102893020F480913002893050F07F
:10B480006BED7CE082ED9FE00E94AFF082ED9FE0EB
:10B490000E9443EFCB57DF4FE881F981C558D04078
:10B4A000108203CFC301C6CF912C812CB12CA12CCB
:10B4B000D12CC12CE9A8FAA80BA91CA92DA93EA939
:10B4C0004FA958AD6FEFC3010E94A13BCD57DF4F8D
:10B4D00028813981C358D0402115310509F4E5CEC2
:10B4E000D30118968C9187FDE0CEF9012186328632
:10B4F00043865486DACE19821A821B821C828A8184
:10B50000807F8A831D821E821F82188688E0FE014A
:10B510003196CECED12C74CDC957DF4FE881C758B4
:10B52000D040EE2309F4C1CEC857DF4F28813981BE
:10B53000C858D040D12C232B09F4B7CEC857DF4FC1
:10B54000A881B981C858D04018968C9118978F70EF
:10B55000823009F05ACE19968D919D910D90BC9133
:10B56000A02D81309105A105B10509F4D1CE029736
:10B57000A105B10509F049CED30112966D917C91D8
:10B5800040E050E2CACE2F923F924F925F926F926C
:10B590007F928F929F92AF92BF92CF92DF92EF9263
:10B5A000FF920F931F93CF93DF93CDB7DEB76897CA
:10B5B0000FB6F894DEBF0FBECDBF6115710509F45B
:10B5C00091C05E8B498B9D8B8C8BFB018680978015
:10B5D0008114910409F486C0F40180858F70823053
:10B5E00031F0853031F1F40182809380F1CF6184B4
:10B5F000728441E050E069897E89C3010E94072C72
:10B60000882389F3B12CA12CCC24C394730183012A
:10B61000298950E040E0B3018C899D890E9429541A
:10B6200029873A874B875C876D877E878F87988BC2
:10B63000DACFC4010F943A148230A9F660E0C40155
:10B640000F94A913FC01C184D284E384F48461E0E3
:10B65000C4010F94A913FC012184328443845484CF
:10B66000388E2F8ADB8ACA8AA1014C195D094F5F87
:10B670005F4F69897E89C6010E94072C882309F4DF
:10B68000B2CF80913102893020F48091300289302C
:10B6900020F082ED9FE00E9443EF712C612C6A89BB
:10B6A0007B89660D771D8F89988D861797070CF417
:10B6B0009ACFB12CA12CCC24C39471010A891B8987
:10B6C0002989A3018C899D890E94295429833A8361
:10B6D0004B835C836D837E838F8398879FEF691A8A
:10B6E000790ADDCF68960FB6F894DEBF0FBECDBFE6
:10B6F000DF91CF911F910F91FF90EF90DF90CF904E
:10B70000BF90AF909F908F907F906F905F904F9081
:10B710003F902F9008952F923F924F925F926F9299
:10B720007F928F929F92AF92BF92CF92DF92EF92D1
:10B73000FF920F931F93CF93DF9300D01F921F921E
:10B74000CDB7DEB761307105D1F490E080E00F90A5
:10B750000F900F900F900F90DF91CF911F910F914D
:10B76000FF90EF90DF90CF90BF90AF909F908F9021
:10B770007F906F905F904F903F902F900895209111
:10B78000C9093091CA09232B01F78C01DC01ED9125
:10B79000FC910284F385E02D19950297B1F6809112
:10B7A000CF099091D009A091D109B091D209892BEC
:10B7B0008A2B8B2B79F4D8011296ED91FC9162E0E3
:10B7C000848195810F94A9139C838B83892BB1F479
:10B7D000B12C0BC40F94C927C090CF09D090D009C9
:10B7E000E090D109F090D2096C197D098E099F096A
:10B7F000683C710581059105F0F6A7CFEB81FC81CE
:10B8000080858F70863021F7C680D7801D82B12C4D
:10B81000C114D10409F4E5C3D60118968C91982F70
:10B820009F702BEF290F223008F0DBC3BD81B111CF
:10B83000D8C3282F22952F7087FF7AC522FD78C59F
:10B84000953009F0A7C0F6018681978160E775E021
:10B850000F94F7121C01892B09F46AC581E090E06E
:10B860009093CA098093C909B11003C0C8010E940E
:10B87000872CD10119964D905C9069EE76E082EDAF
:10B880009FE00E9499F0D8011296ED91FC91028000
:10B89000F381E02D6081718182ED9FE00E9499F03B
:10B8A0006DE578E082ED9FE00E9499F0F6016081FD
:10B8B000718182ED9FE00E9499F06CEC75E082ED61
:10B8C0009FE00E9499F0D10119964D915D916D9183
:10B8D0007C911C972AE030E082ED9FE00E9408F006
:10B8E00082ED9FE00E9443EFF60180809180D801B5
:10B8F0001496ED91FC916AE77EE0309759F0B4011F
:10B90000828993890F94F7127C01009709F044C053
:10B9100067E57EE08DE29FE00E94AFF08DE29FE060
:10B920000E9443EFEE24EA94FE2C4201550CAA0833
:10B93000BB08D10119964D905D906D907C901C973D
:10B9400084149504A604B70409F4A7C48091CF0910
:10B950009091D009A091D109B091D209892B8A2B5D
:10B960008B2B09F486CF0F94C9272091CF093091F2
:10B97000D0094091D1095091D209621B730B840BFD
:10B98000950B683C71058105910508F072CF0E9406
:10B9900033A4D6CFC6015ACF66E176E00F94F712F2
:10B9A0003C01892B79F465EA76E0C7010F94F71220
:10B9B0003C0164E37EE0892B69F0F10180858F70A2
:10B9C000806B8087D30118968C918F70823079F0CC
:10B9D0006EE17EE08DE29FE00E94AFF08DE29FE09D
:10B9E0000E9443EFEEEFEE2EFF24FA949ECF69E023
:10B9F00076E0C7010F94F7127C01009709F442C169
:10BA0000FC0180858F70813009F061C181858823B8
:10BA100009F45DC1D10118968C91807FF12CE12C45
:10BA2000803B19F072E0E72EF12C63E17EE082EDBD
:10BA30009FE00E94AFF0B40182ED9FE00E9499F078
:10BA400060E17EE082ED9FE00E94AFF0F30141856E
:10BA50005285638574852AE030E082ED9FE00E9484
:10BA600008F065EF76E082ED9FE00E9499F04AE0F1
:10BA700050E0B70182ED9FE00E9450F064E875E06D
:10BA800082ED9FE00E9499F0F1E0F093D50D81E006
:10BA900090E08C0F9D1F90935B0E80935A0E41E0B7
:10BAA00050E0B701D30119968D919C910E94072C0B
:10BAB000F82E4FEF5FEFBA0180E00F94C30F609351
:10BAC000CF097093D0098093D1099093D209FF20B8
:10BAD00009F4FAC0D8011296ED91FC9162E08481DC
:10BAE00095810F94A9137C01009709F4C2C0FC0151
:10BAF00080858F70863009F0E7C0B401C7010F94CC
:10BB0000F7127C01009709F4B4C00F94D8227C018D
:10BB1000892B09F4AEC080913102893020F48091E4
:10BB20003002893028F169E07EE082ED9FE00E94DA
:10BB3000AFF0D70119964D915D916D917C911C9755
:10BB40002AE030E082ED9FE00E9408F063E07EE0B2
:10BB500082ED9FE00E94AFF069817A814AE050E077
:10BB600082ED9FE00E9460EF82ED9FE00E9443EF34
:10BB7000F701418552856385748589819A81B0E09A
:10BB8000A0E0481759076A077B0719F16DEF7DE0C0
:10BB900082ED9FE00E94AFF0B40182ED9FE00E9431
:10BBA00099F06FEE7DE082ED9FE00E94AFF082EDB4
:10BBB0009FE00E9443EFF0E4F093D50D8AED9DE005
:10BBC00090935B0E80935A0E6DEFE62EFF24FA944D
:10BBD000ACCEF10181859285A385B48548175907BC
:10BBE0006A077B0789F569EE7DE082ED9FE00E94A0
:10BBF000AFF0B40182ED9FE00E9499F067EE7DE026
:10BC000082ED9FE00E94AFF069817A814AE050E0C6
:10BC100082ED9FE00E9460EF66ED7DE082ED9FE0A7
:10BC20000E94AFF082ED9FE00E9443EFF0E4F093BA
:10BC3000D50D8AED9DE090935B0E80935A0E5CEFDC
:10BC4000E52EFF24FA9471CE60ED7DE082ED9FE059
:10BC50000E94AFF0B40182ED9FE00E9499F065EB85
:10BC60007DE082ED9FE00E94AFF082ED9FE00E94B8
:10BC700043EF90E49093D50DAAEDBDE0B0935B0E39
:10BC8000A0935A0ED1011896EC91E295EF70E15015
:10BC9000AA24AA94BA2CEB3008F066C0F0E0D301D5
:10BCA00019962D913C918827E75AF14A8F4F0D94B0
:10BCB0005E476A5E7F5E6A5E7F5E295F245F295F02
:10BCC000245F6A5E6A5E355FF12CE12CD2CFF12CE5
:10BCD000E12CD8CFF1018185928530935D0E2093C0
:10BCE0005C0E10925F0E10925E0E9093610E809328
:10BCF000600E86E00F945829A82EB12C35C0D101D2
:10BD000019968D919C9198278927982730935D0EDD
:10BD100020935C0E10925F0E10925E0E9093610E57
:10BD20008093600E86E00F945829A82EB12CF10163
:10BD300081859285A385B4853A2F2B2FD30119963F
:10BD40008D919C91019690935D0E80935C0E109264
:10BD50005F0E10925E0E3093610E2093600E86E0AF
:10BD60000F945829A80EB11C4FEF5FEFBA0180E085
:10BD70000F94C30F6093CF097093D0098093D109BA
:10BD80009093D2096AEA7DE082ED9FE00E94AFF0D5
:10BD90004AE050E0B50182ED9FE00E9450F068EA71
:10BDA0007DE082ED9FE00E94AFF0B40182ED9FE064
:10BDB0000E9499F06CEF76E082ED9FE00E9499F08E
:10BDC000F30141855285638574852AE030E082ED78
:10BDD0009FE00E9408F062EA7DE082ED9FE00E9411
:10BDE000AFF0D10119964D915D916D917C911C97A9
:10BDF0002AE030E082ED9FE00E9408F082ED9FE0B3
:10BE00000E9443EFA114B104B9F4F10180858F7051
:10BE1000823091F4E114F10479F0D70118968C91F5
:10BE20008F70823049F481859285A385B485F701AE
:10BE300081879287A387B48791E080E0AB2809F0DF
:10BE400090E0E92EF82E71CDF10181859285992738
:10BE500044CFF10181859285A385B485892F9A2FDE
:10BE6000AB2FBB27A7FDBA95F2CFD10119968C91C4
:10BE700030935D0E20935C0E882341F080E09FEFAD
:10BE800090935F0E80935E0E85E034CF90E080E06B
:10BE9000F7CFD60118968C911897806418968C93DA
:10BEA00067E07FE08DE29FE00E94AFF0D80112963C
:10BEB000ED91FC910280F381E02D608171818DE232
:10BEC0009FE00E9499F06DE578E08DE29FE00E948E
:10BED00099F0F601608171818DE29FE00E9499F0F6
:10BEE00069EF7EE08DE29FE00E94AFF0D6011896E8
:10BEF0008C911897982F92959F70292F237023303B
:10BF000039F09F5F9295907F8F70892B18968C9354
:10BF100061EF7EE08DE29FE00E94AFF0D8011296C3
:10BF2000ED91FC910280F381E02D608171818DE2C1
:10BF30009FE00E9499F06DE578E08DE29FE00E941D
:10BF400099F0F601608171818DE29FE00E9499F085
:10BF500062E077E08DE29FE00E9499F0D6011896AA
:10BF60006C916295637070E04AE050E08DE29FE072
:10BF70000E9450F08DE29FE00E9443EFD7C163EE34
:10BF80007EE08DE29FE00E94AFF0D8011296ED9125
:10BF9000FC910280F381E02D608171818DE29FE050
:10BFA0000E9499F06DE578E08DE29FE00E9499F0A3
:10BFB000F601608171818DE29FE00E9499F060ED51
:10BFC0007EE08DE29FE00E94AFF08DE29FE00E9454
:10BFD00043EFD60118968C9118978F7018968C9312
:10BFE000A5C11092CA091092C909D8011496ED9101
:10BFF000FC91C480D580F12CE12C0F94C927C11489
:10C00000D104E104F10491F0D8011496ED91FC9172
:10C010004680578060847184641975098609970980
:10C020006C157D058E059F0508F4C3C08091CF096E
:10C030009091D009A091D109B091D209892B8A2B76
:10C040008B2B09F0A2C0EB81FC81EF2B09F0B8C06B
:10C05000D8011496ED91FC9182859385892B69F422
:10C0600084859585892B49F486859785892B29F4C4
:10C0700080899189892B09F4FFC080913102893030
:10C0800020F4809130028930B8F06AEA7EE082EDD7
:10C090009FE00E94AFF0D8011296ED91FC910280D2
:10C0A000F381E02D6081718182ED9FE00E9499F023
:10C0B00082ED9FE00E9443EF81E090E09093CA09F7
:10C0C0008093C909B11003C0C8010E94872CD80110
:10C0D0001496ED91FC916285738542E050E0C801B1
:10C0E0000E94C35AD8011496ED91FC916485758520
:10C0F00043E050E0C8010E94C35AD8011496ED9164
:10C10000FC916685778550E040E0C8010E94C35AE3
:10C11000D8011496ED91FC916089718941E050E05D
:10C12000C8010E94C35A80913102893020F4809165
:10C1300030028930B8F06AE97EE082ED9FE00E942B
:10C14000AFF0D8011296ED91FC910280F381E02DC1
:10C150006081718182ED9FE00E9499F082ED9FE005
:10C160000E9443EF0F94C9276B017C010F94C927EC
:10C170006C197D098E099F0962337105810591054E
:10C1800008F076C00E9433A4F1CF0F94C927C09065
:10C19000CF09D090D009E090D109F090D2096C1964
:10C1A0007D098E099F09683C71058105910508F09C
:10C1B0004ACFD8011496ED91FC9184819581C7CA2C
:10C1C000AB81BC8118968C9118978F70863009F0DE
:10C1D0003FCF1696ED90FC90E114F10409F438CFAE
:10C1E000F7018085982F9F702BEF290F223008F0E0
:10C1F0002FCF82958F7082FF05C08B708295807FD4
:10C20000892B8087D70118968C9182958370833013
:10C2100059F56DE077E08DE29FE00E9499F0D8013A
:10C220001296ED91FC910280F381E02D6081718185
:10C230008DE29FE00E9499F06DE578E08DE29FE04D
:10C240000E9499F0F701608171818DE29FE00E9468
:10C2500099F08DE29FE00E9443EFD70118968C91F0
:10C2600018978F7018968C93F701E280F380B4CF03
:10C270001092CA091092C909F801E480F5804FEFC5
:10C280005FEFBA0180E00F94C30FD70116966D934C
:10C290007D938D939C9319978CCFBDEFEB16BFEFD9
:10C2A000FB0609F46CCEACF5FCEFEF16FFEFFF06D2
:10C2B000B9F162EC7EE08DE29FE00E94AFF0D80120
:10C2C0001296ED91FC910280F381E02D60817181E5
:10C2D0008DE29FE00E9499F06DE578E08DE29FE0AD
:10C2E0000E9499F0F601608171818DE29FE00E94C9
:10C2F00099F067EB7EE08DE29FE00E94AFF08DE267
:10C300009FE00E9443EFD60118968C9118978F7783
:10C3100065CEE114F10409F4BCCDEA94EF2849F6A6
:10C32000F60180858F708087F1E0FD83BB24B39494
:10C33000F601C280D3806CCA8F929F92AF92BF9257
:10C34000CF92DF92EF92FF920F931F93CF93DF93E1
:10C3500000D000D01F921F92CDB7DEB7E982FA82DB
:10C360000B831C832D833E834F835887DC011296F9
:10C37000ED91FC91309791F1048115810115110522
:10C3800069F1F80180858F70853041F57B01C80126
:10C390000F943A14823010F161E0C8010F94A91390
:10C3A0000097E1F0DC0118962C912F702630B1F443
:10C3B000B7010F94F712009789F0912C812CB12CC2
:10C3C000A12CD12CC12CE980FA800B811C812D81FC
:10C3D0003E814F8158856FEF0E94A13B28960FB692
:10C3E000F894DEBF0FBECDBFDF91CF911F910F91AB
:10C3F000FF90EF90DF90CF90BF90AF909F908F9085
:10C4000008953F924F925F926F927F928F929F9288
:10C41000AF92BF92CF92DF92EF92FF920F931F9352
:10C42000CF93DF93CDB7DEB7C75AD1090FB6F894D3
:10C43000DEBF0FBECDBFDC0114962D913C91159748
:10C44000232B09F4D2C58B016C01ED91FC91028480
:10C45000F385E02D19958230910509F418C1C4F5D2
:10C4600097FFC3C5F60187819085DC01ED91FC91B2
:10C470000084F185E02D199585970CF4F4C045E210
:10C4800050E0BE016F5F7F4FF601878190850E946B
:10C49000C5EED60117968D919C91DC01ED91FC9132
:10C4A0000084F185E02D1995892B09F437C162E0EC
:10C4B00070E080E090E00F94C925F60187819085B7
:10C4C000DC01ED91FC910284F385E02D1995E1CF1B
:10C4D0008430910509F474C0C4F1059719F6013050
:10C4E000110509F000C162EA79E082ED9FE00E9447
:10C4F000D3F04DE050E060E072E0C6010E941221EE
:10C50000F601048115814FEF5FEFBA0180E00F94CF
:10C51000C30FD80198966D937D938D939C939B97B1
:10C52000D601ED91FC910484F585E02D62E0C60111
:10C530001995D6011496ED91FC9115978FEF808394
:10C540001496ED91FC9181838DCFD6011496ED91D7
:10C55000FC9180A591A5A2A5B3A5892B8A2B8B2B35
:10C5600009F480CF0F94C927D6011496ED91FC9160
:10C57000159700A511A522A533A5601B710B820B91
:10C58000930B663971058105910508F46BCFED9128
:10C59000FC910484F585E02D62E0C6011995F60151
:10C5A000048115814FEF5FEFBA0180E00F94C30F54
:10C5B000D80198966D937D938D939C939B9752CFC2
:10C5C000D6011496ED91FC9180A591A5A2A5B3A5E5
:10C5D000892B8A2B8B2BD9F10F94C927D60114965E
:10C5E000ED91FC9100A511A522A533A5601B710B4F
:10C5F000820B930B683873418105910540F1D60198
:10C60000ED91FC910484F585E02D65E0C601199556
:10C61000F601048115814FEF5FEFBA0180E00F94BE
:10C62000C30FD80198966D937D938D939C939B97A0
:10C63000D6011496ED91FC9117A26EEA79E082ED95
:10C640009FE00E94AFF082ED9FE00E9443EFF60171
:10C6500087819085DC01ED91FC910084F185E02DCE
:10C660001995892B19F481E090E03FC062E070E0F9
:10C6700080E090E00F94C925F60187819085DC0168
:10C68000ED91FC910284F385E02D1995E0CFD60160
:10C690001496ED91FC9180A591A5A2A5B3A5892B37
:10C6A0008A2B8B2BE1F00F94C927D6011496ED91BC
:10C6B000FC9140A451A462A473A46419750986096D
:10C6C0009709683873418105910548F0D601ED91CD
:10C6D000FC910484F585E02D65E0C60119950130D3
:10C6E000110509F4BFCE90E080E0C955DF4F0FB6C9
:10C6F000F894DEBF0FBECDBFDF91CF911F910F9198
:10C70000FF90EF90DF90CF90BF90AF909F908F9071
:10C710007F906F905F904F903F9008956EE979E021
:10C7200082ED9FE00E94AFF04AE050E0F6016681A2
:10C7300082ED9FE00E9466EF69E979E082ED9FE07B
:10C740000E94AFF08E010F5F1F4F7E01F5E2EF0EEA
:10C75000F11CD8016D918D0140E150E06A3058F430
:10C7600068E475E082ED9FE00E9499F040E150E0BE
:10C77000F8013197608182ED9FE00E9466EFE0163C
:10C78000F10639F76EE282ED9FE00E9401F082ED42
:10C790009FE00E9443EFFE01339680E00E171F07D3
:10C7A00019F09191890FFACF9DA1981313C462E9F2
:10C7B00079E082ED9FE00E94AFF082ED9FE00E9461
:10C7C00043EF8DA1D6011496ED91FC91159797A199
:10C7D000891709F448CF87A314960D90BC91A02D1A
:10C7E00085E2FE01319601900D928A95E1F7D6011E
:10C7F0001496ED91FC91C056DF4F188219821A826F
:10C800001B82C05AD040CC55DF4F188219821A8241
:10C810001B82C45AD040CF55DF4F8881C15AD040C7
:10C82000807FCF55DF4F8883C15AD04083A190E0ED
:10C830004C01B0E18B0E911C499708F014CF358460
:10C84000878986A3118D738CD60114962D913C9106
:10C85000858DD90195968C93E48CF12C878DD6012A
:10C860001296ED91FC910280F381E02D40E257E0B9
:10C870006AE676E080FD02C06BE776E08081918118
:10C880000F948428B0E8EB16F10409F086C0D601B5
:10C890001296ED91FC910280F381E02D47E257E082
:10C8A0006AE676E0808191810F9484286DE277E0DA
:10C8B00082ED9FE00E9499F0D6011496ED91FC91D3
:10C8C0004AE050E065A182ED9FE00E9466EF82EDB4
:10C8D0009FE00E9443EFD6011496ED91FC911597CD
:10C8E00085A11296ED91FC910280F381E02D48E341
:10C8F00057E06AE676E083FD02C06BE776E0808170
:10C9000091810F948428D6011296ED91FC91139792
:10C910000280F381E02D808191811496ED91FC914C
:10C9200025A14FE357E06AE676E021FD02C06BE700
:10C9300076E00F9484281EA2113009F4F8C1E0F1CA
:10C94000123009F429C2133009F45BC262E879E0BD
:10C95000CE0186960F94D63F60E0CE0180569F4F61
:10C960000E946576E9962FAFE997EA963FAFEA977E
:10C97000EB964FAFEB97EC965FAFEC97ED966FAF02
:10C98000ED97EE967FAFEE97EF968FAFEF97C1588A
:10C99000DF4F9883CF57D04043C0EF2809F086CFB0
:10C9A000D6011296ED91FC910280F381E02D47E2D1
:10C9B00057E06BE776E076CF69E57AE0CE018696C0
:10C9C0000F94D63F60E1CE0180569F4F0E9465765E
:10C9D000C856DF4F2883C859D040C756DF4F388329
:10C9E000C959D040C656DF4F4883CA59D040C556B2
:10C9F000DF4F5883CB59D040C456DF4F6883CC59A2
:10CA0000D040C356DF4F7883CD59D040C256DF4F58
:10CA10008883CE59D040C156DF4F9883CF59D0403C
:10CA2000D6011296ED91FC910280F381E02D45EA4A
:10CA300055E0BE016A5D7F4F808191810F9484280B
:10CA4000C056DF4FE880C05AD040CF55DF4FF88046
:10CA5000C15AD040CE55DF4F0881C25AD040CD5583
:10CA6000DF4F1881C35AD040CC55DF4F2881C45ABC
:10CA7000D040CB55DF4F3881C55AD040CA55DF4F23
:10CA80004881C65AD040C955DF4F5881C75AD04057
:10CA900066EA75E0C6010E949C61D6011296ED918E
:10CAA000FC910280F381E02D4AEA55E06BE776E0E5
:10CAB000772011F06AE676E0808191810F948428D6
:10CAC000092C000CAA08BB08D6011296ED91FC9126
:10CAD0000280F381E02D608171810BE915E0A501F1
:10CAE0009401C6010E9490E6432C512C712C612CBC
:10CAF000BFEF3B1681F0D6011296ED91FC910280BA
:10CB0000F381E02D608171810BE417E0A3019201B4
:10CB1000C6010E9490E618AA19AA1AAA1BAA1CAA62
:10CB20001DAA1EAA1FAA89A9807F89ABB501A401ED
:10CB3000CE01C0960E948776E1962FAFE197E296EC
:10CB40003FAFE297E3964FAFE397E4965FAFE4978A
:10CB5000E5966FAFE597E6967FAFE697E7968FAFDE
:10CB6000E797E8969FAFE89779018A019B01AC01AE
:10CB70006CE975E0C6010E949C6118AA19AA1AAA5C
:10CB80001BAA1CAA1DAA1EAA1FAA89A9807F89AB5D
:10CB9000B301A201CE01C0960E94877628AF39AFBB
:10CBA0004AAF5BAF6CAF7DAF8EAF9FAF63E0CE019E
:10CBB000C8960E944376A9962FAFA997AA963FAF31
:10CBC000AA97AB964FAFAB97AC965FAFAC97AD96CD
:10CBD0006FAFAD97AE967FAFAE97AF968FAFAF9773
:10CBE000E0969FAFE09779018A019B01AC016CE46C
:10CBF00077E0C6010E949C611EA2D6011496ED91B9
:10CC0000FC9186A1811132C165E47AE0CE0186965D
:10CC10000F94D63F6EE0CE0180569F4F0E946576FE
:10CC2000A1962FAFA197A2963FAFA297A3964FAF21
:10CC3000A397A4965FAFA497A5966FAFA597A69666
:10CC40007FAFA697A7968FAFA797A8969FAFA897F5
:10CC5000D6011496ED91FC91159726A130E050E095
:10CC600040E01296ED91FC910280F381E02D60810D
:10CC7000718101E517E0C6010E9490E6D601149685
:10CC8000ED91FC9185A180FD14C06DEC79E0CE01A1
:10CC900086960F94D63F62E0CE0180569F4F0E9449
:10CCA000657628AB39AB4AAB5BAB6CAB7DAB8EAB7F
:10CCB0009FABD6011296ED91FC910280F381E02D9D
:10CCC00040EA55E0BE016A5D7F4F808191810F94FB
:10CCD0008428C056DF4FE880C05AD040CF55DF4F80
:10CCE000F880C15AD040CE55DF4F0881C25AD0409B
:10CCF000CD55DF4F1881C35AD040CC55DF4F288126
:10CD0000C45AD040CB55DF4F3881C55AD040CA55A0
:10CD1000DF4F4881C65AD040C955DF4F5881C75AA6
:10CD2000D04061EA75E0C6010E949C619CCC63E63C
:10CD30007AE0CE0186960F94D63F61E1CE0180560F
:10CD40009F4F0E946576C057DF4F2883C059D0405F
:10CD5000CF56DF4F3883C159D040CE56DF4F48837E
:10CD6000C259D040CD56DF4F5883C359D040CC561E
:10CD7000DF4F6883C459D040CB56DF4F7883C55905
:10CD8000D040CA56DF4F8883C659D040C956DF4FBE
:10CD90009883C759D04044CE6DE67AE0CE0186969E
:10CDA0000F94D63F62E1CE0180569F4F0E94657678
:10CDB000C857DF4F2883C858D040C757DF4F388344
:10CDC000C958D040C657DF4F4883CA58D040C557CE
:10CDD000DF4F5883CB58D040C457DF4F6883CC58BF
:10CDE000D040C357DF4F7883CD58D040C257DF4F74
:10CDF0008883CE58D040C157DF4F9883CF58D0405A
:10CE00000FCE65E47AE0CE0186960F94D63F6EE0B1
:10CE1000CE0180569F4F0E946576C058DF4F288311
:10CE2000C058D040CF57DF4F3883C158D040CE577D
:10CE3000DF4F4883C258D040CD57DF4F5883C35887
:10CE4000D040CC57DF4F6883C458D040CB57DF4F1A
:10CE50007883C558D040CA57DF4F8883C658D04022
:10CE6000C957DF4F9883C758D040DACD813029F5B4
:10CE70006BE87AE0CE0186960F94D63F65E1CE014D
:10CE800080569F4F0E94657669962FAF69976A9684
:10CE90003FAF6A976B964FAF6B976C965FAF6C978F
:10CEA0006D966FAF6D976E967FAF6E976F968FAFE3
:10CEB0006F97A0969FAFA097CBCE823029F561E8FF
:10CEC0007AE0CE0186960F94D63F64E1CE0180567B
:10CED0009F4F0E94657661962FAF619762963FAF34
:10CEE000629763964FAF639764965FAF649765965A
:10CEF0006FAF659766967FAF669767968FAF6797B8
:10CF000068969FAF6897A4CE833029F56FE47AE0E6
:10CF1000CE0186960F94D63F6FE0CE0180569F4F8C
:10CF20000E94657629962FAF29972A963FAF2A97B8
:10CF30002B964FAF2B972C965FAF2C972D966FAFFC
:10CF40002D972E967FAF2E972F968FAF2F976096A7
:10CF50009FAF60977DCE843029F565E97AE0CE01F8
:10CF600086960F94D63F66E1CE0180569F4F0E9471
:10CF7000657621962FAF219722963FAF2297239671
:10CF80004FAF239724965FAF249725966FAF2597D1
:10CF900026967FAF269727968FAF279728969FAF25
:10CFA000289756CE8D3609F053CE62E879E0CE014F
:10CFB00086960F94D63F60E0CE0180569F4F0E9428
:10CFC000657628AF39AF4AAF5BAF6CAF7DAF8EAF40
:10CFD0009FAF3ECE66E879E082ED9FE00E94AFF021
:10CFE00082ED9FE00E9443EF3ECB8FEF9FEF7DCB22
:10CFF0000F931F93CF93DF93EC010E949F3467E55B
:10D0000077E082ED9FE00E9447EF8091D3099091F5
:10D01000D409892B19F586E190E00F94913C8C019D
:10D020002B853C854A85042E000C550B6885798537
:10D030000E94FEF51093D4090093D309F80186816C
:10D04000978197FD1AC061E00F94842360E0F80196
:10D0500086810F94562381E0F8018183E881F9816C
:10D060000484F585E02D62E0CE01199581E090E021
:10D07000DF91CF911F910F9108951182EFCFE5E0DD
:10D08000F1E080818F7980830895E5E0F1E080818F
:10D090008066808308958FE090E090933B0C8093AE
:10D0A0003A0C88EC90E00895FC0184819581089504
:10D0B00060E273E2811102C062E273E285E29FE006
:10D0C0000C94AFF061EC7EE185E29FE00E94AFF04E
:10D0D000F0E0E0E0199584EF91E008958091500A26
:10D0E0008823B1F0E091510AF091520A309731F063
:10D0F0008681978190934F0A80934E0A66E17CE186
:10D1000085E29FE00E94AFF085E29FE00C9443EF40
:10D1100008952F923F924F925F926F927F928F92DB
:10D120009F92AF92BF92CF92DF92EF92FF920F93B6
:10D130001F93CF93DF93CDB7DEB768970FB6F89400
:10D14000DEBF0FBECDBF3C018091610A6DE778E282
:10D15000882309F46AC161E070E080E090E00F94F8
:10D16000C925BE016F5F7F4F80E00F94111F892B8F
:10D1700009F059C1898183FF56C144E0BE016F5F48
:10D180007F4F82E00F940B20009791F429813A8120
:10D1900032272327322730939F0D20939E0D2B811A
:10D1A0003C8132272327322730939D0D20939C0DFD
:10D1B0000F94DE1E6CE578E282ED9FE00E94AFF0F6
:10D1C00060919E0D70919F0D90E080E00F94A245BC
:10D1D000562E798B8A8B492E462F572F682F792F01
:10D1E00082ED9FE00F943D1864E578E282ED9FE0C8
:10D1F0000E94AFF060919C0D70919D0D90E080E0D9
:10D200000F94A2456B8B7C8B8D8B9E8BAB01BC01ED
:10D2100082ED9FE00F943D1868E478E282ED9FE094
:10D220000E94AFF042E0BE016F5F7F4F81E10F943B
:10D230000B2049815A81542745275427892B11F007
:10D2400050E040E070E060E040935D0A50935E0A79
:10D2500060935F0A7093600A2AE030E082ED9FE0FD
:10D260000E9408F020E030E44CE156E4652D798915
:10D270008A89942D0F949D4587FF7AC0D301129619
:10D28000ED91FC912080318064E677E0C1010F943C
:10D29000F712988F8F8B68E677E0C1010F94F71231
:10D2A0001C0119821A821B821C828A81807F8760FE
:10D2B000F82E8A83252D852D9989AA89B42D8D83F1
:10D2C0009E83AF83B887912C812CB12CA12CD12CBB
:10D2D000C12CE9800B811C813E814F8158856FEF05
:10D2E0008F89988D0E94A13B19821A821B821C8211
:10D2F0008A81807F8760F82E8A832B89822F9C8980
:10D30000AD89BE898D839E83AF83B887E9800B8109
:10D310001C813E814F8158856FEFC1010E94A13B66
:10D320002DE637E0452D59896A89742DC3010E9485
:10D3300068E622E737E04B895C896D897E89C30105
:10D340000E9468E660915D0A70915E0A80915F0AB2
:10D350009091600A2AE0AE014F5F5F4F0F946640E4
:10D3600048E757E0BE016F5F7F4FC3010E943EE672
:10D370006EE777E082ED9FE00E9447EFBE016F5FAE
:10D380007F4F80EE0F94111F892B19F419811F3FD5
:10D3900049F46FE178E28DE29FE00E94D3F081E0F2
:10D3A00090E04DC0112331F060E178E28DE29FE022
:10D3B0000E94AFF015FF06C063E078E28DE29FE0C7
:10D3C0000E94AFF014FF06C067EF77E28DE29FE0A6
:10D3D0000E94AFF013FF06C069EE77E28DE29FE096
:10D3E0000E94AFF012FF06C069ED77E28DE29FE088
:10D3F0000E94AFF011FF06C06AEC77E28DE29FE079
:10D400000E94AFF010FF0BC06FEB77E28DE29FE060
:10D410000E94AFF08DE29FE00E9443EFC0CF112346
:10D4200009F4BDCFF7CF62E678E282ED9FE00E947B
:10D43000AFF082ED9FE00E9443EF90E080E06896BD
:10D440000FB6F894DEBF0FBECDBFDF91CF911F9115
:10D450000F91FF90EF90DF90CF90BF90AF909F9093
:10D460008F907F906F905F904F903F902F90089596
:10D470002F923F924F925F926F927F928F929F92E4
:10D48000AF92BF92CF92DF92EF92FF920F931F93D2
:10D49000CF93DF93CDB7DEB760970FB6F894DEBFBA
:10D4A0000FBECDBF6130710579F42C0180915C0A0B
:10D4B000811125C066EA77E28DE29FE00E94AFF01D
:10D4C0008DE29FE00E9443EF90E080E060960FB60F
:10D4D000F894DEBF0FBECDBFDF91CF911F910F91AA
:10D4E000FF90EF90DF90CF90BF90AF909F908F9084
:10D4F0007F906F905F904F903F902F90089565E9D7
:10D5000077E282ED9FE00E94AFF082E00F94FC256D
:10D51000692E712C40E150E0B30182ED9FE00E9442
:10D5200050F08FEF6816710409F42DC160E877E0C0
:10D5300082ED9FE00E9499F080E00F94FC25BC01F1
:10D5400090E080E00F94A24520E030E040E857E30F
:10D550000F94034620E030E045E253E40F94034685
:10D5600020E030E040E252E40F949047762E272EE0
:10D57000382E692E462F572F682F792F82ED9FE086
:10D580000F943D186EE877E282ED9FE00E94AFF0C5
:10D5900081E00F94FC25BC0190E080E00F94A2454F
:10D5A00020E030E040E857E30F94034620E030E00D
:10D5B00048EC52E40F94034669877A878B879C87EF
:10D5C000AB01BC0182ED9FE00F943D1864E877E069
:10D5D00082ED9FE00E9447EFD2011296ED91FC91FF
:10D5E000E080F1806CE477E0C7010F94F7129E872A
:10D5F0008D8766E877E0C7010F94F712988B8F87C5
:10D60000272D322D432D562D672D722D832D962DCE
:10D610000F940549811140C019821A821B821C8215
:10D620008A81807F8760F82E8A83272D872D922D0F
:10D63000A32DB62D8D839E83AF83B887912C812C2B
:10D64000B12CA12CD12CC12CE9800B811C813E81F5
:10D650004F8158856FEF8D859E850E94A13B198271
:10D660001A821B821C828A81807F8760F82E8A83BF
:10D670002985822F9A85AB85BC858D839E83AF8358
:10D68000B887E9800B811C813E814F8158856FEFFF
:10D690008F8598890E94A13B2AE837E0472D522DBB
:10D6A000632D762DC2010E9468E62DE837E049859A
:10D6B0005A856B857C85C2010E9468E68091610A6B
:10D6C000882309F45DC020E030E048EC51EC672D80
:10D6D000722D832D962D0F949D4587FD51C020E01E
:10D6E00030E048E452E4672D722D832D962D0F947F
:10D6F000A54818160CF444C020E030E048EC52E491
:10D7000069857A858B859C850F94A5481816C4F188
:10D7100020E030E04AE754E469857A858B859C8572
:10D720000F9403460F94764866507F4F8F4F9F4F5C
:10D7300024EFC22EDD24D394E12CF12CA701960115
:10D740000F94E74629831A8220E030E04AE754E448
:10D75000672D722D832D962D0F9403460F947648D6
:10D760006E557D498F4F9F4FA70196010F94E74655
:10D770002B831C82BE016F5F7F4F85E00F94611F7A
:10D7800088EE93E0A3CE82ED9FE00E9443EF0F94DA
:10D79000490FF6CFEF92FF920F931F93CF93DF9332
:10D7A000CDB7DEB760970FB6F894DEBF0FBECDBF22
:10D7B00080915C0A8823C9F06AE277E282ED9FE0FB
:10D7C0000E94AFF082ED9FE00E9443EF90E080E086
:10D7D00060960FB6F894DEBF0FBECDBFDF91CF913C
:10D7E0001F910F91FF90EF9008956EE777E282ED21
:10D7F0009FE00E94AFF00F949B1F80E48093A80DE0
:10D800000F949B1F10E01B7F8091A80D0F94071FA2
:10D8100062E085E89DE00E949AEA612F85E89DE03C
:10D820000E949AEA60E085E89DE00E949AEA85E815
:10D830009DE00F94820B6AE070E080E090E00F942E
:10D84000C9256BE677E282ED9FE00E94AFF08EEF94
:10D850000F94FC2540E150E0BC0182ED9FE00E9466
:10D8600060EF6DE577E282ED9FE00E94AFF08FEF11
:10D870000F94FC2540E150E0BC0182ED9FE00E9446
:10D8800060EF82ED9FE00E9443EF67E477E285E27C
:10D890009FE00E94AFF08BEF0F94FC25182F092F0B
:10D8A0008CEF0F94FC25F82EE92E8DEF0F94FC25BC
:10D8B0009F938F93EF92FF920F931F9380E997E0CE
:10D8C0009F938F938E010F5F1F4F1F930F930F94A2
:10D8D000504CB80185E29FE00E9447EF81E08093C1
:10D8E0005C0A0FB6F894DEBF0FBECDBF81E090E0BA
:10D8F0006FCF0F931F93CF93DF9300D000D01F9271
:10D90000CDB7DEB78091610A882369F06DEE76E2CB
:10D910008DE29FE00E94AFF08DE29FE00E9443EF16
:10D9200090E080E0B0C06DE177E285E29FE00E9488
:10D93000D3F00F949B1F8091600290916102A0919F
:10D940006202B091630289839A83AB83BC8385E8CA
:10D950009DE09093920D8093910D1E8280E197E25D
:10D960002E812F5F2E830197D9F71D82BE016B5F39
:10D970007F4F80E20F94111F8C01892BF1F48D8170
:10D9800001E010E08138C9F4BE016F5F7F4F8FEF77
:10D990000F94611F1F8280E89EE32F812F5F2F83EA
:10D9A0000197D9F7BE016B5F7F4F80E00F94111F85
:10D9B0008D8180FF0CC003E010E069E077E28DE22A
:10D9C0009FE00E94AFF0C8010F94DE1EA9CFBE01F8
:10D9D0006B5F7F4F80E00F94111F892B61F78D8162
:10D9E00084FFE9CF8091930D0F94071F8091910DD3
:10D9F0009091920DDC01ED91FC910190F081E02D70
:10DA000064EF19958091910D9091920D0F94820B76
:10DA1000882319F002E010E0D0CFBE016B5F7F4F8A
:10DA200081E00F94111F8C01892B39F61D811F781D
:10DA300010611D838091930D0F94071F8091910DAC
:10DA40009091920DDC01ED91FC910190F081E02D1F
:10DA500061E019958091910D9091920DDC01ED910D
:10DA6000FC910190F081E02D612F19958091910D2D
:10DA70009091920D0F94820B8111CCCF81E0809315
:10DA8000610A81E090E027960FB6F894DEBF0FBEE2
:10DA9000CDBFDF91CF911F910F910895CF93DF9369
:10DAA00000D000D01F921F92CDB7DEB7EFE0FFE0AD
:10DAB000128A118A80E090E19587848784E890E05B
:10DAC000948B838B81E0868787E7858B1C821B8202
:10DAD00083EE92E09A838983FE83ED838FEF9FEF3D
:10DAE00098878F8363ED76E285E29FE00E94AFF036
:10DAF0006091DB097091DC09CE0101960F946D1ADB
:10DB00008FE09FE00E940CAC63EC76E285E29FE040
:10DB10000E94AFF085E29FE00E9443EF0F943A31FC
:10DB200028960FB6F894DEBF0FBECDBFDF91CF9120
:10DB30000895892B71F0FB01828193810F94C914A0
:10DB400069E073E285E29FE00E94AFF088EC90E02C
:10DB5000089590E080E0F2CF0F931F93CF93DF936F
:10DB6000EB0102970CF49FC00A811B816EEE71E2FB
:10DB7000C8010F94AF3F892B61F40F942F177E7F5C
:10DB80000F94891788EC90E0DF91CF911F910F914E
:10DB9000089568EF71E2C8010F94AF3F892B21F41B
:10DBA0000F942F177160ECCF64EC71E285E29FE077
:10DBB0000E94AFF00F942F17672F609561704AE0B5
:10DBC00050E070E085E29FE00E9450F085E29FE027
:10DBD0000E9443EF8091010F9091020F892B09F46D
:10DBE00052C00A811B810F944A14882309F44BC048
:10DBF000F80101900020E9F73197E01BF10BB09795
:10DC000008F041C0A091010FB091020F52961C92F2
:10DC10001E92519754961C921E92539784E890E05E
:10DC20001D969C938E931C971E961C921E9782E7BE
:10DC300055968C935597ED91FC9111970088F18939
:10DC4000E02D60E270E0CD011995B8018091010FDF
:10DC50009091020F0E9499F08091010F9091020F14
:10DC6000DC01ED91FC910190F081E02D60E01995CF
:10DC70008091010F9091020FDC01ED91FC910488DD
:10DC8000F589E02D19956A817B8185E29FE00E94EC
:10DC900099F06DEB71E285E29FE00E94AFF085E2C2
:10DCA0009FE00E9443EF80913A0C90913B0C0297C9
:10DCB0003CF080EF9FEF90933B0C80933A0C62CF47
:10DCC00060EB71E28DE29FE00E94AFF08DE29FE099
:10DCD0000E9443EF84EF91E057CFCF93DF93EB01A6
:10DCE0000297BCF16EEE71E28A819B810F94AF3F87
:10DCF000892B29F40F942F177D7F0F94891768EFD4
:10DD000071E28A819B810F94AF3F892B29F40F9494
:10DD10002F1772600F94891769E471E285E29FE022
:10DD20000E94AFF00F942F1771FB662760F971E026
:10DD3000672770E04AE050E085E29FE00E9450F0E3
:10DD400085E29FE00E9443EF88EC90E0DF91CF9165
:10DD500008950E944E6DF8CF892B71F0FB018281EE
:10DD600093810F942A156AE971E285E29FE00E948F
:10DD7000AFF088EC90E0089590E080E0F2CFEF9271
:10DD8000FF920F931F93CF93DF93CDB7DEB72C97FE
:10DD90000FB6F894DEBF0FBECDBF8C017B0189E1C9
:10DDA00095E09A8389831B821C821D821E8298873C
:10DDB0008F8319861A861B861C8605301105ECF0A8
:10DDC000BE01695F7F4FF701808591850E941932FE
:10DDD000892B99F0CE0107960F94F415BE01695F67
:10DDE0007F4FF701868197810E941932892B61F05C
:10DDF000CE0107960F94C6160EC0CE0101960F9461
:10DE0000F4150430110554F7CE0101960F94C6168F
:10DE100003301105A4F1BE01695F7F4FF7018481D2
:10DE200095810E941932892B51F1CE0107960F94EA
:10DE30005D16BE01695F7F4FF701828193810E9469
:10DE40001932892B19F1CE0107960F948B1563E8CF
:10DE500071E285E29FE00E94AFF080E00F94ED1741
:10DE600088EC90E02C960FB6F894DEBF0FBECDBFC5
:10DE7000DF91CF911F910F91FF90EF900895CE0108
:10DE800001960F945D16023011059CF6CE010196A5
:10DE90000F948B1501301105D1F6CE0101960F9428
:10DEA0008B156AE871E285E29FE00E94AFF0CFCF68
:10DEB000CF93C1E068EE73E080E090E00F94C92555
:10DEC0004AE050E06C2F85E29FE00E9466EFCF5F52
:10DED000C43181F784EF91E0CF9108950F931F93A0
:10DEE000CF93DF938C01EB010297C4F08A819B8171
:10DEF0000F94613F8093310299270F94F6170230F7
:10DF0000110549F08C819D810F94613F809330020F
:10DF100099270F940018C8ECD0E002C0C0E9D1E006
:10DF20006FE671E285E29FE00E94AFF04AE050E0C8
:10DF30006091310285E29FE00E9466EF6AE571E23E
:10DF400085E29FE00E94AFF04AE050E0609130022D
:10DF500085E29FE00E9466EF85E29FE00E9443EF2A
:10DF6000CE01DF91CF911F910F910895CF92DF9253
:10DF7000EF92FF920F931F93CF93DF93CDB7DEB74E
:10DF800069970FB6F894DEBF0FBECDBFE091BD0A12
:10DF9000F091BE0A309709F483C08091C70A90912E
:10DFA000C80A892B09F47CC08FEF838714861382FB
:10DFB000148215821682178210861186128662EEEE
:10DFC0007EE185E29FE00E94AFF085E29FE00E9443
:10DFD00043EF8E010F5E1F4FBE016E5E7F4F80913B
:10DFE000BD0A9091BE0A0F94090E18160CF058C085
:10DFF000A895DE0111969E012E5E3F4F7D01F9012D
:10E0000041919F01842F90E054E0959587955A9512
:10E01000E1F78C569D4FFC0180818C93E42FEF70CB
:10E02000F0E0EC56FD4F808111968C93119712967B
:10E03000A017B10721F7198AB7018091C70A9091FB
:10E04000C80A0F94F7126C016DED7EE185E29FE046
:10E050000E94AFF0B70185E29FE00E9499F0C114E1
:10E06000D104B9F0C6010E947F347C01892B09F4E8
:10E07000B3CF68ED7EE185E29FE00E94AFF0B7018B
:10E0800085E29FE00E9499F085E29FE00E9443EFC5
:10E09000A3CF63ED7EE185E29FE00E94AFF0F4CF75
:10E0A00088EC90E069960FB6F894DEBF0FBECDBF46
:10E0B000DF91CF911F910F91FF90EF90DF90CF9064
:10E0C0000895EF92FF920F931F93CF93DF9300D0A9
:10E0D00000D0CDB7DEB77C018B0168EE73E182ED35
:10E0E0009FE00E94AFF0D7011296ED91FC91608104
:10E0F000718182ED9FE00E9499F06FED73E182EDF6
:10E100009FE00E94AFF0012E000C220B330B09831D
:10E110001A832B833C8380E190E09E838D83BE0134
:10E120006F5F7F4F82ED9FE00E94FECF0E9443EF22
:10E1300040E050E860E070E0C7010E94E1B126963F
:10E140000FB6F894DEBF0FBECDBFDF91CF911F9108
:10E150000F91FF90EF900895CF92DF92EF92FF9290
:10E160000F931F93CF93DF93CDB7DEB7C154D1097F
:10E170000FB6F894DEBF0FBECDBF6C01AB0130E02F
:10E1800020E060E4CE0101967C010E942F31F7016E
:10E1900001900020E9F731978F010E191F09A8019E
:10E1A000B701C6010F94EB4B892B11F010E000E092
:10E1B000C801CF5BDF4F0FB6F894DEBF0FBECDBFF7
:10E1C000DF91CF911F910F91FF90EF90DF90CF9053
:10E1D00008953F924F925F926F927F928F929F929B
:10E1E000AF92BF92CF92DF92EF92FF920F931F9365
:10E1F000CF93DF93CDB7DEB72C970FB6F894DEBF81
:10E200000FBECDBF5C01362E972E3A01690169E43D
:10E2100074E182ED9FE00E94AFF04AE050E0632D90
:10E22000792D82ED9FE00E9450F061E474E182ED6F
:10E230009FE00E94AFF0C301B0E0A0E08F83988719
:10E24000A987BA8730E1432E512C5C864B86BE01EC
:10E25000695F7F4F82ED9FE00E94FECF4C016DE32E
:10E2600074E10E94AFF04AE050E0B601C4010E94A0
:10E2700050F065E374E1C4010E94AFF0C701B0E063
:10E28000A0E089839A83AB83BC835E824D82BE010A
:10E290006F5F7F4FC4010E94FECF0E9443EF8091C9
:10E2A000C9099091CA0970E060E0892B09F047C064
:10E2B00081E090E09093CA098093C90926E040E884
:10E2C00055E260E070E08DE39CE00E94FCF130924A
:10E2D000D40D8DE39CE09093D30D8093D20D1092DA
:10E2E000E20E1092E40E1092E30E0130110509F4D3
:10E2F0004EC00CF041C0012B09F44EC0C114D10432
:10E3000009F457C082E0C816D10409F062C07092C7
:10E310005D0E60925C0E10925F0E10925E0EF09297
:10E32000610EE092600E86E00F9458291092CA099F
:10E330001092C909882309F456C0682F70E0C501FE
:10E340000E94617090E080E02C960FB6F894DEBFDA
:10E350000FBECDBFDF91CF911F910F91FF90EF9036
:10E36000DF90CF90BF90AF909F908F907F906F90F5
:10E370005F904F903F9008950330110581F0043075
:10E38000110509F0BBCFFE24EF24FE24B7CFFE2CED
:10E39000EE24EE24EA94B2CFFF24FA94AFCFEF2814
:10E3A00021F492E0E92EF12CEECFEE24E394F12C4F
:10E3B000EACF70925D0E60925C0E90E080E0EE20FD
:10E3C00011F080E09FEF90935F0E80935E0E85E0EA
:10E3D000ABCF69E174E182ED9FE00E94AFF0109253
:10E3E000CA091092C90981E090E0AECFEF92FF9286
:10E3F0001F93CF93DF93192F7B01C82FD92FD7FFFE
:10E4000003C0D195C195D10961E08C2F0F9484236D
:10E4100082E0E816F10499F460E08C2F0F94562303
:10E420006BEB76E282ED9FE00E94AFF082ED9FE021
:10E43000DF91CF911F91FF90EF900C9443EF612FEC
:10E44000EF2851F46095661F6627661F8C2F0F9486
:10E45000562367EB76E2E6CF661F6627661F8C2F92
:10E460000F94562362EB76E2DDCFAF92BF92DF923C
:10E47000EF92FF920F931F93CF93DF93CDB7DEB749
:10E480002E970FB6F894DEBF0FBECDBF2091C30A02
:10E490003091C40A232B09F4B8C02091C20A21117B
:10E4A000B4C07C018091C20A8F5F8093C20A8091C0
:10E4B000C10A8F5F8093C10A0F94C9270091580A3F
:10E4C0001091590A20915A0A30915B0A601B710B16
:10E4D000820B930B6B3071058105910508F48BC09D
:10E4E00083E0E816F104A9F00F94C9270091540ABB
:10E4F0001091550A2091560A3091570A601B710BF2
:10E50000820B930BDD24D39464367105810591054C
:10E5100008F4D12CE091C30AF091C40A0681178156
:10E520000115110509F449C0F80180858F70863006
:10E5300009F03FC01987088770E060E0CE010896B7
:10E540000E94EAD6B701CE0108960E942ADADD20A1
:10E5500031F064E070E0CE0108960E942ADA60E2B1
:10E5600076E0C8010F94F712FC01892B11F1908518
:10E570009F7095509230E8F4A680B780A114B10442
:10E58000C1F0BA82A982B801CE0101960E94EAD6F2
:10E59000B701CE0101960E942ADADD2031F064E055
:10E5A00070E0CE0101960E942ADAF501A280B380C4
:10E5B000E5CFF80102811381B3CFF3E0EF16F10448
:10E5C00051F00F94C9276093580A7093590A8093A9
:10E5D0005A0A90935B0ADD2051F00F94C92760938B
:10E5E000540A7093550A8093560A9093570A1092D2
:10E5F0000E1010920F108091C10A81508093C10AB1
:10E600008091C20A81508093C20A2E960FB6F89468
:10E61000DEBF0FBECDBFDF91CF911F910F91FF9055
:10E62000EF90DF90BF90AF900895A89582E090E0C2
:10E630000C9435728091390C8F5F8093390CA895BA
:10E6400083E090E00E9435720E9440F88091390C7E
:10E6500081508093390C089560E976E285E29FE06D
:10E660000E94AFF06DE776E285E29FE00E94AFF096
:10E670006FE676E285E29FE00E94AFF067E676E221
:10E6800085E29FE00E94AFF085E29FE00E9443EFA9
:10E6900067E576E285E29FE00E94AFF06BE476E208
:10E6A00085E29FE00E94AFF063E276E285E29FE0C0
:10E6B0000E94AFF063E176E285E29FE00E94AFF056
:10E6C00066E076E285E29FE00E94AFF061EF75E2DE
:10E6D00085E29FE00E94AFF062EE75E285E29FE086
:10E6E0000E94AFF06AED75E285E29FE00E94AFF014
:10E6F00069EC75E285E29FE00E94AFF063EA75E2A3
:10E7000085E29FE00E94AFF066E975E285E29FE056
:10E710000E94AFF06CE875E285E29FE00E94AFF0E6
:10E720006DE775E285E29FE00E94AFF065E775E274
:10E7300085E29FE00E94AFF069E675E285E29FE026
:10E740000E94AFF06FE475E285E29FE00E94AFF0B7
:10E7500060E375E285E29FE00E94AFF06BE175E255
:10E7600085E29FE00E94AFF063E075E285E29FE002
:10E770000E94AFF065EF74E285E29FE00E94AFF087
:10E7800069EE74E285E29FE00E94AFF061EE74E210
:10E7900085E29FE00E94AFF066ED74E285E29FE0C3
:10E7A0000E94AFF069EC74E285E29FE00E94AFF056
:10E7B00061EC74E285E29FE00E94AFF066EB74E2E8
:10E7C00085E29FE00E94AFF067EA74E285E29FE095
:10E7D0000E94AFF06EE974E285E29FE00E94AFF024
:10E7E00060E974E285E29FE00E94AFF062E874E2C3
:10E7F00085E29FE00E94AFF066E774E285E29FE069
:10E800000E94AFF06EE674E285E29FE00E94AFF0F6
:10E810006BE574E285E29FE00E94AFF061E574E28F
:10E8200085E29FE00E94AFF085E29FE00C9443EF09
:10E830000F931F93CF93DF9300D000D0CDB7DEB7F7
:10E840000E942C736DE27CE185E29FE00E94AFF0B4
:10E85000CE0101960F944121CE0101960E94C33151
:10E8600009E115E01A83098380917F0D9091800D55
:10E87000A091810DB091820D8B839C83AD83BE836B
:10E88000CE0101960E94C3311A8309831B821C8228
:10E890001D821E8280E590E00F94102144E050E03C
:10E8A000BE016D5F7F4F81E090E00E942DFB0E94D2
:10E8B00024FCCE0101960E94C3311A8309831B8276
:10E8C0001C821D821E8280E590E00F94102144E09E
:10E8D00050E0BE016D5F7F4F85E090E00E942DFB10
:10E8E0000E9424FCCE0101960E94C33163E57CE1C5
:10E8F00085E29FE00E94AFF088EC90E026960FB68C
:10E90000F894DEBF0FBECDBFDF91CF911F910F9165
:10E910000895CF92DF92EF92FF921F93CF93DF93F0
:10E9200000D000D0CDB7DEB76BE078E185E29FE0A4
:10E930000E94AFF089E0E82E8FE0F82E10E090E121
:10E94000C92ED12CF70181917F01803130F468E428
:10E9500075E085E29FE00E9499F0153041F1F701E2
:10E960003197808190E0B0E0A0E089839A83AB8307
:10E97000BC83DE82CD82BE016F5F7F4F85E29FE068
:10E980000E94FECF69E078E10E94AFF01F5F163071
:10E99000C9F626960FB6F894DEBF0FBECDBFDF9145
:10E9A000CF911F91FF90EF90DF90CF9008958091CD
:10E9B0000E0F90E0B0E0A0E089839A83AB83BC8324
:10E9C000DE82CD82BE016F5F7F4F85E29FE00E94B5
:10E9D000FECF0E9443EFDACFEF92FF920F931F9387
:10E9E000CF93DF9300D000D01F92CDB7DEB77B016D
:10E9F000CE0107969F938F9301979F938F930197D3
:10EA00009F938F9301979F938F9301979F938F93DA
:10EA100001979F938F938E010F5F1F4F1F930F934B
:10EA20008FE997E09F938F93DB0113968C91139757
:10EA30008F9312968C918F930F94804C0FB6F8940D
:10EA4000DEBF0FBECDBF0697ECF46EED72E28DE235
:10EA50009FE00E94AFF0D70112966D917C918DE2FC
:10EA60009FE00E9499F080E991E027960FB6F89414
:10EA7000DEBF0FBECDBFDF91CF911F910F91FF90F1
:10EA8000EF9008958091010F9091020F892B09F466
:10EA900049C00F944A14882309F444C0A091010F7F
:10EAA000B091020F52961C921E92519754961C924E
:10EAB0001E92539784E890E01D969C938E931C972A
:10EAC0001E961C921E9782E755968C935597ED9152
:10EAD000FC9111970088F189E02D64E070E0CD0190
:10EAE00019958091010F9091020FDC01ED91FC913D
:10EAF0000280F381E02D46E050E0B801199586E0F0
:10EB0000F801A9E0BFE001900D928A95E1F78091AC
:10EB1000010F9091020FDC01ED91FC910488F589C1
:10EB2000E02D19950E94897460EF72E285E29FE002
:10EB30000E94AFF088EC90E098CFCF92DF92FF92E6
:10EB40000F931F93CF93DF93F12C6115710509F497
:10EB50008DC06A01EB018C01CB010E94BCAFF82E85
:10EB6000882309F483C0D6FE0EC0D8018C918B3067
:10EB700009F450C008F041C040E051E060E070E0AE
:10EB80008A3009F450C0D4FE09C0F801608186EFD4
:10EB9000860F843018F0CE010E942DB8D5FE66C0D5
:10EBA000D80114964D915D916D917C9117971196B6
:10EBB0008C918F70873030F08930C8F18A50823064
:10EBC00008F45DC0CE010E9469B0EE81FF813097EC
:10EBD00009F44CC080858F709EEF980F923010F032
:10EBE000811144C0D80111968C91982F9295907FF5
:10EBF00080858F70892B808739C08C3081F040E010
:10EC000056E060E070E08D3009F0BDCFCE010E948B
:10EC1000E1B1B9CF40E051E060E070E0F7CF40E013
:10EC200056E060E070E0CE010E94B8B1ACCFEE815A
:10EC3000FF813097D9F080858F709EEF980F9230CA
:10EC400010F0811113C04187528763877487EE816A
:10EC5000FF818085807F83608087EE81FF81808552
:10EC6000982F907F8F708067903629F28F2DDF91DB
:10EC7000CF911F910F91FF90DF90CF900895CE011B
:10EC80000E9469B0F3CFCF93DF9300D000D01F92E2
:10EC90001F92CDB7DEB7FC01628398E0DE011196CA
:10ECA00001900D929A95E1F729813A814B815C811F
:10ECB0006D817E818F81988528960FB6F894DEBF8E
:10ECC0000FBECDBFDF91CF910895CF93DF9300D0DA
:10ECD00000D01F921F92CDB7DEB7FC01608398E091
:10ECE000DE01119601900D929A95E1F729813A8102
:10ECF0004B815C816D817E818F81988528960FB6CE
:10ED0000F894DEBF0FBECDBFDF91CF910895CF93B2
:10ED1000DF9300D000D01F921F92CDB7DEB7FC0169
:10ED20009181907F9A609183448355836683778332
:10ED300088E0DE01119601900D928A95E1F7298114
:10ED40003A814B815C816D817E818F819885289687
:10ED50000FB6F894DEBF0FBECDBFDF91CF910895FF
:10ED6000AF92BF92CF92DF92EF92FF920F931F93D9
:10ED7000CF93DF9300D000D01F921F92CDB7DEB7A4
:10ED80006115710509F45FC05A016B017C01CB016B
:10ED90000E94BCAF082F882369F1D60116968D9189
:10EDA0009C91009709F443C0FC011085212F2F701E
:10EDB0003EEF320F323010F021112EC012951F702D
:10EDC000B4FE59C0C6010E944CB8F70180831123DC
:10EDD00081F18181807F182B1183D6011696ED91E8
:10EDE000FC9181859285A385B485F7018483958301
:10EDF000A683B783802F28960FB6F894DEBF0FBE88
:10EE0000CDBFDF91CF911F910F91FF90EF90DF90D9
:10EE1000CF90BF90AF900895253049F460E00F94F3
:10EE2000A913009721F0DC0118961C91C7CF10E0C0
:10EE3000C7CFD6011696ED91FC9180858F708230F8
:10EE400021F0833051F000E0D5CF418552856385B4
:10EE50007485C7010E948776CDCF41855285638531
:10EE60007485F7018181807F876081834483558326
:10EE700066837783BFCF1123E1F2F701AACFCF9347
:10EE8000DF9300D000D01F921F92CDB7DEB7FC01F8
:10EE90006F3F710519F014F06FEF70E077FD60E0DF
:10EEA0009181892F8F7081508230C8F4648388E00B
:10EEB000DE01119601900D928A95E1F729813A8140
:10EEC0004B815C816D817E818F81988528960FB6FC
:10EED000F894DEBF0FBECDBFDF91CF910895907F34
:10EEE00091609183E3CFCF92DF92EF92FF92DC01AA
:10EEF000362F1196EC911197EF70EC3008F0B6C0F8
:10EF0000F0E08827E957F8488F4F0D945E4739782D
:10EF1000BF77BF773678367836780478C677367814
:10EF200036789377937714968D919D910D90BC913F
:10EF3000A02D662399F0B7FD9FC08F3F9105A105D5
:10EF4000B10529F024F08FEF90E0A0E0B0E02FEFC2
:10EF500030E0A901481B590BCA010CC0B7FD89C09C
:10EF60008F3F9105A105B10529F024F08FEF90E0C6
:10EF7000A0E0B0E0FF90EF90DF90CF90089514965E
:10EF80002C91822F90E06623A9F3E1CF1496CD90C7
:10EF9000DD90ED90FC901797662301F120E030E0C2
:10EFA000A901C701B6010F949D4587FD65C020E00A
:10EFB00030E04FE753E4C701B6010F94A548181697
:10EFC0000CF457C0A701960160E070E08FE793E46E
:10EFD0000F9490470F946F48CB01CCCF20E030E0E6
:10EFE000A901C701B6010F949D4587FD42C020E0ED
:10EFF00030E04FE753E4C701B6010F94A548181657
:10F00000DCF1C701B601E6CF14966D917D918D912B
:10F010009C9117973323B1F06D395FEF7507850722
:10F02000950754F1611524E67207810591050CF5E9
:10F030002CE93FEF4FEF5FEF0F940947C901815073
:10F040009F4F98CF6D394FEF7407840794078CF06A
:10F05000611554E675078105910574F424E630E0E6
:10F0600040E050E00F940947C90184CF8FEF9FEF34
:10F0700081CF90E080E07ECF8FEF90E07BCFCF9389
:10F08000DF93EC01DB0189818F708630E1F128F498
:10F0900081508230C8F080E014C0873009F18A5076
:10F0A0008230C8F72FEF30E00F94754724E630E048
:10F0B00040E050E00F9409472C833D834E835F83EB
:10F0C00081E0DF91CF9108952FEF30E00F947547E5
:10F0D00024E630E040E050E00F9409472C83F0CF65
:10F0E0002FEF30E00F94754724E630E040E050E029
:10F0F0000F940947CA01B9010F94A4456C837D831D
:10F100008E839F83DDCF2CE933E60F94754724E689
:10F1100030E040E050E00F9409472C833D834E835C
:10F120005F83B9CFDC011196EC911197EF70E1503C
:10F13000EB3008F039C0F0E08827EE55F7488F4FE4
:10F140000D945E47C578C578D478AD78AD78B6783B
:10F15000CD78CD78CD78AD78AD7814966D917D91E0
:10F160008D919C9117970F94A445089514966D91D5
:10F170007D918D919C91179724E630E040E050E01E
:10F180000F940947CA01B901EECF14966C9170E053
:10F1900090E080E00F94A245089514966D917D91C2
:10F1A0008D919C911797089560E070E0CB010895D0
:10F1B000DC011196EC911197EF70E150EB3008F003
:10F1C00037C0F0E08827E851F7488F4F0D945E472D
:10F1D000FA78FA781879F378F37809790079007970
:10F1E0000079F378F37814966D917D918D919C91CF
:10F1F0001797089514966C9170E090E080E0089560
:10F2000014966D917D918D919C9117970F946F48F5
:10F21000089514966D917D918D919C91179724E698
:10F2200030E040E050E00F940947CA01B901089569
:10F2300060E070E0CB010895DC011196EC9111972C
:10F24000EF70E150EB3008F03EC0F0E08827E45D5D
:10F25000F6488F4F0D945E4742794279637937794A
:10F2600037795C794D794D794D79377937791496BD
:10F270002D913D914D915C911797A4E6B0E00F94CC
:10F280002847089514966C9184E6689FB001112474
:10F29000072E000C880B990B089520E030E048EC15
:10F2A00052E414966D917D918D919C9117970F94D6
:10F2B00003460F946F48089514966D917D918D913A
:10F2C0009C911797089560E070E0CB010895FC01D0
:10F2D000A7812A2F2E7FC9F081818F7081508330C2
:10F2E000A0F4A695A150BB0B2BE531E00F94754718
:10F2F00024E630E040E050E00F940947DA01C9010C
:10F3000087569F4FAF4FBF4F08958FEF9FEF0895E0
:10F310002F923F924F925F926F927F928F929F9225
:10F32000AF92BF92CF92DF92EF92FF920F93CF9363
:10F33000DF9300D01F92CDB7DEB77C017A8369835B
:10F340005C834B83DB011C92FC0160818FEF860F95
:10F35000883108F04BC034FF49C0FAE06F9FB0011C
:10F3600011246E5D794ECD010F940440D7011196A2
:10F370008C918F7041F04B815C8164E875E08981EC
:10F380009A810F94DB4BE981FA8101900020E9F723
:10F39000319729813A81E21BF30B19012E0E3F1E92
:10F3A0004B815C814E1B5F0B415051095C834B8349
:10F3B000D7011196EC911197EF7009F4F5C0E15067
:10F3C000EC3008F0F1C0F0E08827E651F6488F4FA6
:10F3D0000D945E47F9799C7A097B687B837B477A39
:10F3E000197B197B197B357A1D7A9F7B29803A809E
:10F3F000DFCFF7018481282F30E050E040E0002388
:10F4000059F030E0A4E6B0E00F943B472FEF30E036
:10F4100040E050E00F9409475F934F933F932F9341
:10F4200083EB97E09F938F93FC81FF932B812F9326
:10F430003F922F920F94134CB2C017968C9117974E
:10F440008F9316968C9116978F9315968C9115978E
:10F450008F9314968C918F9386EB97E09F938F9365
:10F46000BC81BF93EB81EF93E3CF17968C911797F5
:10F470008F9316968C9116978F9315968C9115975E
:10F480008F9314968C918F938AEB97E0E7CF149625
:10F49000CD90DD90ED90FC901797F7FE34C084E698
:10F4A000882E912CA12CB12CC701B601A501940185
:10F4B0000F9409479B01AC0188279927DC01821B27
:10F4C000930BA40BB50BBF93AF939F938F936627BA
:10F4D0007727CB016C197D098E099F09A50194013D
:10F4E0000F9409475F934F933F932F938EEB97E0D1
:10F4F0009F938F933C813F934B814F933F922F92E9
:10F500000F94134C4CC0C701B60124E630E040E034
:10F5100050E00F9409479F938F937F936F935F936E
:10F520004F933F932F938FEB97E09F938F939C8103
:10F530009F93AB81AF93E2CFC7010E946779BC0173
:10F54000D7011696CC9016971796DC901797D0FA9D
:10F55000DD24D0F814969C9114971596FC90EB80BE
:10F56000BC80292F30E050E040E077FD35C001112C
:10F5700035C07F936F931F921F921F929F931F928C
:10F58000FF92DF92CF9288EC97E09F938F93FC815C
:10F59000FF932B812F933F922F920F94134C0FB612
:10F5A000F894DEBF0FBECDBF89819A810F900F9076
:10F5B0000F900F90DF91CF910F91FF90EF90DF9020
:10F5C000CF90BF90AF909F908F907F906F905F9003
:10F5D0004F903F902F900895002361F0292F30E045
:10F5E000A4E6B0E00F943B472FEF30E040E050E05E
:10F5F0000F9409475F934F933F932F931F92FF926E
:10F60000DF92CF928BEC97E09F938F93BF92EF9214
:10F6100075CF15968C9115971F928F9316969C9186
:10F62000169717968C9181708F939F938EEC97E02D
:10F6300015CF14968D909D90AD90BC90179720E0BB
:10F6400030E0A901C501B4010F949D4524013501A5
:10F6500087FF04C077FA709477F87094C301B20101
:10F660000F946F486B01072E000C880B990B0F94B9
:10F67000A4459B01AC01C301B2010F94904720E067
:10F6800030E04AE754E40F9403460F94FA480F948D
:10F690006F48062F772E20E030E0A901C501B401A4
:10F6A0000F949D4587FF07C07F920F93DF92CF9203
:10F6B00084ED97E0D3CE7F920F93DF92CF9285EDCA
:10F6C00097E09F938F933C813F934B814F93B0CEB4
:10F6D00014968C9114971F928F9315968C91159771
:10F6E0001F928F9316968C911F928F938BEC97E0BD
:10F6F0009F938F93BC81BF93EB81EF933F922F92A7
:10F700000F94134C4CCF17968C9117971F928F9391
:10F7100014968C9114971F928F9315968C91159730
:10F720001F928F9316968C911F928F9388EC97E07F
:10F730009F938F93BC81BF93EB81EF93DFCE1496A1
:10F740006D917C914B815C81C1010F94F94B2CCF61
:10F75000EF92FF920F93CF93DF93CDB7DEB7A097D1
:10F760000FB6F894DEBF0FBECDBF7C0100E020E0F5
:10F7700030E340E250E0BE016F5F7F4F0E94887926
:10F78000BE016F5F7F4F82ED9FE00E9499F063E2C0
:10F7900077E182ED9FE00E94AFF0F70161816F7029
:10F7A0004AE050E082ED9FE00E9466EF6CE177E175
:10F7B00082ED9FE00E94AFF04AE050E0F7016281E5
:10F7C00082ED9FE00E9466EF82ED9FE00E9443EF92
:10F7D000A0960FB6F894DEBF0FBECDBFDF91CF91DC
:10F7E0000F91FF90EF900895CF93DF93EC01611597
:10F7F000710539F48F8181708F8381E0DF91CF9122
:10F8000008958981982F9F7029F180E09430B0F796
:10F810009B01770F440B550B2959310941095109B7
:10F82000A4E6B0E00F9428472BE531E040E050E03B
:10F830000F94094737FF02C030E020E0253631053C
:10F8400014F024E630E02F5F220F8F818170282B87
:10F850002F83D3CF807F82608983DACFFC019181AF
:10F86000892F8F7021F0823029F080E00895907FF9
:10F87000926091839B0177FF02C030E020E02E363A
:10F8800081E0380714F02DE631E02683878130FBD4
:10F8900080F9878381E00895EF92FF920F931F9381
:10F8A000CF93DF93FC01892B69F19081992351F16A
:10F8B0009D3291F180ED890F8A3070F1C8E0D0E07F
:10F8C000953211F1CEEFDFEF9B37F1F0C7E1D0E0D9
:10F8D0009332D1F08F018CE2E82E86E1F82EC1E060
:10F8E000D0E0C7010F94DD3FAC01B701C8010F9410
:10F8F000F63F892B49F021968AE0E80EF11CC931C8
:10F90000D10579F7CFEFDFEFCE01DF91CF911F91D6
:10F910000F91FF90EF900895D0E0C0E0F5CFEF9207
:10F92000FF920F931F93CF93DF93EC01892B51F13B
:10F9300088858F70843009F5E984FA84C7010E94B4
:10F940004C7C8C0118161906ECF4C7010E9494F83F
:10F95000C801012E000CAA0BBB0B89879A87AB87C5
:10F96000BC878885807F82608887C801DF91CF91BE
:10F970001F910F91FF90EF900895823019F409853F
:10F980001A85F3CF10E000E0F0CF2F923F924F9214
:10F990005F926F927F928F929F92AF92BF92CF921F
:10F9A000DF92EF92FF920F931F93CF93DF93CDB728
:10F9B000DEB7A4970FB6F894DEBF0FBECDBF7C01B3
:10F9C0006B0161EA75E0C6010F94F712FC01892B07
:10F9D00009F422C180858F70843009F455C08530C8
:10F9E00009F01AC1068117810115110509F414C126
:10F9F000D80118968C9118978F70823019F412964E
:10FA00000D911C910115110509F406C1F8018085BD
:10FA10008F70853011F0D801F2CFC8010F943A14DD
:10FA20008230C9F760E0C8010F94A9135C010E94FD
:10FA30008F7C61E0C8010F94A9134C01FC01808503
:10FA40008F70823041F7C7010E94D878D40119968F
:10FA50004D905D906D907C901C97641575058605A2
:10FA60009705C9F6A114B10409F4D6C019861A86FF
:10FA70001B861C861D861E861F86188A8A85807FA7
:10FA80008A87F50161854DC066EA75E081859285BA
:10FA90000F94CB4B892B09F0BFC0C7010E94D878C7
:10FAA000611571058105910509F49CC0660F771FEA
:10FAB000881F991F2FEF30E040E050E00F94094776
:10FAC00057FD16C023303105410551050CF070C0BB
:10FAD000DA01C9010196A11DB11D82309105A10570
:10FAE000B10509F44BC00397A105B10509F460C045
:10FAF000198A1A8A1B8A1C8A1D8A1E8A1F8A188ED6
:10FB00008A89807F8A8B67E0CE0141960E94437686
:10FB100029873A874B875C876D877E878F87988B8D
:10FB200062E1CE0109960E94657629833A834B8370
:10FB30005C836D837E838F83988729813A814B8193
:10FB40005C816D817E818F819885A4960FB6F89433
:10FB5000DEBF0FBECDBFDF91CF911F910F91FF9000
:10FB6000EF90DF90CF90BF90AF909F908F907F905D
:10FB70006F905F904F903F902F900895198A1A8A46
:10FB80001B8A1C8A1D8A1E8A1F8A188E8A89807F7A
:10FB90008A8B67E0CE0141960E94437629873A8797
:10FBA0004B875C876D877E878F87988B61E1B9CFA4
:10FBB000198A1A8A1B8A1C8A1D8A1E8A1F8A188E15
:10FBC0008A89807F8A8B67E0CE0141960E944376C6
:10FBD00029873A874B875C876D877E878F87988BCD
:10FBE00060E19FCF198A1A8A1B8A1C8A1D8A1E8A85
:10FBF0001F8A188E8A89807F8A8B67E0CE014196A2
:10FC00000E94437629873A874B875C876D877E877A
:10FC10008F87988B62E085CF6FEB75E0C6010F94FC
:10FC2000F7128C01009709F41CC1DC0118968C9125
:10FC30008F70853009F0FEC0C8010F943A148430EB
:10FC400008F40FC160E0C8010F94A9135C0161E0E2
:10FC5000C8010F94A9133C0162E0C8010F94A913D5
:10FC6000DC0119962D913D914D915C911C97298F46
:10FC70003A8F4B8F5C8F63E0C8010F94A9134C013E
:10FC800065E0C8010F94A9136C0167E0C8010F94E7
:10FC9000A9138C01C7010E94D878298D3A8D4B8D0C
:10FCA0005C8D621773078407950714F5C114D1049E
:10FCB00009F4C2C0D60118968C9118978F708230C3
:10FCC00009F0BAC019861A861B861C861D861E86F8
:10FCD0001F86188A8A85807F8A8719964D915D9143
:10FCE0006D917C911C97CE0109960E9487761DCF5D
:10FCF000D40119962D913D914D915C911C972D8FBA
:10FD00003E8F4F8F58A32617370748075907D4F45B
:10FD10000115110509F490C0F80180858F708230BB
:10FD200009F08AC019861A861B861C861D861E86C7
:10FD30001F86188A8A85807F8A87418552856385D8
:10FD40007485D1CFD5011996CD90DC90F301218433
:10FD5000328419861A861B861C861D861E861F867F
:10FD6000188A8A85807F8A872101032C000C660807
:10FD7000770846010D2C000CAA08BB08098D1A8DC6
:10FD8000012E000C220B330B09A31AA32BA33CA3B7
:10FD9000C7010E94D8789B01AC01E9A0FAA00BA191
:10FDA0001CA12E193F09400B510BC301B201681968
:10FDB00079098A099B090F94D7460D8D1E8D9801EC
:10FDC000110F440B550BE9A0FAA00BA11CA12E1991
:10FDD0003F09400B510B0F940947820E931EA41E3E
:10FDE000B51EC1018C199D096D8D7E8D098D1A8DF1
:10FDF000601B710B0F944A4777FF02C06F5F7F4F04
:10FE000075956795CB01770FAA0BBB0B880D991DD4
:10FE1000AA1DBB1D40E050E0BA01B7FD64CFB3019D
:10FE2000A20184179507A607B7070CF05CCFAC01B9
:10FE3000BD0159CF811115C019861A861B861C86F3
:10FE40008A85807F8A871D861E861F86188A88E09D
:10FE5000FE013996DE01119601900D928A95E1F727
:10FE60006CCE88E0F701F6CF2F923F924F925F92CF
:10FE70006F927F928F929F92AF92BF92CF92DF92BA
:10FE8000EF92FF920F931F93CF93DF93CDB7DEB71F
:10FE900065970FB6F894DEBF0FBECDBF6115710533
:10FEA00049F528E0FC01DE01119601900D922A959A
:10FEB000E1F729813A814B815C816D817E818F815F
:10FEC000988565960FB6F894DEBF0FBECDBFDF9163
:10FED000CF911F910F91FF90EF90DF90CF90BF9047
:10FEE000AF909F908F907F906F905F904F903F90DA
:10FEF0002F9008953B018C0161EA75E0C3010F94D6
:10FF0000F7126C01D801FC90FF2009F45AC0009749
:10FF100009F457C0FC0180858F70843009F4DEC07D
:10FF2000853009F04EC080913102893020F48091F3
:10FF30003002893050F06DED77E082ED9FE00E9455
:10FF400099F082ED9FE00E9443EFD6011696ED9066
:10FF5000FC90E114F104A9F1F70180858F7057013D
:10FF6000823069F0B12CA12CE114F10409F436C1FE
:10FF7000D70118968C918F70853021F0F701E280BF
:10FF8000F380F2CFC7010F943A148230B9F760E0E2
:10FF9000C7010F94A9130E948F7C4C0161E0C70137
:10FFA0000F94A9136C01D8018C918815190431F7AD
:10FFB000F60180858F70823009F7C114D10409F0F1
:10FFC00017C16FEB75E0C3010F94F7127C01D801E4
:10FFD00011968C918F7009F43BC1E114F10409F47E
:10FFE0003BC1F70180858F70853009F0D0C1C70112
:10FFF0000F943A14843008F4CAC164E0C7010F9426
:020000021000EC
:10000000A9136C0166E0C7010F94A9131C01C80174
:100010000E94D8784B015C0160E0C7010F94A913DE
:10002000DC0119964D905D906D907C901C97B0917D
:100030003102B98B84149504A604B7040CF016C1E0
:10004000B93020F480913002893050F162E076E1DD
:1000500082ED9FE00E94AFF0C8010E94D878AB010A
:10006000BC012AE030E082ED9FE00E9408F06CEED7
:1000700075E182ED9FE00E94AFF060E0C7010F9450
:10008000A913FC0141855285638574852AE030E01F
:1000900082ED9FE00E9408F082ED9FE00E9443EF16
:1000A000C114D10409F479C1D60118968C9118971E
:1000B0008F70823009F071C119821A821B821C82F2
:1000C0001D821E821F8218868A81807F8A831996EC
:1000D0004D915D916D917C911C9743C066EA75E0EE
:1000E000818592850F94CB4B892B09F06ACFB0E1C3
:1000F000FB1609F463C0BF1580F0E2E0FE1619F1AB
:10010000D8014D915D916D917C91139714968D91CD
:100110009D910D90BC91A02D38C0F1E1FF16F1F139
:1001200022E1F212EDCF19821A821B821C821D82FB
:100130001E821F8218868A81807F8A8344E150E074
:1001400060E070E00EC019821A821B821C821D8240
:100150001E821F8218868A81807F8A8340E050E059
:10016000BA01CE0101960E94877629873A874B878C
:100170005C876D877E878F87988B49855A856B85CD
:100180007C858D859E85AF85B88949835A836B832D
:100190007C838D839E83AF83B8878BCE19821A822E
:1001A0001B821C821D821E821F8218868A81807F8C
:1001B0008A8340E850E060E070E0D3CF19821A8271
:1001C0001B821C821D821E821F8218868A81807F6C
:1001D0008A834FEF50E060E070E0C3CFA114B10418
:1001E00009F4EFCEF50180858F7009F4EACE650140
:1001F00080913102893020F4809130028930B8F04A
:100200006EE076E182ED9FE00E94AFF0D601199694
:100210004D915D916D917C911C972AE030E082EDCB
:100220009FE00E9408F082ED9FE00E9443EF198258
:100230001A821B821C821D821E821F8218868A815E
:10024000807F8A83F601418552856385748589CFD5
:10025000E114F10409F09BC0F801408151816281F1
:10026000738184819581A681B7818FCF61E0C701B9
:100270000F94A913DC0119962D913D914D915C913C
:100280001C972A8B3B8B4C8B5D8B281539054A05B7
:100290005B053CF5B989B93020F480913002893092
:1002A00050F06EEC75E182ED9FE00E94AFF082EDC0
:1002B0009FE00E9443EF2114310409F46EC0F10164
:1002C00080858F70823009F068C019821A821B8283
:1002D0001C821D821E821F8218868A81807F8A83EB
:1002E000B2CF63E0C7010F94A9138C0162E0C7018C
:1002F0000F94A913DC011996CD90DD90ED90FC9040
:100300001C97F80121853285438554852C193D09B8
:100310004E095F09C501B401641975098609970979
:100320000F94D7462A893B894C895D892419350960
:10033000460957090F940947C20ED31EE41EF51E45
:10034000F989F93020F480913002893090F069EB1E
:1003500075E182ED9FE00E94AFF02AE030E0B70146
:10036000A60182ED9FE00E9408F082ED9FE00E94CE
:1003700043EF19821A821B821C821D821E821F82F9
:1003800018868A81807F8A83B701A601EACED701C9
:1003900018968C918F7009F05FCF19821A821B8298
:1003A0001C828A81807F8A8349815A816B817C810A
:1003B00080E090E0DC01E9CE8F929F92AF92BF92F5
:1003C000CF92DF92FF920F931F93CF93DF93EC01B5
:1003D0008A819B810F943A14082F10E00430110594
:1003E00054F40F940A19BC018A819B810F94171948
:1003F0000F5F1F4FF3CFEA81FB8106811781011543
:10040000110531F0D80112968D919C919D838C83BA
:10041000EC81FD81309721F0828193819F838E83CF
:10042000EE81FF81309749F00280F381E02D309713
:1004300021F082819381998788870115110541F008
:10044000F80180858F70843059F128F4823071F082
:10045000FF24FA940CC0853001F18630C9F767E6B5
:1004600075E0C8010F94F7128C01E7CFF184FA868A
:10047000CE010E94BCAF811138C010E000E01C87A3
:100480000B87DF91CF911F910F91FF90DF90CF905D
:10049000BF90AF909F908F90089506811781CDCF28
:1004A000C184D284C114D10499F2F60180818823D9
:1004B00079F293E5892E94E1992EB12CA12CFA2C96
:1004C000C4010F94DD3FAC01B401C6010F94F63FA7
:1004D000892BB9F1FFEFAF1ABF0A89E0880E911C92
:1004E000A7E1AA16B10459F7B3CFCE010F941F1894
:1004F0008C010097B1F0FC0182819381892B39F046
:100500008F2D0F9435198C01892B09F4B6CFD801A2
:10051000ED91FC910684F785E02DBE01C801199587
:10052000AECF8F2D0F9435198C01892B09F4A5CFEF
:10053000EA85F0E0EE0FFF1FE052F04F11830083D9
:10054000E6CFC6010E9494F88A2D90E0B0E0A0E0CA
:10055000F80181879287A387B4878085807F826036
:10056000808785CF8F929F92AF92BF92CF92DF927A
:10057000EF92FF920F931F93CF93DF93CDB7DEB728
:1005800060970FB6F894DEBF0FBECDBF8C017B0124
:1005900040E050E860E070E00E940AB2672B682BF0
:1005A000692B09F0B5C062E070E0C8010E94D9B0C3
:1005B0006C0119861A861B861C861D861E861F8660
:1005C000188A8A85807F8A87D7FCA2C040E050E2E3
:1005D000B801CE0109960E94B07663E070E0C801D0
:1005E0000E94D9B0AC011816190614F04FE350E080
:1005F00081E0C816D10429F4EF2CFF0CFF08FF247A
:1006000004C082E0C816D104D4F32FEF30E0D70144
:100610000F9475479A01550F440B550B0F940947DA
:1006200049016901C8010E944CB8E82EF12C60E034
:10063000CE0109960E94737788169906F9F4CD28A1
:1006400041F082E0E816F10419F185E0E816F104C2
:10065000F9F081E090E060960FB6F894DEBF0FBE2F
:10066000CDBFDF91CF911F910F91FF90EF90DF9061
:10067000CF90BF90AF909F908F900895CD2899F123
:1006800086E0E816F10441F081E0E816F10421F07B
:1006900061E0C8010E942DB8B401CE0109960E9404
:1006A0003F7740E050E2B801CE0109960E949D7567
:1006B00082E0E816F10421F085E0E816F10449F43F
:1006C00030E020E040E050E160E070E0C8010E94CE
:1006D00091B530E020E040E050E260E070E0C80119
:1006E0000E9491B5B6CF85E0E816F10409F4B1CFC8
:1006F00082E0E816F10409F4ACCF62E0C8010E9480
:100700002DB830E020E040E050E160E070E0E7CF5D
:1007100090E080E0A0CFCF92DF92EF92FF920F9314
:100720001F93CF93DF9300D000D01F921F92CDB7BD
:10073000DEB77C0109831A832B833C834D835E8360
:100740006F837887CE0101960F94B8138C0189814D
:10075000882351F09B81923008F0BAC0823011F0AA
:10076000853011F410E000E070E060E0C7010E9405
:10077000D9B0D82EC92E6CEF73E182ED9FE00E94B4
:10078000AFF04AE050E06D2D7C2D82ED9FE00E949D
:1007900050F06AEF73E182ED9FE00E94AFF04AE013
:1007A00050E0B80182ED9FE00E9450F082ED9FE0A2
:1007B0000E9443EF8091C9099091CA09892BE9F001
:1007C00040E050E3B701CE0101960E949D7570E0B4
:1007D00060E0C7010E94617090E080E028960FB64B
:1007E000F894DEBF0FBECDBFDF91CF911F910F9167
:1007F000FF90EF90DF90CF90089581E090E090938C
:10080000CA098093C90926E040E855E260E070E03B
:100810008DE39CE00E94FCF1D092D40D8DE39CE02E
:100820009093D30D8093D20D1092E20E1092E40EAD
:100830001092E30E80ED97E090935D0E80935C0E36
:1008400010925F0E10925E0E01151105E1F185E028
:1008500090E09093610E8093600E86E00F9458298B
:10086000D82E64E670E080E090E00F94C925D110A6
:100870000AC063EF73E182ED9FE00E94AFF082ED6A
:100880009FE00E9443EF82ED97E090935D0E80938E
:100890005C0E10925F0E10925E0E24E6209FC00147
:1008A000219F900D11249093610E8093600E86E03D
:1008B0000F9458291092CA091092C909882359F037
:1008C000682F70E086CF1092610E1092600EC5CF37
:1008D0008FEF9FEF83CF81E090E080CF2F923F9208
:1008E0004F925F926F927F928F929F92AF92BF9240
:1008F000CF92DF92EF92FF920F931F93CF93DF93EC
:10090000CDB7DEB72C970FB6F894DEBF0FBECDBFC4
:100910005C0109831A832B833C834D835E836F8341
:100920007887CE0101960F94B8131C01023011F0A4
:10093000053011F4312C212CF50104811581F801C9
:1009400080858F70853009F07FC0C8010F943A14FC
:10095000E82EF12CF2E0EF16F1040CF475C060E023
:10096000C8010F94A913FC01818592859C878B8710
:1009700061E0C8010F94A913FC014184528463848F
:10098000748488248A94982CF2E0EF16F10459F0CC
:1009900062E0C8010F94A913FC0181849284F3E002
:1009A000EF16F104A1F48FE390E09A87898792E033
:1009B000C92ED12C29853A85D1010F946D4724E6A3
:1009C00030E040E050E00F94094779011CC063E03B
:1009D000C8010F94A913FC01818592859A878987A4
:1009E00082E0C82ED12CF4E0EF16F10439F064E077
:1009F000C8010F94A913FC01C184D28489859A850A
:100A00007101892BB9F684019601A2016B857C8561
:100A1000C5010E94E9702C960FB6F894DEBF0FBE98
:100A2000CDBFDF91CF911F910F91FF90EF90DF909D
:100A3000CF90BF90AF909F908F907F906F905F907E
:100A40004F903F902F90089590E080E0E4CFFF9288
:100A50000F931F93CF93DF9300D000D0CDB7DEB7B5
:100A60008C01BC01CE0101960E94D0ECBE016F5FEB
:100A70007F4F82ED9FE00E94A1F082ED9FE00E94F7
:100A800043EFCE0101960E94C8EC1A8219821C82A3
:100A90001B821E821D8264E273E2CE0101960E94D7
:100AA0006BECF801248135818D819E81F12C281712
:100AB000390738F0BE016F5F7F4FC8010F943522B0
:100AC000F82ECE0101960E94C8ECFF2069F0B80113
:100AD000CE0101960E94D0ECCE0101960F94B93060
:100AE000CE0101960E94C8EC26960FB6F894DEBFA0
:100AF0000FBECDBFDF91CF911F910F91FF90089551
:100B00000F931F93CF93DF9300D000D0CDB7DEB704
:100B1000A091010FB091020F109709F478C052967E
:100B20001C921E92519754961C921E92539784E8E1
:100B300090E01D969C938E931C971E961C921E9778
:100B400087E755968C935597ED91FC911197008806
:100B5000F189E02D70E060E0CD01199510E000E032
:100B60008091010F9091020FDC01ED91FC911197A2
:100B70001C962D913C910217130740F40190F081CF
:100B8000E02D60E019950F5F1F4FEACF0088F189D3
:100B9000E02D70E060E0199500E914E08091010F0C
:100BA0009091020FF80161918F01DC01ED91FC91B0
:100BB0000190F081E02D1995B4E004391B0771F71D
:100BC0008091010F9091020FDC01ED91FC9104885E
:100BD000F589E02D19956CE379E0CE0101960E942C
:100BE000D9ECCE0101960F94B930CE0101960E9446
:100BF000C8EC87E090E00F94F61787E090E00F9440
:100C0000001869EF72E285E29FE00E94AFF0109257
:100C1000210F1092200F80E090E190931C0F8093A1
:100C20001B0F84E890E09093230F8093220F81E0C4
:100C300080931D0F82E78093240F8FE09FE00E9436
:100C4000A6AB8FE09FE00E940CAC88EC90E026966B
:100C50000FB6F894DEBF0FBECDBFDF91CF911F91CD
:100C60000F9108956F927F928F929F92AF92BF9251
:100C7000CF92DF92EF92FF920F931F93CF93DF9368
:100C8000CDB7DEB7AE970FB6F894DEBF0FBECDBFBF
:100C90008091DB099091DC09892B09F473C680915E
:100CA000C10A81116FC68091C10A8F5F8093C10A0A
:100CB00063ED70E285E29FE00E94AFF085E29FE085
:100CC0000E9443EF0091DB091091DC096BEE77E0A5
:100CD000C8010F94F7129093C60A8093C50A61EF7A
:100CE00077E0C8010F94F7129093CE098093CD0955
:100CF00067E379E0C8010F94F7129093C40A8093D8
:100D0000C30A68EF77E0C8010F94F7129093520A74
:100D10008093510A009749F1DC011696ED91FC9100
:100D2000309719F120852F702530F9F46FEB70E2C0
:100D300085E29FE00E94AFF08091510A9091520AA3
:100D40000F943A148093500A4AE050E0682F85E2ED
:100D50009FE00E9466EF85E29FE00E9443EFE091F2
:100D6000510AF091520A8681978190934F0A80939D
:100D70004E0A6DEF77E08091DB099091DC090F94CA
:100D8000F7129093DA098093D909009709F4B2C059
:100D90000F943A14082F10E00115110509F4AAC0A8
:100DA000000F111F000F111F8091D7099091D809D2
:100DB000892B09F08EC07801013811051CF040E83C
:100DC000E42EF12CC7010F94913C9093D8098093A5
:100DD000D709E092D6091092B60A1092B50A10927D
:100DE0004D0A10924C0A1092B40A1092B80A10924E
:100DF000B70AC70101960F94913C9093BA0A809369
:100E0000B90A9093B30A8093B20A8E0D9F1D9093F6
:100E1000AD0A8093AC0A0F94C9276093AE0A709311
:100E2000AF0A8093B00A9093B10A90E080E0E0911D
:100E3000B90AF091BA0AE80FF91F10820196E81674
:100E4000F906ACF782E090E09093B60A8093B50A79
:100E500080914C0A90914D0A009741F061E00F9407
:100E6000842360E080914C0A0F94562380E980939C
:100E7000C9001092C8001092CD0083E08093CC008E
:100E80008EE08093CA00F0922F02E0922E02209111
:100E9000B90A3091BA0A80912E0290912F02820FE6
:100EA000931F9093AD0A8093AC0A232B09F45FC083
:100EB0006FE470E282ED9FE00E94AFF0B70182ED37
:100EC0009FE00F940B188DEA9EEA9093AB0A8093F3
:100ED000AA0A65EA70E285E29FE00E94AFF04AE06C
:100EE00050E0B80185E29FE00E9450F085E29FE06B
:100EF0000E9443EF63E078E08091DB099091DC0988
:100F00000F94F7128C01009709F471C00F943A14F2
:100F1000882309F46CC06FEF680FC8010F94A91300
:100F2000FC01E184F2849091A80A992359F0809100
:100F300070008E7F809370001092A80A10922A028F
:100F40001092290282E18093280291110F94530993
:100F5000C7010F947B0901E010E0E016F10674F080
:100F600060E0C8010F94AF090F5F1F4FF6CF68E331
:100F700070E282ED9FE00E94D3F0A5CF6AE270E2BA
:100F800082ED9FE00E94AFF00E94B032AB01BC0145
:100F90002AE030E082ED9FE00E945EEF82ED9FE06C
:100FA0000E9443EF69E870E285E29FE00E94AFF0A3
:100FB0004AE050E0B70185E29FE00E9450F085E2F0
:100FC0009FE00E9443EF63E870E282ED9FE00E94A1
:100FD000AFF00E94B032AB01BC012AE030E082EDFC
:100FE0009FE00E945EEF82ED9FE00E9443EF009140
:100FF000DB091091DC0967E078E0C8010F94F71273
:101000009093C8098093C7096EE078E0C8010F94F7
:10101000F7129093C80A8093C70A892B09F448C035
:101020008091C90A811144C08091BD0A9091BE0A85
:10103000892B09F0DFC164E070E282ED9FE00E943D
:10104000AFF082ED9FE00E9443EF8FE090E00F94BD
:10105000913C8C0188E1D80111968C9311971296DE
:101060001C9212971C921E961C921E921D970F9412
:101070009B1F1093BE0A0093BD0A012B09F08CC080
:1010800065EF7FE18DE29FE00E94AFF08DE29FE08F
:101090000E9443EF80E081708093C90A8091C90A61
:1010A000882331F063E770E285E29FE00E94AFF0B1
:1010B0001092C00A1092BF0AE091C50AF091C60AC8
:1010C000309709F4CCC2C680D7800091C50A109130
:1010D000C60A0115110509F4BBC2C114D10409F4F3
:1010E000B7C2F60180858F70853099F7C6010F94DD
:1010F0003A14823070F3A801B601CE0101960E9425
:1011000068B9CE0101960E94BCAF8823E1F18C85BD
:101110009D85009709F40DC2DC01ED91FC910284DC
:10112000F385E02D1995892B49F08C859D85DC018F
:10113000ED91FC910084F185E02D19958C859D85BC
:10114000DC01ED91FC910680F781E02D1995892B4A
:10115000D1F0CE0101960E944CB8882341F040E0C6
:1011600050E160E070E0CE0101960E94E1B18F8114
:101170009885892B41F040E050E260E070E0CE01BC
:1011800001960E94E1B1D6011296CD90DC90CE017D
:1011900001960E9435B999CF0F949B1F8091BD0A8B
:1011A0009091BE0A0F94DD0985E89DE00F94820BB3
:1011B000811189C066ED7FE185E29FE00E94D3F056
:1011C0008091BD0A9091BE0A0F94210DE091BD0A55
:1011D000F091BE0A81E080838091BD0A9091BE0AA1
:1011E0000F942F0D62EC7FE1811102C06DEA7FE167
:1011F00082ED9FE00E94D3F08091C70A9091C80AC7
:10120000892B09F447CF8091BB0A9091BC0A892BA6
:1012100009F0E2C083E190E00F94913C8C01809151
:10122000BD0A9091BE0A22E337EEF801328B218B82
:10123000968385831482108289E0818381E0828392
:1012400083831093BC0A0093BB0A0F94C9276B01D8
:101250007C01F0E1CF0EF7E2DF1EE11CF11CD801AA
:101260001596ED91FC9116978FEF83871486138264
:1012700014821582168217821086118612861496A1
:101280001C92BB24B394BE01605E7F4FF801858140
:1012900096810F94090E18160CF099C00F94C92767
:1012A0006C157D058E059F0508F091C0DE019096B6
:1012B00098E080E0915039F1ED91E827F0E0EB58AB
:1012C000FF4C8491F7CF0F94490F8091BD0A909104
:1012D000BE0A0F94DD0985E89DE00F94820B811111
:1012E0000BC060E97FE185E29FE00E94AFF085E2FC
:1012F0009FE00E9443EF80CF64E77FE18DE29FE0B3
:101300000E94D3F0C7CE9FA19813BDCFD8018C9176
:10131000811138C015968D919C910F942F0DBE01AF
:10132000605E7F4FF801858196810F94020D40E049
:1013300064EBD80115968D919C910F94DC0CF8010B
:1013400085809680C4010F94600CC4010F94DD0960
:1013500067E885E89DE00E949AEA60E885E89DE0FC
:101360000E949AEA0F940720C4010F94600CA82EE3
:10137000D80115968D919C910F942F0DA5FC02C05C
:10138000F801B082AE014F5F5F4FBE01605E7F4FDC
:10139000C8010F94700DD8011196AC9088A18031CE
:1013A00009F4F2C2BE01605E7F4FC8010F94DF0DE9
:1013B0008A1510F5F8018181D80111968C93119747
:1013C00014968C9114978F5F14968C935CCFE09158
:1013D000BB0AF091BC0A1282E091C70AF091C80AD8
:1013E000E680F7803FE7D32E8091C70A9091C80A24
:1013F000892B71F481E04FCE88A1803111F48CE00B
:10140000DBCFBE01605E7F4FC8010F94DF0DD4CFEC
:10141000E114F10479F3BE01605E7F4FF701808132
:1014200091810E944534882329F36DE57FE182EDA7
:101430009FE00E94AFF0D7016D917C9182ED9FE01B
:101440000E9499F082ED9FE00E9443EF0091BB0A59
:101450001091BC0AAE014F5F5F4FBE01605E7F4FCF
:10146000C8010F94C50D882309F45EC088A180319E
:1014700009F45AC0DD82F801858196810F942F0D01
:10148000BE01605E7F4FD80115968D919C910F949F
:10149000020D40E06EE4F801858196810F94DC0C2A
:1014A00040E06B81D80115968D919C910F94DC0CD6
:1014B00040E06C81F801858196810F94DC0C88A155
:1014C000803141F040E06D81D80115968D919C915D
:1014D0000F94DC0CF801858196810F942F0DBE01CD
:1014E000605E7F4FD80115968D919C910F94020DEF
:1014F000F801408168E4858196810F94DC0C64E1F9
:1015000070E080E090E00F94C925D8018C91882389
:1015100031F06AE070E080E090E00F94C925F801B6
:10152000858196810F942F0DD7011296ED90FC9036
:101530005BCF70E060E0CE0101960E94D9B08C01D3
:10154000912C812C97FF06C01195019511098824D3
:101550008394912CCE0101960E944CB8E82EF12C78
:101560008B85853091F0863009F00DCEB02E61E08C
:10157000802F0F94842361E0892809F443C0EA9402
:10158000EF2809F043C060E041C0EF2829F462E091
:10159000CE0101960E942DB840E050E160E070E07D
:1015A000CE0101960E94E1B18F819885892B41F08F
:1015B00040E050E260E070E0CE0101960E94E1B1AF
:1015C00061E0802F0F94842360E0802F0F945623D6
:1015D0006BE670E282ED9FE00E94AFF04AE050E0DF
:1015E000B80182ED9FE00E9450F066E670E282ED65
:1015F0009FE00E94AFF064E670E282ED9FE00E94FF
:10160000AFF0C1CDEA94EF2809F0BDCFE62EF12C62
:101610008B2D0F9456236FE570E282ED9FE00E94C0
:10162000AFF04AE050E0B80182ED9FE00E9450F038
:101630006DE570E282ED9FE00E94AFF04AE050E07D
:10164000B70182ED9FE00E9450F06BE570E2D5CFCC
:10165000F801868197819093C00A8093BF0A82ED3A
:101660009FE00E9443EF69E47FE185E29FE00E94F2
:10167000AFF085E29FE00E9443EFE091C30AF09152
:10168000C40A309709F4CFC08091C10A8F5F80935C
:10169000C10A068117815E01F8E2AF0EB11C8BEB27
:1016A000682E82E0782E99EA892E92E0992E011513
:1016B000110509F4B3C0D80118968C918F7086304B
:1016C00009F07CC019A708A770E060E0C5010E947E
:1016D000EAD68DA59EA5892B09F470C08091DB09FF
:1016E0009091DC09892B09F469C0E8A4F9A4E114FC
:1016F000F104B9F1F70180858F70863091F5F9A278
:10170000E8A270E060E0CE0180960E94EAD6EDA1EA
:10171000FEA1108211821282138260E276E0C7017C
:101720000F94F712FC01892BE1F090859F70955082
:101730009230B8F4C680D780C114D10491F0DA8217
:10174000C982B701CE0101960E94EAD6EE81FF81DF
:101750001082118212821382D6011296CD90DC90F3
:10176000EBCF64E47FE182ED9FE00E94AFF04AE0BE
:1017700050E06BA582ED9FE00E9466EF62E47FE19E
:1017800082ED9FE00E94AFF04AE050E06AA582ED52
:101790009FE00E9466EF82ED9FE00E9443EFEDA57F
:1017A000FEA510821182128213828AA5853069F10A
:1017B00048F48230F0F060E08430E0F0F80102811B
:1017C000138175CF8032A9F058F48630B9F7BC8206
:1017D000AB829A828982CE0101960E94CA6BEECFBB
:1017E000803489F060E0823449F78BA50F9484231C
:1017F000E5CF62E08BA50F948423EDA5FEA5818142
:10180000807F8183DBCF62E0F0CFBC82AB827A82C3
:101810006982CE0101960E94796CD0CF8091C10A75
:1018200081508093C10A65E37FE185E29FE00E94D9
:10183000AFF06DE27FE185E29FE00E94AFF081E0D2
:101840002091C50A3091C60A232B09F480E00E943A
:10185000586864E27FE185E29FE00E94AFF081E09A
:101860002091C30A3091C40A232B09F480E00E941E
:10187000586865E17FE185E29FE00E94AFF06AE091
:101880007FE185E29FE00E94AFF081E02091C709EF
:101890003091C809232B09F480E00E94586863E066
:1018A0007FE185E29FE00E94AFF081E020914E0A47
:1018B00030914F0A232B09F480E00E9458686AEFA8
:1018C0007EE185E29FE00E94AFF081E02091C70AAF
:1018D0003091C80A232B09F480E00E94586885E201
:1018E0009FE00E9443EF65EF7EE185E29FE00E946A
:1018F000AFF00E94B032AB01BC012AE030E085E2DB
:101900009FE00E945EEF85E29FE00E9443EF81E04E
:101910008093530A84EF9EE00F94AC00882351F02B
:1019200084EF9EE00F94640784E090E090933B0C7A
:1019300080933A0C80913A0C90913B0C079731F4CC
:1019400084E090E090933B0C80933A0C8091C10A24
:1019500081508093C10A8091530AAE960FB6F894D5
:10196000DEBF0FBECDBFDF91CF911F910F91FF90D2
:10197000EF90DF90CF90BF90AF909F908F907F902F
:101980006F90089580E0E9CFFCE0FA1508F412CDDD
:1019900036CD8F929F92AF92BF92CF92DF92EF920D
:1019A000FF920F931F93CF93DF93CDB7DEB7CF5541
:1019B000D1090FB6F894DEBF0FBECDBF8C016B010D
:1019C0006115710519F04115510579F567E078E168
:1019D00082ED9FE00E94AFF06EEF77E182ED9FE035
:1019E0000E94AFF0B80182ED9FE00E9499F06CEF89
:1019F00077E182ED9FE00E94AFF082ED9FE00E94D0
:101A000043EFC15ADF4F0FB6F894DEBF0FBECDBF14
:101A1000DF91CF911F910F91FF90EF90DF90CF90CA
:101A2000BF90AF909F908F900895460F571FDA0197
:101A30001C920E94B0324B0166EF77E182ED9FE08D
:101A40000E94AFF04AE050E0B40182ED9FE00E94B6
:101A500050F063EF77E182ED9FE00E94AFF0B801B4
:101A600082ED9FE00E9499F060EF77E182ED9FE0C8
:101A70000E94AFF0BAE38B16B1E09B064CF463EE24
:101A800077E18DE29FE00E94AFF08DE29FE0B7CF5B
:101A900061EE77E182ED9FE00E94AFF0B60182ED4A
:101AA0009FE00E9499F06FED77E182ED9FE00E9448
:101AB000AFF082ED9FE00E9443EF1A821982FE018F
:101AC00033968EE3DF011D928A95E9F780913A0CF7
:101AD00090913B0C059791F563E070E0C8010E947E
:101AE000AC707C01892BD1F5E091AF0DF091B00D78
:101AF000808180FF86CF61E070E0C8010E94AC70F9
:101B0000892B09F47ECF64E270E0C8010F94084C81
:101B1000892B09F076CF61EC77E182ED9FE00E949E
:101B2000AFF0B80182ED9FE00E9499F082ED9FE056
:101B30000E9443EFC8010F944A2263CF61E070E036
:101B4000C8010E94AC707C01892B09F465C04FE389
:101B500050E0B801CE0101960F94F94BA12CBB24A3
:101B6000B394E00EF11E68EB77E1C7010F94CD3F0F
:101B7000892B09F45EC064E270E0C8010F94084C40
:101B8000892B09F03ECFB11003C0AA2009F439CF48
:101B90004091C50A5091C60AB701CE018F5B9F4F95
:101BA0000E9498B8CE018F5B9F4F0E94BCAF182F48
:101BB000882359F0B601CE018F5B9F4F0F94F31B22
:101BC00011E0181619060CF010E0CE018F5B9F4F44
:101BD0000E9435B9112309F414CF8981882309F4AF
:101BE00010CF80913A0C90913B0C059709F409CFE6
:101BF0006AE977E182ED9FE00E94AFF0BE016F5F7E
:101C00007F4F82ED9FE00E9499F082ED9FE00E945D
